:100000000C94B2150C94C7F00C949CF00C9471F005
:100010000C9446F00C941BF00C94F0EF0C94C5EF8C
:100020000C949AEF0C94E3150C94E3150C94E315DF
:100030000C94E3150C94E3150C94E3150D9404074C
:100040000C94E3150C94E3150C94E3150C94E31550
:100050000C94E3150C94E3150C94E3150C9405EE45
:100060000C94E3150C9407F40C94DDF30C94E31555
:100070000C94E3150C94E3150C94E3150C94E31520
:100080000C94E3150C94E3150C94E3150C94E31510
:100090000C9463F50C94D9F40C941BF50D94CA0BD5
:1000A0000C94E3150C94E3150C94E3150C94E315F0
:1000B0000C94E3150C94E3150C94E3150C94E315E0
:1000C0000C94E3150C94E3150C94E3150C94A7F32E
:1000D0000C947DF30C94E3150C94E3150C94E31548
:1000E0000C94E31507634236B79BD8A71A396856B4
:1000F00018AEBAAB558C1D3CB7CC5763BD6DEDFD4A
:10010000753EF6177231BF000000803F0800000006
:10011000BE922449123EABAAAA2ABECDCCCC4C3EFC
:1001200000000080BEABAAAAAA3E00000000BF00EB
:100130000000803F0000000000084178D3BB4387E7
:10014000D1133D190E3CC3BD4282AD2B3E68EC82FB
:1001500076BED98FE1A93E4C80EFFFBE01C4FF7F80
:100160003F00000000000C943A730C9459D40C9496
:10017000BD240C94FCEC0C9432760D945D020C942E
:10018000762F0C949C930C9442180D94E8040C94D4
:100190007A860C9409F80C9499250C9499340C9453
:1001A000A9750C94EDEB0C94BE340C9443C80C94DC
:1001B000A51E0C944AC80C9459850C9420C80C9424
:1001C000FAFB0C94BD770C945F7C0D947D060C9427
:1001D000A7590C94A7450C94DECE0C94421F0C94A6
:1001E000D7E80C9465810C94B68A0C94A8AA0C9458
:1001F00059320C9426D00C94C1CF0C94AC160C94AC
:10020000C9770C94E6C10C9468EB0C9427250C94E8
:10021000621F0C9496E90C94701E0C9488250C9423
:10022000ECCE0C94F5C10C9427C80C94E47C0C948F
:10023000AB340C9419FB0C94D0A40C9465200C9452
:10024000B7870C9478180C942BC20C94321E0C9423
:100250001FA40C94266E0C9447730C94131D0C94DD
:1002600008990C947C770C94274B0C9400760C9492
:100270007A4B0C94E1450C94A52F0C94604B0D9493
:100280002E050C94ED240C9436720C943D7B0C944A
:10029000D4C10D94C5040C940D850C9482160C9455
:1002A0006C250C9492240C9405750D94D0020C943A
:1002B000D1CF0C9408D00C9430260C94C24B0C94E3
:1002C000E6A60C94429E0C94C61C0C94FA750C94F1
:1002D000C5770C94D9860C9424E90C94FECF0C9429
:1002E000331F0C940DEC0C947C240C94AFEA0C940A
:1002F000E1770C94C1580C94D4E90C9466730C9477
:10030000EDEA0C9425EA0C9474810C9473500C94CF
:10031000FBA60C949A750C9472390C9453320C947D
:100320003E220C94ED4A0C9486160C94CB180C9437
:1003300002750C941F6E0C94025A0C94C0590C94C4
:1003400040930C9437E80C94C3980C9477EB0C947E
:10035000D1A40C94F5EA0C9479A10C94A9250C94E1
:1003600001AB0C9435C80C9438450C94EFCF0C9429
:1003700042210C94DBCF0C94B7CF0C94464B0C94D9
:100380008A870C9475D40C9424FC0C94C1770C943B
:10039000EA230C94DA1C0C94D0F70C94CC160C9431
:1003A000284A0C94C6CE0C94DB980C94D6750C9409
:1003B00084ED0C948EEA0C94AF330C94E5CF0C943E
:1003C0005A210C94241F0C94ADCF0C94B2980C9429
:1003D00035E80C94BDCE0C9437930C94D6250C9430
:1003E00087340C9443ED0C948A160C94F7580C94B3
:1003F000A9330C949DEA0C94F15A0C9480A50C94AA
:10040000211D0C9486200C9467EB0C945DF90C94E0
:10041000B1CE0C949E7F0C948DED0C9467190C94C6
:1004200084280C94CD5A0C9407810C94E8160C94F3
:1004300074FE0C944C4D0C9487E90C94ED230C94B1
:10044000B9CE0C94EE340C94F8340C94326E0C94B7
:10045000464D0C947E340C94DE170C94C9EA0C942F
:100460001D340C94484D0C94E2EA0C948B740C945B
:1004700014C20C94417B0C948F930C9422310C94F5
:10048000B0A70C94B3E90C94C3A70C94C3320C949A
:100490008B980C9436E80C9451760C9466EB0C9483
:1004A0003D5A0C9491EB0C94FF1D0C9478FE0C9427
:1004B000DA920C9446590C9450320C94A44B0C9440
:1004C00034E80C94E4340C94F2860C9429170C94C0
:1004D000682F0C94E2E90C94EA7D0C94D8CE0C942D
:1004E00058D40C9452250C94147D0C9431A10C9486
:1004F000B5CE0C94B22F0C9403240C942F1C0C94A6
:10050000BC320C9407450C9478D40C94D05A0C94BB
:10051000CACE0C94691F0C949E980C942D1D0C94BB
:1005200011780C9435730C943BAA0C94E0EA0C946B
:10053000F7BA0C946C210C9427760C94CB770C941E
:1005400013170C948D220C94E6CE0C94DBFB0C94C8
:10055000AE4B0C9472A00C946C1C0C9445760C94CD
:1005600069ED0C9448250C9441F70C94AA250C9441
:100570002D590C9464E80C9424760C9495E80C9412
:1005800012D00C94B5230C94B2330C9490340C9488
:100590009ECF0C9496770C9486810C946F1F0C94CC
:1005A00098A00C94AC180C94BEEB0C94717B0C943A
:1005B00000170C94C0CE0C9496CF0C9406300C947B
:1005C000097D0C94ED1C0C9472F70C9436170C9466
:1005D000BFED0C94147C0C94EF970C943B1F0C947F
:1005E0009A4B0C942E220C94806E0C9471240C94D3
:1005F000ED160C94F0CE0C94871F0C94245A0C9496
:10060000DC730C9492160C94A8220C941B1F0C946F
:1006100070200C94D9250C948E6C0C942EC80C94DC
:1006200014870C94D4CE0C94EBCE0C94BF770C941E
:10063000EA160C940B370C9426FB0C94C2730C94A2
:100640005BF70C942B1E0C940F660C9421300C94C9
:100650008E160C94C9FF0C94A3CF0C9451C80C9423
:1006600052F70C94C5EA0C947A250C94AE240C94A1
:100670007A590C941EEA0C9499380C94FD750C94DC
:10068000AC330C94C19F0C94E2CE0C94D0CE0C945D
:1006900022940C94C3770C94D0230C94B7330C940D
:1006A000B4A60C947C500C941E210C94674A0C94B4
:1006B000C4220C94D1340C940CEB0C9492FE0C9448
:1006C000725A0C94968F0C943B7A0C9474980C94F8
:1006D00011250C94A21E0C94781F0C9485A50C94E3
:1006E000839F0C94BB770C9404950C9485A00C9478
:1006F000FA340C949A160C9405900C94D9EA0C9444
:100700007F200C948AA40C9496380C9432850C9417
:100710004B810C94E4160C94041D0C94101D0C9445
:10072000C1210C9482500C94DD240C9487E80C9425
:1007300020A40C94219D0C94E4870C9425EC0C943B
:1007400065980C9489F20C949FF10C94E0840D94BC
:10075000CA130D94DF130C94ABCE0C9403760C9457
:1007600096160C94D9750C94C7770C9421A40C940C
:10077000BEF70C9414460C9410260C94D6160C94C8
:1007800071EC0C9443980C94C9CF0C94CDC10C948B
:1007900030D00C940C750C94882F0C94457B0C94E1
:1007A0008AEB0C94E9730C94472F0C941EA40C94C0
:1007B000F6EA0C945B2F0C9473E80C94B24A0C94F8
:1007C000BB240C94BA1D0C9496A50C947D790C94C2
:1007D00094250C941E1D0C94E5150C940CEA0C94B5
:1007E0001CD00C94CA5A0C945A204E414E494E4982
:1007F0005459494E46CDCCCC3D0AD7233C17B7D1EE
:100800003877CC2B329595E6241FB14F0A00002093
:10081000410000C84200401C4620BCBE4CCA1B0E12
:100820005AAEC59D746364696E6F70737578585B5A
:1008300000556E6B6E6F776E2073756666697820F3
:1008400000556E6B6E6F776E20636D642000636C75
:10085000724374723A2000454F46002F00496E3AA9
:1008600020003D00494E3A003D004C454741435968
:1008700020494E3A002500C2B04320483D002044A4
:100880004854323220747970652E20543D00494E10
:100890003A00204E6F20656D697420646174612197
:1008A0000020436F756E74657220747970652E2018
:1008B00076616C3D00494E3A0020436F756E746559
:1008C0007220747970652E20494E434F5252454331
:1008D0005420496E74657272757074206E756D6205
:1008E0006572212121004952513A002D3E0020001D
:1008F00023002D3E00200050656E6465643A20237D
:1009000000536574436D643A007375666669784395
:100910006F64653A0020666F7220286D73293A0073
:100920004354524C3A205363686564756C65206388
:100930006D642000206D73203A0041726D65642063
:10094000666F7220002044697361726D65640020D7
:1009500074696D653A004354524C3A205265733ABB
:10096000003D0050696E3A004354524C3A20436FA8
:100970006D6D616E6420626C6F636B65642062797B
:1009800020647269766572206F72206368616E6E92
:10099000656C2066726F7A656E004354524C3A2043
:1009A0004F4E3A416C726561647920416374697697
:1009B000650A004354524C3A2048414C543A416C29
:1009C000726561647920496E6163746976650A00B5
:1009D0004354524C3A20584F4E3A20446973616256
:1009E0006C65640A004354524C3A20584F4E3A41C9
:1009F0006C7265616479204163746976650A0043AD
:100A000054524C3A20584F464620736B69707065BB
:100A1000642E205072657620636D643A0043545210
:100A20004C3A205475726E6564206F66662066725B
:100A30006F6D3A004354524C3A20526573746F7292
:100A400065642066726F6D3A004354524C3A2049F7
:100A5000676E6F7265642C206368616E6E656C20D2
:100A6000636D643D0020457865633A004354524C01
:100A70003A204163746976653A004354524C3A20F7
:100A800048414C543A416C726561647920496E6109
:100A900063746976650A004354524C3A20584F4EAD
:100AA0003A2044697361626C65640A004354524C95
:100AB0003A20584F4E3A416C726561647920416327
:100AC000746976650A004354524C3A20584F4646A2
:100AD00020736B69707065642E2050726576206398
:100AE0006D643A004354524C3A205475726E6564FA
:100AF000206F66662066726F6D3A004354524C3A1E
:100B000020526573746F7265642066726F6D3A006F
:100B10004354524C3A204E6F7420656E6F7567686F
:100B2000206D656D6F727920666F722067726F75C8
:100B300070206F7065726174696F6E00496E7661C6
:100B40006C69642061726700496E76616C6964202B
:100B5000617267004354524C3A20556E6B6E6F774A
:100B60006E2073756666697800536B697070656492
:100B700020686F6D696520737475666600200020BB
:100B80005375623D00204974656D3D004354524CDD
:100B90003A2052414D3D004354524C3A204F757417
:100BA0004F664D656D6F72793A2000282D2920001F
:100BB000282B2920002076616C7565206973200040
:100BC00020756E6B6E6F776E0A005D3D005B0020D6
:100BD000696E76616C6964002000206F6B003A00DA
:100BE000206661696C6564003A00526574727969C7
:100BF0006E6720564354454D5020434D440A0052E1
:100C000065747279696E6720564320434D440A002B
:100C10005265747279696E67206D6F6462757320B6
:100C2000434D440A005265747279696E6720434DE2
:100C3000440A00206572726F723D004D423A207086
:100C40006F6C6C696E6720002056616C3A20004D15
:100C5000423A20004D423A204E6F742073757070F6
:100C60006F727465642072656720747970650A001C
:100C70004D423A20706F6C6C696E672064696D6DCF
:100C8000657220004D423A20496C6C6567616C20AA
:100C9000617267756D656E74730A00206572726F9C
:100CA000723D004D423A20706F6C6C696E67205047
:100CB0004920002D004D423A2050492056616C20B9
:100CC0003A004D423A20706F6C6C696E6720504953
:100CD00020004D423A20706F6C6C696E6720464D63
:100CE000206661756C742000206572726F723D0021
:100CF0004D423A20706F6C6C696E6720002D004D7C
:100D0000423A20464D2056616C203A004D423A202E
:100D1000706F6C6C696E6720464D20004354524CD6
:100D20002F706F6C6C3A204F75744F664D656D6F08
:100D300072793A2000207365632072656D61696E77
:100D4000696E6700537461747573206465666665C7
:100D50007265640A002D3E005075623A20002D3EF7
:100D6000005075623A20002D3E005075623A200016
:100D70000000000000636D6400007365740000767D
:100D8000616C000064656C000048535600005247D7
:100D900042000066616E00006D6F646500637472EE
:100DA0006C006875650000736174000074656D7097
:100DB0000072617700002D3E005075623A20002DD0
:100DC0003E005075623A2000556E6B6E6F776E2054
:100DD000636D64200A000000000000000000004F66
:100DE0004E000000000000004F46460000000000DA
:100DF00000524553540000000000544F47474C45F3
:100E000000000048414C540000000000584F4E00C4
:100E10000000000000584F46460000000000494E08
:100E200043524541534500444543524541534500D3
:100E3000454E41424C4500000044495341424C4517
:100E40000000554E465245455A4500465245455AC2
:100E5000450000004155544F000000000046414E3F
:100E60005F4F4E4C59004849474800000000004D74
:100E7000454449554D0000004C4F5700000000000C
:100E800000484541540000000000434F4F4C000013
:100E900000000044525900000000000053544F501D
:100EA00000000000005247420000000000004853CC
:100EB00056000000000000206661696C65643A001D
:100EC0004D6F64627573206F7020004D423A206F41
:100ED0006B003D004D423A205643230020636D6471
:100EE0003D003D004D423A2056435F6865617423E2
:100EF000004D423A204E6F7420737570706F72749B
:100F000065642072656720747970650A00205661F7
:100F10006C3A30780020543A00205265673A3078B5
:100F2000004D423A20416464723A00444D5800003A
:100F300000000000444D58524742570000444D58AD
:100F400052474200000050574D0000000000004D85
:100F500042555344494D0000544845524D4F0000FE
:100F60000052454C41590000000047524F55500077
:100F7000000000564354454D500000004D4255536B
:100F80005643000000414348414945520000535038
:100F9000494C45440000004D4F544F5200000000A2
:100FA0005049440000000000004D4255530000002D
:100FB000000055415254425244470052454C415959
:100FC00050574D00444D5852474257570056454ED2
:100FD000545300000000454C455641544F520043C5
:100FE0004F554E544552000048554D00000000003A
:100FF000004D455243555259000020002D3E0043FC
:101000006F6E76657274696E6720002D3E005772B0
:101010006F6E672041737369676E6D656E74200033
:10102000524742783A200020764C6576656C3A004B
:1010300020436F6E76563A0020436F6E76533A0027
:1010400020486F743A00436F6C643A0020436F6E1F
:1010500076657274656420563A00436F6E766572E9
:1010600074656420533A002D3E0057726F6E6720FE
:1010700041737369676E6D656E7420002D3E005775
:10108000726F6E672041737369676E6D656E742051
:101090000053617665643A00000000000000000023
:1010A000004F4E000000000000004F4646000000C8
:1010B000000000524553540000000000544F4747C1
:1010C0004C4500000048414C540000000000584FBF
:1010D0004E000000000000584F464600000000008F
:1010E000494E4352454153450044454352454153BF
:1010F0004500454E41424C450000004449534142A1
:101100004C450000554E465245455A45004652450D
:10111000455A450000004155544F0000000000466C
:10112000414E5F4F4E4C590048494748000000006F
:10113000004D454449554D0000004C4F57000000FC
:10114000000000484541540000000000434F4F4C50
:1011500000000000004452590000000000005354F9
:101160004F50000000000052474200000000000005
:1011700048535600000000000020537566663A0090
:101180002041543A00206973200044656C657469FD
:101190006E6720636F6E662E2052414D207761731B
:1011A0003A0053746F70706564006E6F7468696E96
:1011B0006720746F2073746F700053746F70706960
:1011C0006E67206368616E6E656C73202E2E2E0034
:1011D0004E6F7420756E6C6F636B656420696E2052
:1011E000313073202D20636F6E74696E7565202E0B
:1011F0002E2E00556E6C6F636B696E6720636F6E89
:10120000666967202E2E2E00436F6D706C657465C5
:101210002E2052656D6F766520746F7069632000B3
:1012200024636F6D6D616E6400536B697070696EDD
:10123000672E2E00436C65616E5570207265746177
:10124000696E656420746F7069632000220022005B
:101250004F75744F664D656D6F727921005D20008A
:101260003A5B000A005D00456D7074793A205B00BE
:101270000A003A004D41433A0055445020537973D7
:101280006C6F6720696E697469616C697A65642E38
:101290000A005379736C6F6720706172616D733AE5
:1012A000002E6C6F63616C00536572766963652014
:1012B0007265636F72643A20006D444E532072650C
:1012C00073706F6E64657220737461727465642EDE
:1012D000004572726F722073657474696E67207551
:1012E00070204D444E5320726573706F6E6465724A
:1012F0002100476F742049502061646472657373E4
:101300003A00276970205B69705B2C646E735B2CFC
:1013100067775B2C7375626E65745D5D5D5D27201C
:101320002D20736574207374617469632049500AB9
:10133000004661696C656420746F20636F6E666936
:10134000677572652045746865726E657420757383
:10135000696E6720444843502E20596F75206361A1
:101360006E20736574206970206D616E75616C6CA0
:10137000792100204D41534B3A002047573A002035
:10138000444E533A004C6F616465642066726F6D21
:1013900020666C6173682049503A000A7573657362
:1013A00020444843500A005374617274696E672088
:1013B0006C616E00546F6F206D616E79204D5154D9
:1013C0005420636F6E6E656374696F6E2065727210
:1013D0006F72732E2052657374617274204C414E8B
:1013E000002074727920616761696E20696E203512
:1013F000207365636F6E6473006661696C65642C4D
:101400002072633D004177616974696E6720666F81
:10141000722072657461696E656420746F706963AF
:101420007300636F6E6E6563746564206173200082
:10143000202E2E2E0020757365723A003A000A4164
:101440007474656D7074696E67204D5154542063D7
:101450006F6E6E656374696F6E20746F20006469CF
:1014600073636F6E6E6563746564005573696E6750
:10147000204D5154542070617373776F72642066ED
:10148000726F6D20636F6E666967002E6C6F6361AB
:101490006C006D444E53206E616D65207570646103
:1014A0007465643A2000446576696365204E616D19
:1014B000653A004174206C656173742064657669D7
:1014C0006365206E616D6520616E642062726F6B72
:1014D0006572204950206D75737420626520636FBA
:1014E0006E6669677572656400757074696D652CE8
:1014F00066726565686561700034643930396464AA
:101500005F323032332D31312D3230004C69676813
:10151000744875622000246E616D650052656269D1
:101520006E6420737563636573732E204950206168
:101530006464726573733A004572726F723A207216
:101540006562696E64206661696C0052656E6577DC
:10155000656420737563636573732E204950206141
:101560006464726573733A004572726F723A2072E6
:10157000656E65776564206661696C000A4E6F2050
:101580006C696E6B0033307320454550524F4D20CF
:101590006973206E6F742072656C6F616465642E70
:1015A000205265626F6F7400416363657074696E89
:1015B0006720636F6D6D616E64732E2E2E0A004E70
:1015C0006F204D51545420636F6E66696775726564
:1015D00064004C6F6164696E6720636F6E66696753
:1015E0002066726F6D20706F7274616C2064697315
:1015F00061626C65642E2075736520676574204F89
:101600004E20746F20656E61626C6500436F6E667C
:1016100069672069732076616C696400436F6E743A
:10162000696E756520776974682070726576696F78
:1016300075736C79206C6F6164656420636F6E668E
:1016400069670043757272656E74204C414E206369
:101650006F6E6669672869702C646E732C67772CCF
:101660007375626E6574293A000A55736520746853
:1016700065736520636F6D6D616E64733A202768D2
:10168000656C7027202D20746869732074657874E8
:101690000A276D61632064653A61643A62653A6560
:1016A000663A66653A3030272073657420616E644F
:1016B0002073746F7265204D41432D6164647265BF
:1016C000737320696E20454550524F4D0A2769704B
:1016D000205B69705B2C646E735B2C67775B2C738B
:1016E00075626E65745D5D5D5D27202D2073657488
:1016F000207374617469632049500A2773617665A9
:1017000027202D20736176652063757272656E7473
:1017100020636F6E66696720696E204E5652414D98
:101720003B204F4E7C4F4646202D20656E61626CFB
:10173000652F64697361626C65206175746F736194
:1017400076650A2767657427205B636F6E66696735
:1017500020616464725D27202D2067657420636FAB
:101760006E6669672066726F6D207072652D636F9B
:101770006E666967757265642055524C20616E64AF
:101780002073746F726520616464722C204F4E7CEC
:101790004F4646202D20656E61626C652F6469732B
:1017A00061626C6520646F776E6C6F6164206F6E30
:1017B00020737461727475700A276C6F61642720DE
:1017C0002D206C6F616420636F6E6669672066729E
:1017D0006F6D204E5652414D0A2770776427202D99
:1017E00020646566696E6520616E642073746F7233
:1017F00065204D5154542070617373776F72640A81
:10180000276F746170776427202D20646566696E88
:101810006520616E642073746F7265204854545063
:10182000204150492070617373776F72640A276C8E
:101830006F67205B73657269616C5F6C6F676C6565
:1018400076656C5D205B7564705F6C6F676C657648
:10185000656C5D27202D20646566696E65206C6F60
:1018600067206C6576656C2028302E2E37290A2774
:101870006B696C6C27202D207465737420776174FC
:101880006368646F670A27636C65617227202D2087
:10189000636C65617220454550524F4D0A27736550
:1018A0006172636827202D2073656172636820313F
:1018B0002D77697265206465760A277265626F6F9D
:1018C0007427202D207265626F6F7420636F6E74B1
:1018D000726F6C6C657200536F6674207265626F14
:1018E0006F74696E672E2E2E00206E65770020695A
:1018F0007320003157543A003157543A20536561F0
:10190000726368696E67206465760052414D3D00E0
:101910000A5379736C6F6720000A312D77697265FD
:1019200020000A6D71747420000A6D6F6462757313
:10193000207632000A6D6F6462757320763120283C
:101940002B29000A696E7075747320000A6974652A
:101950006D7320000A436F6E666967757265643A3D
:1019600000496E697469616C697A696E6720496EB5
:1019700070757473003157543A2073657475702014
:101980007265736F6C7574696F6E20003157543ACD
:10199000204453323438322D313030206E6F742071
:1019A00070726573656E74003157543A2044533237
:1019B0003438322D3130302049324320726573740F
:1019C0006F726564003157543A2042757320726516
:1019D000736574206572726F72003157543A2042F9
:1019E000757320526573657420646F6E650031579E
:1019F000543A204453323438322D31303020707212
:101A00006573656E742C207265736574004572721F
:101A10006F7220312D7720696E6974003157543A06
:101A2000204453323438325F3130305F4932435FC3
:101A3000544F5F31575F42524944474520696E69B0
:101A40007400444D584F75742E20467265653A00F7
:101A5000444D58696E2042756666657220616C6CF3
:101A60006F632065727200496E697420696E20632D
:101A7000683A003B003D0050696E3A003B003D4C27
:101A80004F5700546865726D6F3A004F6E6520774E
:101A90006972652052656164790A00467265653A2B
:101AA00000444D58206F75742073746172746564BE
:101AB0002E204368616E6E656C733A2000444D5869
:101AC00020696E20737461727465642E20436861AE
:101AD0006E6E656C733A004170706C79696E672048
:101AE000636F6E66696700436F6E66696720617534
:101AF000746F736176653A000A5379736C6F67206F
:101B00006465627567206C6576656C3A0053657232
:101B100069616C206465627567206C6576656C3AF6
:101B20000053617665640A005365742064796E61C0
:101B30006D69632049500A00454550524F4D20635E
:101B40006C65617265640A004D5154542050617394
:101B500073776F726420757064617465640A004FF6
:101B600054412050617373776F72642075706461A3
:101B70007465640A00636F756C64206E6F74207006
:101B8000617273653A2000557064617465640A007F
:101B90004E6F204950206164726573730052656C0A
:101BA000656173696E6720736F636B657420616E26
:101BB0006420726574727900205361766564004C0C
:101BC0006F6164696E67204854545020636F6E667D
:101BD0006967206F6E20737461727475703A0000CB
:101BE00000000000000000004F4E00000000000058
:101BF000004F4646000000000000524553540000CC
:101C0000000000544F47474C4500000048414C54E9
:101C10000000000000584F4E000000000000584F28
:101C200046460000000000494E43524541534500DE
:101C3000444543524541534500454E41424C4500C1
:101C4000000044495341424C450000554E46524520
:101C5000455A4500465245455A45000000415554F5
:101C60004F000000000046414E5F4F4E4C59004867
:101C700049474800000000004D454449554D0000CB
:101C8000004C4F5700000000000048454154000040
:101C9000000000434F4F4C00000000004452590028
:101CA000000000000053544F500000000000524755
:101CB00042000000000000485356000000000000F1
:101CC0002B002D00455461673A200047657420457C
:101CD0005441473A2000485454502F312E310025AA
:101CE000733A2025730D0A0020485454502F312E8A
:101CF000310D0A486F73743A2025730D0A416363EE
:101D00006570743A202A2F2A0D0A436F6E6E656340
:101D100074696F6E3A20636C6F73650D0A002573EA
:101D20000020000D0A00474554006661696C656437
:101D300020746F20636F6E6E6563740A00455252A3
:101D40004F523A20536572766572207265747572CF
:101D50006E65642000436F6E666967206E6F742045
:101D60006368616E6765640A00446F6E652E0A00E1
:101D7000436F6E6669672070617273696E67206673
:101D800061696C65640A00676F7420436F6E6669F1
:101D9000670A006874747020726574636F646520EC
:101DA00000667265652000436F6E66696720555254
:101DB000493A20687474703A2F2F00204465666198
:101DC000756C7420636F6E666967207365727665E3
:101DD0007220757365643A20006C617A79686F6D62
:101DE000652E7275000A282D294D455243555259CA
:101DF000000A282B294D554C544956454E54000A8B
:101E0000282B2950574D5F52454C4159000A282B29
:101E1000294D444E53000A282D295541525442520F
:101E200049444745000A282B295359534C4F470032
:101E30000A282B29504944000A282D294D435032A5
:101E400033303137000A282D294152544E45540071
:101E50000A282D294F5441000A282D295350492082
:101E60004C4544000A282B294D4F544F52204354CF
:101E700052000A282D294143204841494552000A71
:101E8000282D2943435338313120262048444331FB
:101E9000303830000A282B29524553544152545FA0
:101EA0004C414E5F4F4E5F4D5154545F4552524F1F
:101EB0005253000A282D2948415244524553455453
:101EC0002C207573696E6720736F6674000A282B67
:101ED00029434F554E544552000A282B2944485453
:101EE000000A282B294453323438322D3130300047
:101EF0000A282B294F57495245000A282D294950B5
:101F00004D4F44425553000A282B294D4F4442550A
:101F10005320307830362061742053657269616CCB
:101F2000322073706565643A39363030000A282BE8
:101F3000294144414652554954204C4544000A2801
:101F40002B29444D58000A282B2957697A4E65746D
:101F500035353030000A282B294672656552616D8F
:101F6000207072696E74696E67000A282B295741C8
:101F7000544348444F47006C617A79686F6D652E11
:101F80007275000A436F6E666967207365727665C5
:101F9000723A003230313130334C0020432B2B2049
:101FA00076657273696F6E3A0034643930396464EF
:101FB0005F323032332D31312D3230000A4C617AAC
:101FC00079686F6D652E7275204C69676874487505
:101FD0006220636F6E74726F6C6C65722000204FAC
:101FE000464600204F4E0020425950415353007244
:101FF0006561647900247374617465007570746937
:102000006D65006672656568656170002473746152
:102010007473002054696D65723A00204C6F636BD5
:10202000733A002000204C6F636B733A000A5241F0
:102030004D3D0020457870697265640A00202D745A
:102040006172676574207A6F6E652D0020416C6146
:10205000726D20457870697265640A0020636D6452
:102060003A00204375723A00205365743A00536178
:1020700076656420746F20454550524F4D00536182
:1020800076696E6720636F6E66696720746F20459E
:102090004550524F4D2E2E004C6F616465642045B3
:1020A0005441473A004E6F2073746F726564206329
:1020B0006F6E666967004C6F616465642066726F5D
:1020C0006D20454550524F4D006C6F616420666134
:1020D000696C6564004A534F4E206465746563748F
:1020E0006564004C6F6164696E6720436F6E66695A
:1020F000672066726F6D20454550524F4D00556EFA
:102100006B6E6F776E207375666669782000556E0A
:102110006B6E6F776E20636D642000436F756E7415
:1021200065723A2000444D582D4F757420496E69F0
:10213000743A2000444D582D4F75742073746F709D
:102140003A200041737369676E65643A00444D58E4
:10215000206374726C3A20006931360001693332B1
:1021600000027531360003753332000469386800A7
:102170000569386C0006753868000775386C00080A
:102180007831300009313030000A44656661756C81
:10219000742073657269616C206D6F6465204E38C0
:1021A00031207573656400384531002600384E31A2
:1021B000000600384532002E00384E32000E00383E
:1021C0004F31003600384F32003E00374531002491
:1021D00000374532002C00374F31003400374F3282
:1021E000003C00374E31000400374E32000C004DE9
:1021F0004255533A204D6F646275732074656D705B
:102200006C617465206E6F7420666F756E643A2021
:10221000004D4255533A20496E76616C69642074D2
:10222000656D706C6174652E002C002C002C002CE8
:10223000004D4255533A20636F6E666967206661B0
:10224000696C65643A004D4255533A20636F6E667F
:102250006967206572726F72004D4255533A206370
:102260006F6E666967206C6F6164656420004D4223
:1022700055533A204F7574206F66206D656D6F72EF
:1022800079004D4255533A20506F6C6C696E67204F
:102290006572726F7220004D425553443A2049676F
:1022A0006E6F726564202D20657175616C20776991
:1022B0007468207365747465642076616C004D42A7
:1022C00055533A204164642040533A20004D425512
:1022D00053443A204D61707065643A004D42555345
:1022E000443A204E65737465644D61707065643A5C
:1022F000004C6173744B6E6F776E2076616C756500
:102300003A2000536561726368696E672072656781
:102310003A200072656723206F7574206F66207203
:10232000616E676500536561726368696E672072EC
:10233000656723003A002066726F6D2074797065BE
:1023400020004D425553443A2020676F74200020EE
:1023500076616C3A0020005265733A200020696E65
:102360007465726E616C2073656E64206572726F45
:1023700072202D206E6F207265672F636F696C006D
:1023800020696E7465726E616C2073656E64206581
:1023900072726F72202D206E6F2074656D706C618B
:1023A00074650020696E7465726E616C2073656E71
:1023B00064206572726F72202D206E6F2073746FAF
:1023C0007265004D425553443A20656E64506F6CFF
:1023D0006C20004D425553443A20506F6C6C2000E5
:1023E000206E6F7420666F756E64004D4255533ACF
:1023F0002020706172616D20002073656E6420651D
:1024000072726F722E20004D4255533A20200041C7
:1024100064642040563A20002056616C3A20004DFA
:10242000425553443A207375666669783A00206FC6
:10243000722073756666697820004D4255533A20C4
:102440004E6F2074656D706C61746520666F7220CC
:10245000004D6F746F723A2074696D656F7574000A
:10246000556E6B6E6F776E20636D64004D6F746F89
:10247000723A20466F72636564206578656375748F
:10248000696F6E004D756C746956656E7420636F6C
:102490006E666967206661696C6564004D756C7471
:1024A0006956656E7420696E6974004D756C746947
:1024B00076656E742044652D496E697400204F75F1
:1024C000743A00206D33002066726F6D2000204D3D
:1024D000617820726571756573743A002066616E6B
:1024E000253A002061637469766520563A00546F7E
:1024F00074616C20563A005049443A20616C726510
:1025000061647920696E697469616C697A656400D7
:102510005049443A20496E76616C6964207061725A
:10252000616D2061727261792E002C002C002C00EC
:102530002C005049443A20636F6E666967206661DB
:10254000696C65643A005049443A20636F6E66696D
:1025500067206572726F72005049443A20636F6E53
:10256000666967206C6F6164656420005049443A75
:10257000204F7574206F66206D656D6F7279005005
:1025800049443A2044652D496E69742000203C413D
:102590004C4D3E0020443A0020493A0020503A0079
:1025A00020696E3A00207365743A005049443A201D
:1025B000005049443A20496E76616C69642070612C
:1025C00072616D2061727261792E00536574206FA3
:1025D000757420746F20002050494420616C617232
:1025E0006D2E20002050494420616C61726D3A20AC
:1025F000636C6F736564005049443A20556E6B6E8E
:102600006F776E2073756666697820005049443A8A
:1026100020556E6B6E6F776E20636D6420002053C3
:102620006574706F696E743A005049443A20002016
:10263000496E7075742076616C75653A0050494436
:102640003A200020696E697400200050574D2D4FCC
:1026500075742023002073746F7000200050574D54
:102660002D4F75742023003D0050696E3A0020699B
:102670006E69740052656C61792D4F75742023006A
:102680002073746F700052656C61792D4F757420E2
:1026900023003D3E003A0070756220616374696FEB
:1026A0006E200069646C65006F6666006865617421
:1026B000696E670066616E00647279696E670063B7
:1026C0006F6F6C696E670020697320004F7574200E
:1026D00000556E6B6E6F776E207375666669782035
:1026E00000556E6B6E6F776E20636D6420006163C2
:1026F00074696F6E0072656C61794374723A200080
:102700002072656164206572726F7220666F72203C
:10271000003E2000203C003157543A003157543AD3
:10272000206E6F7420696E6974003157543A2042EC
:102730005553592074696D656F7574003157543A5B
:10274000204453323438325F4552524F525F434F28
:102750004E464947003157543A20312D776972650A
:102760002073686F72746564005B305D3A200020EE
:102770002D202D202D20EFBBBF003E003E31202D0F
:10278000200000002100240027002A002D00300036
:10279000330001010000040107010A0100002200CA
:1027A000250028002B002E0031003400020100001B
:1027B000050108010B0105050505070508080808BE
:1027C000020202020A0A08080404040401010101C9
:1027D00001010101030303030303030304070707C4
:1027E0000C0C0C0C0C0C0C0C020202020606060669
:1027F000060606060B0B0B0B0B0B0B0B0102102036
:102800002008081020401020408002010201080426
:1028100002010102040810204080804020100804BA
:102820000201800402018040201008040201080413
:102830000201010204081020408001020408102057
:10284000408000000A0B02090C0D0E08070304016A
:102850000000000000000000000000000000000078
:102860000000000000000000000000000000121145
:102870001000000000000000000000000000000048
:10288000000000000000000057726F6E672070614A
:10289000796C6164004354524C2F7478743A204F21
:1028A00075744F664D656D6F72793A2000202D3E2C
:1028B0002041543A004368616E20747970653A0093
:1028C0004E6F2073746F7265642076616C756573EA
:1028D000202D2064656661756C743A200053617622
:1028E000656420455441473A00536574204554417E
:1028F000473A20000000000000636D64000073652B
:1029000074000076616C000064656C0000485356EA
:102910000000524742000066616E00006D6F646502
:10292000006374726C006875650000736174000068
:1029300074656D7000726177000020002E00696E72
:1029400000735F6F7574006D79686F6D6500435437
:10295000524C2F657865633A204F75744F664D650C
:102960006D6F72793A2000202D3E2000456D69740C
:102970003A203C00202D3E20004974656D436D6473
:102980003A2000202D3E20004974656D3A20003128
:1029900057543A20427573207265736574206572CE
:1029A000726F72003157543A20427573205265732A
:1029B000657420646F6E65003157543A2044533279
:1029C0003438322070726573656E742C20726573B2
:1029D00065740049324320526573657400005EBC23
:1029E000E2613FDD83C29C7E20A3FD1F419DC32188
:1029F0007FFCA2401E5F01E3BD3E6082DC237D9F21
:102A0000C1421CFEA0E1BF5D0380DE3C62BEE0026D
:102A10005CDF81633D7C22C09E1D43A1FF4618FA06
:102A2000A427799BC584DA3866E5BB5907DB85673F
:102A300039BAE406581947A5FB7826C49A653BD9EC
:102A400087045AB8E6A7F91B45C6987A24F8A64425
:102A50001A99C7257B3A6486D85B05E7B98CD230D2
:102A60006EEDB3510F4E10F2AC2F7193CD114FADEF
:102A7000F3702ECC92D38D6F31B2EC0E50AFF113B8
:102A80004DCE90722C6D33D18F0C52B0EE326C8ED5
:102A9000D0530DEFB1F0AE4C1291CF2D73CA947696
:102AA00028ABF517490856B4EA6937D58B5709EBB7
:102AB000B536688AD495CB2977F4AA4816E9B75574
:102AC0000B88D6346A2B7597C94A14F6A8742AC89D
:102AD00096154BA9F7B6E80A54D7896B353E3E20C8
:102AE00000496E76616C696420636F6D6D616E6420
:102AF00000000020002300260029002C002F0032B7
:102B000000000100000301060109013E3E3E004EA7
:102B10006F204D414320636F6E666967757265640F
:102B20003A20736574206669726D776172652773E8
:102B3000204D41430A00454550524F4D207369676F
:102B40006E6174757265206F6B00496E697469619E
:102B50006C697A696E6720454550524F4D2E0000D2
:102B6000A903A70311241FBECFEFD1E2DEBFCDBF63
:102B700000E00CBF18E0A0E0B2E0E2E5F6E502E01C
:102B80000BBF02C007900D92A43CB107D9F72FE00C
:102B9000A4ECB8E001C01D92AD38B207E1F715E131
:102BA000C1EBD5E100E006C021970109802FFE01AD
:102BB0000F94ED22C03BD10780E00807A9F70F94DE
:102BC000C3160D94172B0C940000FC018481958191
:102BD0000895FC01A481B581109721F118969C916C
:102BE00018979F708EEF890F823010F091111AC0E4
:102BF00019964D935D936D937C931C97A481B58139
:102C000018969C911897907F926018969C930480D8
:102C1000F581E02D8085982F907F903619F48F7084
:102C2000806A80870895FC01238130E090E080E095
:102C3000FC01EE0FFF1FE050F74FA081B181A217FA
:102C4000B30761F4880F991F880F991FFC01E451A5
:102C5000F74F40835183628373830895A081B181CC
:102C6000AB2B19F420813181EDCF01968530910590
:102C7000F9F60895FC01238130E090E080E0FC014A
:102C8000EE0FFF1FE050F74F40815181421753076D
:102C900061F4880F991F880F991FFC01E451F74FC9
:102CA0006081718182819381089540815181452B9A
:102CB00089F431832083880F991F880F991FFC01A5
:102CC000E451F74F108211821282138260E070E0AB
:102CD000CB01089501968530910589F6F7CF880FCD
:102CE000991F880F991FFC01EC52F74F8081918149
:102CF000A281B3810196A11DB11D80839183A2831E
:102D0000B383089585E090E00C946F1684E090E022
:102D10000C946F1683E090E00C946F1682E090E0C4
:102D20000C946F1681E090E00C946F1690E080E0B8
:102D30000C946F16CF93DF93EC01E881F981048442
:102D4000F585E02D199529893A892F5F3F4F3A8BF8
:102D5000298BDF91CF910895CF93DF93EC018E857E
:102D600081110DC081E090E049895A892C853D850B
:102D70004217530708F080E0DF91CF910895E88172
:102D8000F9810484F585E02DCE0119958F3F9105D9
:102D900049F780E090E0F0CFFC01848595856817C5
:102DA000790708F4CB01928B818B0895DC011E9684
:102DB0002C911E97222339F0ED91FC910190F08126
:102DC000E02D6FEF19940895FC018785908908958F
:102DD00081E0089590E080E00895DC011296ED9185
:102DE000FC91309761F00190F081E02D309739F03F
:102DF000862F8295807F60856F70682B608708952D
:102E0000DC011296ED91FC91309751F00190F08128
:102E1000E02D309729F0808582958F7090E008959D
:102E200090E080E008950F931F93CF93DF9300D03D
:102E300000D01F921F92CDB7DEB781E028960FB663
:102E4000F894DEBF0FBECDBFDF91CF911F910F91E0
:102E5000089590E080E0089560EB7BE0811102C06E
:102E60006BEA7BE082E59DE00C9431F3DC01559642
:102E70002C915597273781F4ED91FC91008CF18DC1
:102E8000E02D199567E578E082E59DE00E9431F339
:102E900082E59DE00C947BF10895009789F0FC0198
:102EA00020852F70253061F40E949FC1009741F06A
:102EB000FC0120852F70243019F4818592850895B6
:102EC00090E080E0089565E0FC01808191810E949E
:102ED0009FC1009749F0FC018085982F907F21F0D9
:102EE00082958F7090E0089590E080E00895EF92D1
:102EF000FF920F931F93CF93DF930097C1F0FC01D4
:102F000020812223A1F08C0185E7E82E8DE0F82EA8
:102F1000C1E0D0E0B701C8010F94371B892B49F0FD
:102F20002196F5E0EF0EF11CCE30D10599F7D0E0F7
:102F3000C0E0CE01DF91CF911F910F91FF90EF90F4
:102F40000895CF92DF92EF92FF920F931F93CF934A
:102F5000DF93CDB7DEB7C154D1090FB6F894DEBF09
:102F60000FBECDBF6C01AB0130E020E060E4CE01CC
:102F700001967C010F940D0EF70101900020E9F7F6
:102F800031978F010E191F09A801B701C6010F94CF
:102F90007A27892B11F010E000E0C801CF5BDF4FEA
:102FA0000FB6F894DEBF0FBECDBFDF91CF911F915A
:102FB0000F91FF90EF90DF90CF900895CF92DF9226
:102FC000EF92FF920F931F93CF93DF93CDB7DEB7AE
:102FD000C054D1090FB6F894DEBF0FBECDBF8091AB
:102FE000810E9091820E059709F449C06115710513
:102FF00009F445C069017A018B0140E450E0CE013B
:1030000001960F9488276FE270E0CE0101960F942D
:103010004F27892B41F4980143E050E060E4CE0152
:1030200001960F940D0E4FE350E0B601CE010196CC
:103030000F946A270E9445C1882309F18091810E6F
:103040009091820E0697D9F48091680E811117C075
:10305000B701CE0101960E946BD281E090E0C05C86
:10306000DF4F0FB6F894DEBF0FBECDBFDF91CF911B
:103070001F910F91FF90EF90DF90CF90089590E017
:1030800080E0EDCFCF92DF92EF92FF920F931F93EC
:10309000CF93DF93CDB7DEB760970FB6F894DEBF5E
:1030A0000FBECDBF7C016B01CA01B9012AE0AE01A0
:1030B0004F5F5F4F0F94DB1BD701ED91FC910288AE
:1030C000F389E02D9801AE014F5F5F4FB601C70154
:1030D000199560960FB6F894DEBF0FBECDBFDF9195
:1030E000CF911F910F91FF90EF90DF90CF900895B7
:1030F000CF92DF92EF92FF920F931F93CF93DF93C4
:10310000CDB7DEB760970FB6F894DEBF0FBECDBF68
:103110007C016B01BA01A901CE0101960F94FD0E4D
:10312000D701ED91FC910288F389E02D9801AE0161
:103130004F5F5F4FB601C701199560960FB6F894BF
:10314000DEBF0FBECDBFDF91CF911F910F91FF90DA
:10315000EF90DF90CF9008951F93CF93DF93FC0102
:10316000162FC389D489818992899C012F5F3F4F93
:10317000328B218BC80FD91FCE010F945022181704
:1031800021F0612FCE010F94582281E090E0DF9171
:10319000CF911F910895FC018189928924853585FD
:1031A0008217930740F423893489820F931F0F9469
:1031B000502290E008958FEF9FEF08958F929F9295
:1031C000AF92BF92CF92DF92EF92FF920F931F9335
:1031D000CF93DF93E091830EF091840E309709F442
:1031E00067C0812EF02E932EC22EA52ED42EB72E80
:1031F000E62EBC01CF010E9427C1EC01892B19F4F6
:1032000081E090E057C088858F708530C9F760E015
:10321000CE010E949FC18C0161E0CE010E949FC13E
:10322000FC01C185D285D80119962D913C912130A0
:10323000310561F13CF46F2DCE01232B09F70F947A
:10324000ED07DECF2230310531F127303105C1F6EF
:10325000892BB1F280858F70853091F6C681D78138
:10326000209771F288858F70843061F40F2D182DAE
:103270002C2D392D4D2D5A2D6E2D7B2D89859A851E
:103280000E94DE180A80DB81C02DEACF6F2DCE01AF
:1032900003960F94ED076E2DCE010F94ED076D2D63
:1032A000CE0101960F94ED076C2DCE010296C7CF8B
:1032B00090E080E0DF91CF911F910F91FF90EF9010
:1032C000DF90CF90BF90AF909F908F9008954F92D6
:1032D0005F926F927F928F929F92AF92BF92CF92A6
:1032E000DF92EF92FF920F931F93CF93DF93809122
:1032F000140990911509892B09F49DC0E0901309D8
:10330000F12CF594E794F594E79488248394912C18
:10331000D0E0C0E0AA24A394B12CEC16FD0609F479
:103320008AC025010C2E02C0440C551C0A94E2F7F9
:10333000052C000C660877086401A4E0CA0ED11CB5
:10334000C40160E020911C0230911D02AC012817DD
:10335000390720F440911C0250911D0220917B0EF0
:1033600030917C0E240F351FF901A0814091140982
:1033700050911509FC013197E40FF51F20812A17A0
:10338000B1F04091CB085091CC086091CD0870917C
:10339000CE0844295529662977294093CB085093B4
:1033A000CC086093CD087093CE08A08361E00196AD
:1033B0008C159D0539F66623D9F1809116099091F7
:1033C0001709009751F1DC0118962C912F702530C8
:1033D00021F56C2F0E949FC1FC0190859F70943055
:1033E000E1F4818592850097C1F0409114095091D4
:1033F0001509FE01EE0FFF1FEE0FFF1FE40FF51F73
:10340000038110E0228130E0840E951ED4014C919E
:1034100050E0608170E00E94DE1880E00F94EF0DB4
:103420006093CF087093D0088093D1089093D2080E
:103430002196460172CFDF91CF911F910F91FF909E
:10344000EF90DF90CF90BF90AF909F908F907F9044
:103450006F905F904F900895CF92DF92EF92FF921E
:103460000F931F93CF93DF9300D000D0CDB7DEB77B
:10347000809125098111A4C08091810E9091820EC6
:1034800002970CF49DC080911E0990911F0900972E
:1034900009F496C064EF74E00E9427C18C01009784
:1034A00009F48EC00E9431C2E82EF12CE114F1041F
:1034B00009F486C070E060E0C8010E944D176C01FD
:1034C000EA94EF2809F48BC061E0C8010E949FC113
:1034D000FC010185128585EC94E09A8389831B8227
:1034E0001C821D821E82CE0103960F94E406CE013B
:1034F00001960E948FCB62E972E181EA9CE00E9412
:1035000031F3B60181EA9CE00E94CBF265E477E0FA
:1035100081EA9CE00E94CBF24AE050E0B80181EAE7
:103520009CE00E9482F265E477E081EA9CE00E94E0
:10353000CBF26FE979E081EA9CE00E94CBF281EA6C
:103540009CE00E947BF162E072E080E79DE00E94D7
:10355000C9FFD092660DC092650D1093680D00935F
:10356000670D8FE999E0892BE9F582EF94E090935C
:103570006A0D8093690D809118099091190900973F
:1035800041F070E060E00E944D179093650E8093CB
:10359000640E8091640E9091650E009731F19093C6
:1035A0006C0D80936B0D10926E0D10926D0D81E07D
:1035B0008093250969E772E181EA9CE00E9431F37A
:1035C00026960FB6F894DEBF0FBECDBFDF91CF9128
:1035D0001F910F91FF90EF90DF90CF90089502E040
:1035E00012E079CF8FE999E0C2CF8BEC93E0D7CF8F
:1035F000CF93DF9300D000D01F921F92CDB7DEB7DC
:10360000FC01862F8F706181607F682B618388E069
:10361000DE01119601900D928A95E1F729813A8198
:103620004B815C816D817E818F81988528960FB654
:10363000F894DEBF0FBECDBFDF91CF910895CF9339
:10364000DF9300D000D01F921F92CDB7DEB7FC01F0
:10365000608398E0DE01119601900D929A95E1F752
:1036600029813A814B815C816D817E818F81988532
:1036700028960FB6F894DEBF0FBECDBFDF91CF9175
:1036800008956F927F928F929F92AF92BF92CF9246
:10369000DF92EF92FF920F931F93CF93DF93CDB7FB
:1036A000DEB7A0970FB6F894DEBF0FBECDBF8C017A
:1036B000862E7A01DC018D919C911197892B09F45A
:1036C00066C01496ED91FC91309709F460C080813A
:1036D0008071BFEF6B135DC0B1F481E0A0960FB6AF
:1036E000F894DEBF0FBECDBFDF91CF911F910F9138
:1036F000FF90EF90DF90CF90BF90AF909F908F9012
:103700007F906F9008954330510539F38180829402
:103710002FE0822267EF78E082E59DE00E9431F39E
:103720004AE050E0D80113966C9182E59DE00E943A
:1037300098F165EF78E082E59DE00E9431F3D801D1
:103740001496ED91FC9161816F704AE050E082E542
:103750009DE00E9498F162EF78E082E59DE00E9492
:1037600031F34AE050E0682D82E59DE00E9498F137
:1037700082E59DE00E947BF1D8011496ED91FC91C9
:1037800081818F70881207C080818F7E808380E066
:10379000A5CF8111FCCF198E1A8E1B8E1C8E1D8E0B
:1037A0001E8E1F8E18A28A8D8F708A8FD801149654
:1037B000ED91FC9181818F708815A9F1B3E0EB1632
:1037C000F10489F160EF78E082E59DE00E9431F339
:1037D0004AE050E0F801638182E59DE00E9498F1A3
:1037E0006EEE78E082E59DE00E9431F3D8011496F8
:1037F000ED91FC9161816F704AE050E082E59DE0BF
:103800000E9498F16BEE78E082E59DE00E9431F332
:103810004AE050E0682D82E59DE00E9498F182E543
:103820009DE00E947BF1F80120813181FCE0F815D8
:1038300008F416C1E82DF0E08827EE5DF34E8F4FB7
:103840000D94ED222F1C6C1CED1C041D101DED1C95
:10385000C61CED1C131D1E1DDA1C211D2D1DD801BB
:103860001496CD90DC90F60181818F70853009F43B
:10387000F7C050F48230C1F069E075E0C9010E94E0
:1038800027C13C01912C4BC08730D1F08A30A1F781
:1038900062E075E0C9010E9427C13C01D6019C90FD
:1038A00092FA992490F83BC06CEF74E0C9010E9431
:1038B00027C13C01D6019C9090FA992490F82FC022
:1038C0006BEF74E0C9010E9427C13C01F6019080B2
:1038D00091FA992490F823C06EE075E0C9010E9426
:1038E00027C13C01D8011496ED91FC91808180FBA9
:1038F000992490F8982F9E7F80FF916090836114A7
:10390000710469F461E0CE0149960E941F1B298B66
:103910003A8B4B8B5C8B6D8B7E8B8F8B988FF801EA
:10392000A080B18064E475E0C5010E9427C16C01EC
:1039300069E475E0C5010E9427C15C01892B81F40F
:10394000C114D10469F460E0CE0149960E941F1BA6
:1039500029833A834B835C836D837E838F8398872F
:10396000D8011496ED91FC916114710409F07CC0AA
:10397000898D811179C0B82DBF708B2E8181807F98
:10398000882A818280818F7E8083A7CE63E175E063
:10399000C9010E9427C13C01D8011496ED91FC9108
:1039A000808181FB992490F8982F9D7F81FF926000
:1039B0009083B5CF69E175E0C9010E9427C13C0140
:1039C000D8011496ED91FC91808182FB992490F8A6
:1039D000982F9B7F82FF9460EBCF69E075E0C9016F
:1039E0000E9427C13C01892B09F04CCF62E0CE0137
:1039F00049960E941F1B29873A874B875C876D87F2
:103A00007E878F87988B3ECF6FE175E0C9010E945A
:103A100027C13C01D8011496ED91FC9190804CCFC8
:103A200064E275E0F3CF6AE275E0C9010E9427C144
:103A30003C01D8011496ED91FC9149CF60E375E00B
:103A4000F4CF67E375E0C9010E9427C13C01D801AA
:103A50001496ED91FC91908023CF6DE375E0F3CF48
:103A6000912C712C612C5BCF83E0E816F104B9F046
:103A7000982D9F70892E8181807F882A8182808104
:103A80008F7E8083E98CFA8C0B8D1C8D2D8D3E8D65
:103A90004F8D58A1692DC3010F9412111ECE818143
:103AA0008F70881509F419CE829490EF8922882AA4
:103AB00081828081806168CFCF93DF9300D000D076
:103AC0001F921F92CDB7DEB7FC0191819F70906B62
:103AD0009183448355836683778388E0DE01119662
:103AE00001900D928A95E1F729813A814B815C81A1
:103AF0006D817E818F81988528960FB6F894DEBF00
:103B00000FBECDBFDF91CF910895CF93DF9300D04B
:103B100000D01F921F92CDB7DEB7FC016F3F710539
:103B200019F014F06FEF70E077FD60E09181892F5C
:103B300082958F7081508230C8F4648388E0DE0102
:103B4000119601900D928A95E1F729813A814B8176
:103B50005C816D817E818F81988528960FB6F8945F
:103B6000DEBF0FBECDBFDF91CF9108959F709061F2
:103B70009183E3CFCF93DF93CDB7DEB760970FB6D6
:103B8000F894DEBF0FBECDBF19821A821B821C8241
:103B90001D821E821F8218868A818F708A836FEF32
:103BA00070E0CE0101960E94851D60960FB6F894D4
:103BB000DEBF0FBECDBFDF91CF910895CF92DF92D0
:103BC000EF92FF92DC01362F1196EC911197E2955E
:103BD000EF70EC3008F0B6C0F0E08827ED50F24E00
:103BE0008F4F0D94ED22A51E2B1E2B1EA21EA21E72
:103BF000A21E701E321EA21EA21EFF1DFF1D1496C5
:103C00008D919D910D90BC91A02D662399F0B7FDEB
:103C10009FC08F3F9105A105B10529F024F08FEFDA
:103C200090E0A0E0B0E02FEF30E0A901481B590B75
:103C3000CA010CC0B7FD89C08F3F9105A105B10530
:103C400029F024F08FEF90E0A0E0B0E0FF90EF903B
:103C5000DF90CF90089514962C91822F90E06623E8
:103C6000A9F3E1CF1496CD90DD90ED90FC901797DD
:103C7000662301F120E030E0A901C701B6010F94ED
:103C80002C2187FD65C020E030E04FE753E4C701F9
:103C9000B6010F94342418160CF457C0A7019601EE
:103CA00060E070E08FE793E40F941F230F94FE23EE
:103CB000CB01CCCF20E030E0A901C701B6010F94C1
:103CC0002C2187FD42C020E030E04FE753E4C701DC
:103CD000B6010F9434241816DCF1C701B601E6CF03
:103CE00014966D917D918D919C9117973323B1F02E
:103CF0006D395FEF75078507950754F1611524E667
:103D00007207810591050CF52CE93FEF4FEF5FEF4E
:103D10000F949822C90181509F4F98CF6D394FEF72
:103D20007407840794078CF0611554E675078105C4
:103D3000910574F424E630E040E050E00F949822BE
:103D4000C90184CF8FEF9FEF81CF90E080E07ECFDD
:103D50008FEF90E07BCFCF93DF93EC01DB01898184
:103D600082958F708630E1F128F481508230C8F05E
:103D700080E014C0873009F18A508230C8F72FEFF5
:103D800030E00F94042324E630E040E050E00F944C
:103D900098222C833D834E835F8381E0DF91CF9116
:103DA00008952FEF30E00F94042324E630E040E044
:103DB00050E00F9498222C83F0CF2FEF30E00F9437
:103DC000042324E630E040E050E00F949822CA013A
:103DD000B9010F9433216C837D838E839F83DDCF64
:103DE0002CE933E60F94042324E630E040E050E071
:103DF0000F9498222C833D834E835F83B9CFDC01DF
:103E00001196EC911197E295EF70E150EB3008F0CC
:103E100039C0F0E08827E05FF04E8F4F0D94ED221F
:103E2000331F331F421F1B1F1B1F241F3B1F3B1F22
:103E30003B1F1B1F1B1F14966D917D918D919C91B3
:103E400017970F943321089514966D917D918D915C
:103E50009C91179724E630E040E050E00F949822C0
:103E6000CA01B901EECF14966C9170E090E080E049
:103E70000F943121089514966D917D918D919C91AF
:103E80001797089560E070E0CB010895DC0111966A
:103E9000EC911197E295EF70E150EB3008F037C0EC
:103EA000F0E08827E95AF04E8F4F0D94ED22691FFC
:103EB000691F871F621F621F781F6F1F6F1F6F1F91
:103EC000621F621F14966D917D918D919C91179741
:103ED000089514966C9170E090E080E00895149637
:103EE0006D917D918D919C9117970F94FE2308956C
:103EF00014966D917D918D919C91179724E630E0F9
:103F000040E050E00F949822CA01B901089560E0A2
:103F100070E0CB0108958F929F92AF92BF92CF92A3
:103F2000DF92EF920F931F93CF93DF9300D000D0D7
:103F30001F921F92CDB7DEB7FC0109831A832B8332
:103F40003C834D835E836F83788780819181009766
:103F5000A1F490E080E028960FB6F894DEBF0FBE83
:103F6000CDBFDF91CF911F910F91EF90DF90CF9058
:103F7000BF90AF909F908F9008958F010E9431C2A3
:103F8000C82ED12C86E0C816D10464F40E9404C760
:103F9000BC01F801808191810E9411C7FFEFCF1A07
:103FA000DF0AF0CF65E0F801808191810E949FC116
:103FB0008C01892B71F28981803158F6CE010196EE
:103FC0000E94461F161617061806190644F4F80133
:103FD0008085982F9D70A1F08F70873089F0F8014F
:103FE00080858F70808765E479E082E59DE00E949E
:103FF00031F382E59DE00E947BF181E090E0ABCF60
:104000000E949DD14B015C01CE0101960E94461F8A
:10401000860E971EA81EB91EF80181869286A38679
:10402000B48682E0E11087E099819295907F892B98
:10403000F80180876AE379E082E59DE00E9431F330
:10404000CE0101960E94461FAB01BC012AE030E080
:1040500082E59DE00E943AF264E379E082E59DE02A
:104060000E9431F3F80141855285638574852AE009
:1040700030E082E59DE00E943AF2BBCFDC01119670
:10408000EC911197E295EF70E150EB3008F03EC0F3
:10409000F0E08827E15BFF4D8F4F0D94ED22652006
:1040A000652086205A205A207F20702070207020A2
:1040B0005A205A2014962D913D914D915C9117975D
:1040C000A4E6B0E00F94B722089514966C9184E6AC
:1040D000689FB0011124072E000C880B990B0895DE
:1040E00020E030E048EC52E414966D917D918D9182
:1040F0009C9117970F9492210F94FE230895149684
:104100006D917D918D919C911797089560E070E07D
:10411000CB010895FC01A7812A2F2E7FD1F0818148
:1041200082958F7081508330A0F4A695A150BB0B6F
:104130002BE531E00F94042324E630E040E050E02A
:104140000F949822DA01C90187569F4FAF4FBF4F96
:1041500008958FEF9FEF08952F923F924F925F92B5
:104160006F927F928F929F92AF92BF92CF92DF9287
:10417000EF92FF920F93CF93DF9300D01F92CDB7B2
:10418000DEB77C017A8369835C834B83DB011C92FD
:10419000FC016081662309F44EC030FF4CC0F9E099
:1041A0006F9FB001112468567F4ECD010F946E1B96
:1041B000D70111968C91807F41F04B815C816EEF2D
:1041C00076E089819A810F946A27E981FA810190CA
:1041D0000020E9F7319729813A81E21BF30B19019D
:1041E0002E0E3F1E4B815C814E1B5F0B41505109CF
:1041F0005C834B83D7011196EC9111978E2F807FB2
:1042000009F4F7C0E295EF70E150EC3008F0F1C02E
:10421000F0E08827E15FFE4D8F4F0D94ED221E21C7
:10422000C1212E228D22A8226C213E223E223E2236
:104230005A214221C42229803A80DCCFF7018481AF
:10424000282F30E050E040E0002359F030E0A4E6B1
:10425000B0E00F94CA222FEF30E040E050E00F941E
:1042600098225F934F933F932F938EE495E09F9313
:104270008F93FC81FF932B812F933F922F920F946A
:10428000A227B2C017968C9117978F9316968C9190
:1042900016978F9315968C9115978F9314968C91F2
:1042A0008F9381E595E09F938F93BC81BF93EB81C2
:1042B000EF93E3CF17968C9117978F9316968C9167
:1042C00016978F9315968C9115978F9314968C91C2
:1042D0008F9385E595E0E7CF1496CD90DD90ED9036
:1042E000FC901797F7FE34C084E6882E912CA12C01
:1042F000B12CC701B601A50194010F9498229B012E
:10430000AC0188279927DC01821B930BA40BB50B0A
:10431000BF93AF939F938F9366277727CB016C1939
:104320007D098E099F09A50194010F9498225F933E
:104330004F933F932F9389E595E09F938F933C8113
:104340003F934B814F933F922F920F94A2274CC0E3
:10435000C701B60124E630E040E050E00F94982217
:104360009F938F937F936F935F934F933F932F937D
:104370008AE595E09F938F939C819F93AB81AF9348
:10438000E2CFC7010E948A20BC01D7011696CC90CB
:1043900016971796DC901797D0FADD24D0F814966C
:1043A0009C9114971596FC90EB80BC80292F30E0EF
:1043B00050E040E077FD35C0011135C07F936F9329
:1043C0001F921F921F929F931F92FF92DF92CF9294
:1043D00083E695E09F938F93FC81FF932B812F932E
:1043E0003F922F920F94A2270FB6F894DEBF0FBE14
:1043F000CDBF89819A810F900F900F900F90DF9120
:10440000CF910F91FF90EF90DF90CF90BF90AF9042
:104410009F908F907F906F905F904F903F902F90E4
:104420000895002361F0292F30E0A4E6B0E00F9456
:10443000CA222FEF30E040E050E00F9498225F93C3
:104440004F933F932F931F92FF92DF92CF9286E676
:1044500095E09F938F93BF92EF9275CF15968C91B5
:1044600015971F928F9316969C91169717968C917D
:1044700081708F939F9389E695E015CF14968D9068
:104480009D90AD90BC90179720E030E0A901C50148
:10449000B4010F942C212401350187FF04C077FA61
:1044A000709477F87094C301B2010F94FE236B01EE
:1044B000072E000C880B990B0F9433219B01AC0144
:1044C000C301B2010F941F2320E030E04AE754E417
:1044D0000F9492210F9489240F94FE23062F772E98
:1044E00020E030E0A901C501B4010F942C2187FF21
:1044F00007C07F920F93DF92CF928FE695E0D3CEE5
:104500007F920F93DF92CF9280E795E09F938F93F6
:104510003C813F934B814F93B0CE14968C9114976E
:104520001F928F9315968C9115971F928F931696C5
:104530008C911F928F9386E695E09F938F93BC8119
:10454000BF93EB81EF933F922F920F94A2274CCF12
:1045500017968C9117971F928F9314968C9114979E
:104560001F928F9315968C9115971F928F93169685
:104570008C911F928F9383E695E09F938F93BC81DC
:10458000BF93EB81EF93DFCE14966D917C914B81BD
:104590005C81C1010F9488272CCFEF92FF920F937B
:1045A000CF93DF93CDB7DEB7A0970FB6F894DEBFF9
:1045B0000FBECDBF7C0100E020E033E040E250E0E0
:1045C000BE016F5F7F4F0E94AC20BE016F5F7F4FC7
:1045D00082E59DE00E94CBF260E871E182E59DE01A
:1045E0000E9431F3F701618162956F704AE050E0FB
:1045F00082E59DE00E9498F169E771E182E59DE026
:104600000E9431F3F70161816F704AE050E082E56A
:104610009DE00E9498F182E59DE00E947BF1A096CA
:104620000FB6F894DEBF0FBECDBFDF91CF910F91D3
:10463000FF90EF900895CF93DF93EC016115710522
:1046400039F48F8181708F8381E0DF91CF9108955C
:104650008981982F92959F7029F180E09430A8F776
:104660009B01770F440B550B295931094109510919
:10467000A4E6B0E00F94B7222BE531E040E050E033
:104680000F94982237FF02C030E020E02536310534
:1046900014F024E630E02F5F220F8F818170282BE9
:1046A0002F83D2CF8F7080628983DACF2F923F928F
:1046B0004F925F926F927F928F929F92AF92BF9232
:1046C000CF92DF92EF92FF920F931F93CF93DF93DE
:1046D000CDB7DEB768970FB6F894DEBF0FBECDBF7B
:1046E0001C0109871A872B873C874D875E876F8758
:1046F000788B22E1E216F10408F035C0F701EA5F99
:10470000FB4F3081398BCE0109960E948A2097FD9C
:1047100004C0BC01C1010E941B239A85892F8F70A0
:10472000D1011196EC911197E07FE82B1196EC9353
:10473000119789858C93E295EF70EC3008F063C097
:10474000F0E08827E955FC4D8F4F0D94ED22AA2506
:10475000D023D0234825B523D6251125522552250F
:10476000522511251125198ACECFB12C92959F7013
:104770009D3008F0C9C4E92FF0E08827ED53FC4DC7
:104780008F4F0D94ED220324102630261026D925B4
:10479000D925102610268428842810261026DD24EA
:1047A00092959F709D3008F018C1E92FF0E088279E
:1047B000E352FC4D8F4F0D94ED220324BB24AE2415
:1047C0007124ED23EA239224BD24ED24ED247C24DE
:1047D0007C24DD248889F10187838F85D101169699
:1047E0008C9316978E8515968C9315978D851496B8
:1047F0008C9314979295907F11968C9111978F704E
:10480000982B11969C93B989BB2309F467C0F101D9
:10481000818182958F702B2F30E08217130609F467
:104820005DC06FEF7FE082E59DE00E9431F3D10132
:1048300011966C9162956F704AE050E082E59DE0C0
:104840000E9498F16CEF7FE082E59DE00E9431F3D9
:104850004AE050E0698982E59DE00E9498F16AEFA4
:104860007FE082E59DE00E9431F3F1010081198231
:104870001A821B821C821D821E821F8218868989D1
:104880008295807F9A819F70892B8A830983EE2489
:10489000EA94FE2C11812281338144815581668105
:1048A0007781CE0101960E945623D1012C93119657
:1048B0003C93119712964C93129713965C9313970F
:1048C00014966C93149715967C93159716968C9363
:1048D000169717969C93C1010E94CD2288E0F101A2
:1048E00078C18F859889F1018683878190FB80F953
:1048F00087838E85858387CF8D859E85AF85B88993
:10490000B7FD0EC08F3F9105A105B10529F024F038
:104910008FEF90E0A0E0B0E0D10114968C9373CFBC
:1049200080E0FACF6D857E858F85988920E06D398E
:10493000BFEF7B078B079B076CF02FEF6115E4E659
:104940007E078105910534F424E630E040E050E034
:104950000F949822D10114962C9355CF8F85988966
:10496000F1018683878190FB80F987838E8585831B
:104970008D85848348CF8D85CFCFCD84DE84EF8431
:10498000F88820E030E0A901C701B6010F942C217E
:1049900060E087FD0FC020E030E04FE753E4C7013F
:1049A000B6010F9434246FEF181624F0C701B60136
:1049B0000F940524F101648326CFD10111968C91C7
:1049C00011978F70806C11968C9311978D859E85B1
:1049D00015969C938E93149716CF6FE770E182E53E
:1049E0009DE00E9431F36A8562956F704AE050E065
:1049F00082E59DE00E9498F16CE770E182E59DE020
:104A00000E9431F3F101618162956F704AE050E0DC
:104A100082E59DE00E9498F182E59DE00E947BF195
:104A2000F2CE92959F70933091F09C3031F24D858B
:104A30005E856F857889F10144835583668377832A
:104A40009295907F81818F70982B9183DCCE60E06E
:104A5000C1010E94DE1DD10114968C9314978F859D
:104A6000988916968C93169717968C91179790FBAA
:104A700080F917968C9317978E8515968C931597BA
:104A800011968C9111978F70806211968C93BBCE8A
:104A900060E0CE0109960E94DE1DD10114968C9330
:104AA0001497EECF92959F709D3008F066C0E92F65
:104AB000F0E08827E15AFA4D8F4F0D94ED22032440
:104AC0007A25A9252725A925A9256C259925992584
:104AD000992588259425DD248D859E85AF85B88907
:104AE000F10184839583A683B78381818F7080666B
:104AF000818389CE6D8570E090E080E00F94312154
:104B0000D10114966D937D938D939C9317977BCED3
:104B10006D857E858F8598890F943321F10164839B
:104B20007583868397836FCE6D857E858F85988903
:104B3000E5CF9295907FF10181818F70982B9183C1
:104B40008D859E85AF85B88984839583A683B78339
:104B50005ACE9295907FD10111968C9111978F70BA
:104B6000982B11969C938D859E85AF85B889F10110
:104B700084839583A683B78346CE6AE670E182E597
:104B80009DE00E9431F36A8562956F704AE050E0C3
:104B900082E59DE00E9498F167E670E182E59DE084
:104BA0000E9431F3D10111966C912ECFBB24B394A6
:104BB000DDCD4D855E856F857889F1014483558310
:104BC000668377839295907F81818F70982B9183F4
:104BD00088E0DE01119601900D928A95E1F7298116
:104BE0003A814B815C816D817E818F819885689649
:104BF0000FB6F894DEBF0FBECDBFDF91CF911F91EE
:104C00000F91FF90EF90DF90CF90BF90AF909F906B
:104C10008F907F906F905F904F903F902F9008956E
:104C2000963009F43EC148F46D85913071F06FEF14
:104C300070E0933051F060E008C0973009F43DC156
:104C40009A506D857E859230B0F784E68F8788898B
:104C50008E7F888B1E868A858F7080628A876D879B
:104C60002E8530E0AFEFB0E00F94CA22C12CD12CDA
:104C70007601CA946115F4E67F078105910544F435
:104C800024E630E040E050E00F94982269017A0178
:104C900086012D852A8B622E712CBB2009F475C0EC
:104CA00088898695A82FA150BB0B2D01BFEF4B160D
:104CB0005B0609F023C1003811050CF005C18FE730
:104CC00090E08C199D09869DD001879DB00D969D21
:104CD000B00D11242FEF30E00F94042321E83EE7BC
:104CE00040E050E00F949822F1012783ABE9B0E057
:104CF000A70196010F94B722EFE78E2E912CA12CDD
:104D0000B12CA50194010F94982289019A010C59A4
:104D10001F4F2F4F3F4FAEEFB1E0A70196010F9409
:104D2000B722A50194010F949822D3010F94B722C2
:104D30002FEF30E040E050E00F94982239012FEF40
:104D40006216710421F01CF066246A94712C6AE5E5
:104D500070E182E59DE00E9431F34AE050E0B80145
:104D600082E59DE00E9482F26CE470E182E59DE0C4
:104D70000E9431F34AE050E0B30182E59DE00E94D9
:104D800082F282E59DE00E947BF1E6EBF7E2E4919E
:104D9000F0E0EE0FFF1FE456F84D85919491ECEF93
:104DA000F7E2E4912F8538893170AFEFBFEF0F94B0
:104DB000CA222DE631E040E050E00F9498224427CB
:104DC0005527AAEFB5E00F94B722DC01CB0190582C
:104DD000AF4FBF4FCD01BB2797FDB095AB2F8E3F97
:104DE000E1E09E0708F069C1382F8F3F910508F474
:104DF00086C14EEF481B50E03FEF7301FFEFEF1A03
:104E0000FF0AF801FF273196009510E03E9FC00190
:104E10003F9F900D1124292F3327200F311FD701D9
:104E20000F9404234B015C018824AA24BB245E9FB9
:104E300090015F9F300D1124232F3327200F311F46
:104E40000F940423BB27A92F982F872F882A992AEC
:104E5000AA2A4E9F90014F9F300D1124232F3327F4
:104E6000200F311FD7010F940423B82FA72F962F9F
:104E7000882788279927BB2788299929AA29F101FA
:104E8000A6839583848360E270E182E59DE00E94C1
:104E900031F3C1010E94CD2260E080E00E9422CF68
:104EA000B2CC6D857E858F85988924E630E040E020
:104EB00050E00F949822B901C8CE6D857E858F850C
:104EC00098890F94FE23C1CEA7019601205831097D
:104ED00041095109ABE9B0E00F94B7222FE730E068
:104EE00040E050E00F94982289019A010C591F4F1D
:104EF0002F4F3F4FD10117961C9229CF9201AAEB59
:104F0000BFEF0F94FC2244E6842E912CA12CB12CEF
:104F1000A50194010F949822DA01C9018C599F4F81
:104F2000AF4FBF4F8B8B9C8BAD8BBE8B26E430E09D
:104F3000D2010F940423A50194010F9498224901F2
:104F40005A019EE1890E911CA11CB11C003811056B
:104F50000CF099C08FE790E08C199D09869DD001D7
:104F6000879DB00D969DB00D1124A50194010F945D
:104F7000C2229B01AC01AFEFB0E00F94B72224E650
:104F80003AE640E050E00F949822D10117962C9316
:104F90002B893C894D895E892C0D3D1D4E1D5F1D61
:104FA000AEEFB1E00F94B72223EE30E040E050E0E6
:104FB0000F94982229013A01388F2F8BAFEFB0E080
:104FC000A70196010F94B7222FE730E040E050E0B0
:104FD0000F9498228901EA89AE2FB0E0A3019201D3
:104FE0000F94B7222FEF30E040E050E00F9498226A
:104FF00039012F3F310521F01CF066246A94712C91
:1050000066E470E182E59DE00E9431F32AE030E041
:105010004B895C896D897E8982E59DE00E943AF228
:1050200060E470E182E59DE00E9431F32AE030E027
:10503000B501A40182E59DE00E943AF268E370E1C7
:1050400082E59DE00E9431F34AE050E0B80182E53C
:105050009DE00E9482F260E370E182E59DE00E94A3
:1050600031F34AE050E0B30182E59DE00E9482F214
:1050700067E270E182E59DE00E9431F34AE050E092
:105080006F89788D7ACEA7019601205831094109A0
:105090005109ABE9B0E00F94B7222FE730E040E0D0
:1050A00050E00F94982289019A010C591F4F2F4FFD
:1050B0003F4FD10117961C92A3CF8C3FF3E09F077F
:1050C00068F48D3F22E0920728F452E0580F3FEF3A
:1050D00040E093CE3CEF381B5FEFFACF8A3F35E0DC
:1050E000930781F08B3FE4E09E0728F444E0480FEB
:1050F0005FEF30E082CE5AEF581B30E001C050E045
:105100004FEF7BCE50E0F9CF6EE070E182E59DE09D
:105110000E9431F36A8562956F704AE050E082E543
:105120009DE00E9498F16BE070E138CDFC01918127
:10513000892F82958F7021F0823029F080E00895C8
:105140009F70906291839B0177FF02C030E020E066
:105150002E3681E0380714F02DE631E02683878172
:1051600030FB80F9878381E00895EF92FF920F93DF
:105170001F93CF93DF93FC01892B69F190819923D1
:1051800051F19D3291F180ED890F8A3070F1C8E0C4
:10519000D0E0953211F1CEEFDFEF9B37F1F0C7E1B0
:1051A000D0E09332D1F08F0181EAE82E80E1F82E31
:1051B000C1E0D0E0C7010F94471BAC01B701C801A3
:1051C0000F94601B892B49F0219689E0E80EF11CB1
:1051D000C931D10579F7CFEFDFEFCE01DF91CF9164
:1051E0001F910F91FF90EF900895D0E0C0E0F5CFB0
:1051F000EF92FF920F931F93CF93DF93EC01892BD4
:1052000051F188858F70843009F5E984FA84C701EB
:105210000E94B5288C0118161906ECF4C7010E94EB
:10522000A8F6C801012E000CAA0BBB0B89879A8730
:10523000AB87BC878885807F82608887C801DF91C3
:10524000CF911F910F91FF90EF900895823019F444
:1052500009851A85F3CF10E000E0F0CF2F923F923E
:105260004F925F926F927F928F929F92AF92BF9276
:10527000CF92DF92EF92FF920F931F93CF93DF9322
:10528000CDB7DEB76C970FB6F894DEBF0FBECDBFBB
:105290006115710549F528E0FC01DE0111960190C8
:1052A0000D922A95E1F729813A814B815C816D81CC
:1052B0007E818F8198856C960FB6F894DEBF0FBE05
:1052C000CDBFDF91CF911F910F91FF90EF90DF90B5
:1052D000CF90BF90AF909F908F907F906F905F9096
:1052E0004F903F902F9008956B018C0162EB78E016
:1052F000C6010E9427C1FC01892B09F40EC18085DB
:105300008F70843009F452C0853009F006C1E68000
:10531000F780E114F10409F400C1F70180858F7072
:10532000823011F4E280F380E114F10409F4F5C055
:10533000F70180858F70853011F0F701F3CFC70139
:105340000E9431C28230C9F760E0C7010E949FC14C
:105350005C010E94F82861E0C7010E949FC14C01D6
:10536000FC0180858F70823041F7C8010E94461F82
:10537000F401418452846384748464157505860540
:105380009705D9F6A114B10409F4C7C019821A828D
:105390001B821C821D821E821F8218868A818F704A
:1053A0008A83F5016185CE0101964EC068E775E0FC
:1053B000818592850F945A27892B09F0AEC0C801C8
:1053C0000E94461F611571058105910509F48BC086
:1053D000660F771F881F991F2FEF30E040E050E0E5
:1053E0000F94982257FD15C0233031054105510512
:1053F0000CF05FC0DA01C9010196A11DB11D823018
:105400009105A105B105D9F10397A105B10509F4ED
:1054100050C019821A821B821C821D821E821F822A
:1054200018868A818F708A8367E0CE0101960E9478
:10543000F81A29873A874B875C876D877E878F8725
:10544000988B62E1CE0109960E941F1B298B3A8B33
:105450004B8B5C8B6D8B7E8B8F8B988F49895A8998
:105460006B897C898D899E89AF89B88D49835A83E0
:105470006B837C838D839E83AF83B88714CF19821F
:105480001A821B821C821D821E821F8218868A81BC
:105490008F708A8367E0CE0101960E94F81A2987EF
:1054A0003A874B875C876D877E878F87988B61E112
:1054B000C9CF19821A821B821C821D821E821F8202
:1054C00018868A818F708A8367E0CE0101960E94D8
:1054D000F81A29873A874B875C876D877E878F8785
:1054E000988B60E1AFCF19821A821B821C821D82C9
:1054F0001E821F8218868A818F708A8367E0CE01A0
:1055000001960E94F81A29873A874B875C876D8736
:105510007E878F87988B62E095CF6CE775E0C60138
:105520000E9427C15C01009709F4C5C0FC01808579
:105530008F70853009F0AEC0C5010E9431C2843041
:1055400009F0B9C060E0C5010E949FC14C0161E053
:10555000C5010E949FC13C0162E0C5010E949FC13C
:10556000FC01C184D284E384F48463E0C5010E9419
:105570009FC15C01C8010E94461F6C157D058E0508
:105580009F059CF419821A821B821C821D821E8236
:105590001F8218868A818F708A8340E050E0BA01AA
:1055A000CE0101960E945C1D51CFF4010184F28569
:1055B000E02DFA8FE98FF30121843284F501018413
:1055C000F285E02DFC8FEB8F19821A821B821C82E0
:1055D0001D821E821F8218868A818F708A83298D80
:1055E0003A8D4901330FAA08BB0826010D2C000C87
:1055F00066087708C8010E94461F9B01AC01241968
:10560000350946095709B101032C000C880B990B89
:10561000681979098A099B090F946622EB8DFC8D24
:105620009F01FF0F440B550B2419350946095709F3
:105630000F949822820E931EA41EB51EC101298DBF
:105640003A8D821B930B6B8D7C8D6C197D090F94A9
:10565000D92277FF02C06F5F7F4F75956795CB01A9
:10566000770FAA0BBB0B880E991EAA1EBB1EB7FC98
:105670000CC0A401B5013FEF83169104A104B1044D
:1056800009F00CF48DCF4FEF01C040E050E060E036
:1056900070E086CF81110FC019821A821B821C8292
:1056A0008A818F708A8349815A816B817C8180E0F5
:1056B00090E0DC01DBCEF801408151816281738191
:1056C00084819581A681B781D1CE4F925F926F92EE
:1056D0007F928F929F92AF92BF92CF92DF92EF9282
:1056E000FF920F931F93CF93DF93CDB7DEB76097F1
:1056F0000FB6F894DEBF0FBECDBF6115710539F549
:1057000028E0FC01DE01119601900D922A95E1F747
:1057100029813A814B815C816D817E818F81988561
:1057200060960FB6F894DEBF0FBECDBFDF91CF916C
:105730001F910F91FF90EF90DF90CF90BF90AF90AF
:105740009F908F907F906F905F904F9008956B0126
:105750008C0162EB78E0C6010E9427C15C01F80170
:10576000F080FF2009F44EC0009709F44BC0FC0103
:1057700080858F70843009F4BFC0853009F042C045
:1057800060E875E082E59DE00E94CBF282E59DE055
:105790000E947BF1F501E680F780E114F10491F1BC
:1057A000F70180858F705701823061F0B12CA12CF8
:1057B000E114F10409F41DC1F70180858F70853073
:1057C00021F0F701E280F380F3CFC7010E9431C2DC
:1057D0008230B9F760E0C7010E949FC10E94F8289B
:1057E0004C0161E0C7010E949FC1F801208128158A
:1057F000190439F7FC0120852F70223011F700972A
:1058000009F001C16CE775E0C6010E9427C17C0167
:10581000F8018181807F09F407C1E114F10409F4E2
:105820007DC0F70180858F70853009F001C1C70107
:105830000E9431C2843009F0FBC0C8010E94461F9B
:105840004B015C0160E0C7010E949FC1FC018185A2
:105850009285A385B48519821A821B821C821D82BF
:105860001E821F82188688169906AA06BB060CF4AB
:1058700099C08A818F708A8363E0C7010E949FC1AB
:105880005C0162E0C7010E949FC1FC014184528417
:105890006384748461E0C7010E949FC14C0160E091
:1058A000C7010E949FC1FC01C184D284E384F484B7
:1058B000C8010E94461FF501218532854385548524
:1058C00024193509460957096C197D098E099F0964
:1058D0000F946622F40121853285438554852C1965
:1058E0003D094E095F090F949822BA01A901440DA0
:1058F000551D661D771D31C068E775E0818592856D
:105900000F945A27892B09F07DCFF0E1FF1609F497
:1059100060C0FF1568F082E0F816E1F1F8014081FF
:1059200051816281738184819581A681B78129C06B
:10593000E1E1FE16F1F1F2E1FF12F0CF19821A82D5
:105940001B821C821D821E821F8218868A818F7094
:105950008A8344E150E060E070E0CE0101960E944D
:105960005C1D29873A874B875C876D877E878F8789
:10597000988B49855A856B857C858D859E85AF85FD
:10598000B88949835A836B837C838D839E83AF83DD
:10599000B887BECE19821A821B821C821D821E828B
:1059A0001F8218868A818F708A8340E050E0BA0196
:1059B000D4CF19821A821B821C821D821E821F82F2
:1059C00018868A818F708A8340E850E060E070E03A
:1059D000C4CF19821A821B821C821D821E821F82E2
:1059E00018868A818F708A834FEF50E060E070E004
:1059F000B4CFA114B10409F405CFF50180858F70EF
:105A000009F400CFC50119821A821B821C821D82F3
:105A10001E821F8218862A812F702A83FC014185ED
:105A200052856385748599CFE114F10409F476CF2A
:105A3000F70180858F7009F071CF19821A821B825D
:105A40001C828A818F708A8349815A816B817C8113
:105A500080E090E0DC0195CF0F931F93CF93DF930D
:105A60008C01FC01C081D1816FE270E0CE010F9406
:105A700097270097E9F0FC011192CF010E94771758
:105A8000EC0169E079E082E59DE00E9431F34AE0B3
:105A900050E0BE0182E59DE00E9482F282E59DE039
:105AA0000E947BF1CE01DF91CF911F910F9108955C
:105AB000CE010E947717EC01892BA1F3F801118226
:105AC0001082F0CFDC01ED91FC91309729F09085A8
:105AD0009F7081E0953009F080E00895EF92FF9289
:105AE0000F931F93CF93DF93EC017B018E819F81F6
:105AF000892BA9F4888199810E9431C2082F10E076
:105B00000530110564F40E9404C79F838E83BC0195
:105B1000888199810E9411C70F5F1F4FF1CFEE81DD
:105B2000FF813097D9F08085982F9F70A9F4807FEE
:105B300082608087EE81FF8111861286138614862B
:105B4000EE81FF81F782E682C701DF91CF911F913D
:105B50000F91FF90EF900895923061F3F12CE12CBA
:105B6000F3CFCF92DF92EF92FF920F931F93CF93D9
:105B7000DF93EC016A017B018E819F81892BA9F45F
:105B8000888199810E9431C2082F10E005301105EB
:105B900064F40E9404C79F838E83BC01888199812D
:105BA0000E9411C70F5F1F4FF1CFEE81FF81309729
:105BB00081F08085982F9F7051F4807F826080876C
:105BC000EE81FF81C186D286E386F48602C09230E0
:105BD000B9F3DF91CF911F910F91FF90EF90DF907C
:105BE000CF900895FC0186819781009799F0FC0180
:105BF00020852F70223029F46185728583859485F4
:105C00000895253039F460E00E949FC1009711F09B
:105C1000FC01F2CF60E070E0CB0108950F931F9379
:105C2000CF93DF93FC01C281D3812097C9F18B010F
:105C300088858F70853021F5CE010E9431C2801792
:105C4000110671F16CF1602FCE010E949FC1FC0121
:105C5000892B31F180858F70823039F461857285AE
:105C6000838594850F94332106C08330C9F4618500
:105C7000728583859485DF91CF911F910F9108954F
:105C8000672B71F4823029F469857A858B859C8530
:105C9000E9CF833029F469857A858B859C85EBCFA4
:105CA00060E070E0CB01E7CF0F931F93CF93DF93BA
:105CB000FC01C281D3812097F9F088858F708230F2
:105CC00049F4672BC9F489859A85DF91CF911F919B
:105CD0000F910895853081F48B01CE010E9431C26D
:105CE0008017110649F044F0602FCE010E949FC139
:105CF000FC0181859285E9CF90E080E0E6CF0F93AB
:105D00001F93CF93DF93EC018B017B836A8381E840
:105D100092E09983888370E060E0C8010E94542E6D
:105D200097FD19C09D838C83D8011296ED91FC914B
:105D30003097C1F090859F70923089F0953091F442
:105D4000CF010E9431C290E09F838E83DF91CF917B
:105D50001F910F910895919581959109E3CF81E06D
:105D600090E0F2CF90E080E0EFCF8F929F92AF92E1
:105D7000BF92CF92DF92EF92FF920F931F93CF9338
:105D8000DF93EC01888199810E9431C2082F10E0D5
:105D90000430110554F40E9404C7BC018881998124
:105DA0000E9411C70F5F1F4FF3CF60E08881998178
:105DB0000E949FC17C01009769F1DC0118968C91CB
:105DC00018978F70843041F51996CD90DC90C114EE
:105DD000D10401F1F60180818823E1F08BE2882E65
:105DE0008FE0982EB12CA12C1A2DC4010F94471BC3
:105DF000AC01B401C6010F94601B892B09F42FC1BB
:105E0000FFEFAF1ABF0A89E0880E911CA7E1AA161E
:105E1000B10451F71FEF04C08230E1F7F70111859B
:105E20001887E880F98061E0C7010E949FC16C017A
:105E30009B838A8362E0C7010E949FC19D838C83FC
:105E400064E0C7010E949FC17C019F838E8315314E
:105E500008F031C0E12FF0E08827EE5CF04D8F4F65
:105E60000D94ED22682F682F682F472F5B2F5B2F33
:105E70005B2F5B2F5B2F5B2F5B2F5B2F762FA52F6D
:105E8000882F5B2FB22F682F06305B2F21308AE0DE
:105E900090E00F94FE188C01BE010E947F2E83E2D9
:105EA00093E0D80111969C938E9319961C921E92A2
:105EB00018971A870987DF91CF911F910F91FF9053
:105EC000EF90DF90CF90BF90AF909F908F9008950C
:105ED00088E090E00F94FE188C01BE010E947F2E96
:105EE0008FEF92E0F80191838083E3CF8EE090E022
:105EF0000F94FE188C01DC011396DC93CE9312975D
:105F00008DEA93E08D939C93C8010E9422A4D1CF87
:105F100086E090E00F94FE18FC01D383C2838DEDE0
:105F200092E091838083E114F104C9F0D7011896BF
:105F30008C9118978F70823091F416968D919C9168
:105F400095838483FA87E987B6CF86E090E00F9443
:105F5000FE18FC01D383C2838BEB92E0E2CF90E08A
:105F600080E0EECF8BE090E00F94FE188C01FC01F6
:105F7000D383C2838BE893E091838083168270E0A1
:105F800060E0CE010E94542E97FD2DC0D8011596D9
:105F90009C938E931497D80114968D919C910097A1
:105FA00019F0863491052CF080E290E0F801958399
:105FB000848361E070E0CE010E940E2E20E030E08C
:105FC0004AE754E40F9492210F940524611571055A
:105FD0008105910589F0D80117966D937D938D9376
:105FE0009C931A9766CF919581959109F8019583B5
:105FF000848381E08683CFCF88E893E1A0E0B0E09E
:10600000F80187839087A187B28753CF86E090E01D
:106010000F94FE18FC01D383C28389E693E0918339
:10602000808315821482C114D10409F48BCFD60168
:1060300018968C918F70863009F084CFD582C482F7
:1060400081CF84E090E00F94FE18FC01D383C283DB
:1060500027E433E0318320839A8789872CCFC601D8
:106060000E94A8F68A2D90E0B0E0A0E0F7018187B9
:106070009287A387B4878085807F82608087D0CE17
:10608000CF92DF92EF92FF926A017B0163E0FC0105
:10609000808191810E949FC1FC01892BA9F080859C
:1060A0008D7091F4C094D094E094F094CC24CA9470
:1060B00081859285A385B4858C219D21AE21BF2148
:1060C00081879287A387B487FF90EF90DF90CF906E
:1060D0000895CF92DF92EF92FF926A017B0163E015
:1060E000FC01808191810E949FC1FC01892BA9F054
:1060F0009085892F8D7089F4907F92609087CC2451
:10610000FF2441855285638574854C295D296E295C
:106110007F294187528763877487FF90EF90DF90D4
:10612000CF900895CF92DF92EF92FF926A017B01A8
:1061300063E0FC01808191810E949FC1009791F0F2
:10614000FC0120852F70223069F46185728583857A
:1061500094856C217D218E219F21FF90EF90DF900F
:10616000CF90089560E070E0CB01F7CFAF92BF927F
:10617000CF92DF92EF92FF920F931F93CF93DF9313
:10618000CDB7DEB7CD56D1090FB6F894DEBF0FBE3E
:10619000CDBF5C01A7960FAFA797A8961FAFA89792
:1061A000A9962FAFA997AA963FAFAA97AB964FAFE4
:1061B000AB97AC965FAFAC97AD966FAFAD97AE9621
:1061C0007FAFAE9723961FAE1EAE2397FE01ED5B09
:1061D000FF4F82E1DF011D928A95E9F772961192D5
:1061E000119287E0DF011D928A95E9F7CE018A5965
:1061F0009F4F0E94CD22F0FE2CC0A796EFADA7972F
:10620000E83108F050C1F0E08827E65FFE4C8F4F80
:106210000D94ED22593222315032533253325032E2
:106220002231533253325332533253325332533278
:106230002231223153325332533222312231223130
:10624000533259326FED7DE0CE018B5A9F4F0F9440
:10625000401B0E9445C1882309F407C18091680E44
:10626000811103C1C114D10409F05EC030E020E007
:1062700043E050E060E4CE0101960F940D0ED5018D
:10628000ED91FC91608171814FE350E0CE01019668
:106290000F946A27F1FE10C1A7968FADA7978230A1
:1062A00009F40AC1853009F407C1A8968FADA897F3
:1062B00082958F709FE0980F9F70923018F0883011
:1062C00009F0FAC001E020E032E044E150E0BE0114
:1062D0006F5B7F4FCE018A599F4F0E94AC20BE0159
:1062E0006F5B7F4FCE0101960E946BD262EC7DE026
:1062F00082E59DE00E9431F3BE016F5F7F4F82E532
:106300009DE00E94CBF26FEB7DE082E59DE00E9474
:1063100031F3BE016F5B7F4F82E59DE00E94CBF2BF
:1063200082E59DE00E947BF1A8968FADA897807FC3
:10633000870100271072882311F0F1FC04C00115B9
:10634000110509F4F5C030E020E043E050E060E4DE
:10635000CE0101960F940D0ED501ED91FC91608157
:1063600071814FE350E0CE0101960F946A27C1146A
:10637000D10469F06EE875E0CE0101960F944427D0
:106380004FE350E0B601CE0101960F946A276EE804
:1063900075E0CE0101960F9444274FE350E064E886
:1063A0007DE00115110511F46AE77DE0CE0101964B
:1063B0000F94501BA8968FADA89782958F7084502C
:1063C000823008F09FC067E1CE018A599F4F0E943A
:1063D0001F1B6F962FAF6F97A0963FAFA097A19608
:1063E0004FAFA197A2965FAFA297A3966FAFA39767
:1063F000A4967FAFA497A5968FAFA597A6969FAFBB
:10640000A69700E020E033E044E150E0BE016F5B7E
:106410007F4FCE018A599F4F0E94AC206AE67DE0F3
:1064200082E59DE00E9431F3BE016F5F7F4F82E500
:106430009DE00E94CBF267E67DE082E59DE00E9450
:1064400031F3BE016F5B7F4F82E59DE00E94CBF28E
:1064500082E59DE00E947BF10E9445C1882329F0DE
:106460008091680E882309F455C0A701FF0C660BC4
:10647000770BC5010E94693090E080E0C359DF4F7F
:106480000FB6F894DEBF0FBECDBFDF91CF911F9145
:106490000F91FF90EF90DF90CF90BF90AF90089555
:1064A00068EE7DE0D1CE68EC7DE082E59DE00E9463
:1064B00031F3E894F0F8CDCEF0FE36CF66968FAD8E
:1064C0006697882309F430CFBE016B5A7F4FCE0107
:1064D00001960E946BD269EB7DE082E59DE00E940F
:1064E00031F3BE016F5F7F4F82E59DE00E94CBF2EA
:1064F00066EB7DE082E59DE00E9431F3BE016B5AC0
:106500007F4F0ACF20E032E0012B11F020E033E092
:1065100000E07ACFBE016F5B7F4FCE0101960E94F3
:106520006BD240E052E060E070E0C5010E94403074
:10653000F0FE90C0A796EFADA797E150E53118F5B2
:10654000F0E08827E955FD4C8F4F0D94ED22B233D2
:10655000C332C332C332C332B233C332C332C332A3
:10656000C332C332C332C332B733AF33C332C332A1
:10657000C332BC32A933AC3361E87EE0CE018B5A22
:106580009F4F0F94401B30E020E043E050E060E478
:10659000CE0101960F940D0ED501ED91FC91608115
:1065A00071814FE350E0CE0101960F946A27C11428
:1065B000D10469F06EE875E0CE0101960F9444278E
:1065C0004FE350E0B601CE0101960F946A276EE8C2
:1065D00075E0CE0101960F9444274FE350E065E744
:1065E0007DE0CE0101960F94501B61E67DE082E5CF
:1065F0009DE00E9431F3BE016F5F7F4F82E59DE019
:106600000E94CBF26EE57DE082E59DE00E9431F3D1
:10661000BE016B5A7F4F82E59DE00E94CBF282E57E
:106620009DE00E947BF10E9445C1882309F41DCFA3
:106630008091680E811119CFBE016B5A7F4FCE0138
:1066400001960E946BD240E051E060E070E0C5012D
:106650000E944030F2FE7AC040E050E061E070E01D
:10666000C5010E949230672B682B692B09F482C008
:1066700069E37EE0CE018B5A9F4F0F94401B30E0C0
:1066800020E043E050E060E4CE0101960F940D0E4F
:10669000D501ED91FC91608171814FE350E0CE0115
:1066A00001960F946A27C114D10469F06EE875E071
:1066B000CE0101960F9444274FE350E0B601CE017E
:1066C00001960F946A276EE875E0CE0101960F944B
:1066D00044274FE350E06DE97DE0CE0101960F9431
:1066E000501B68E57DE082E59DE00E9431F3BE012C
:1066F0006F5F7F4F82E59DE00E94CBF265E57DE014
:1067000082E59DE00E9431F3BE016B5A7F4F82E526
:106710009DE00E94CBF282E59DE00E947BF10E9409
:1067200045C1882309F4A1CE8091680E81119DCEC8
:10673000BE016B5A7F4FCE0101960E946BD240E0A2
:1067400054E060E070E0C5010E94403081E090E0DC
:1067500095CE6AE87EE012CF63E97EE00FCF6DE56B
:106760007EE00CCFF5018085853009F00CCF64E523
:106770007EE004CF40E050E062E070E0C5010E949E
:106780009230672B682B692B19F06BE47EE072CF97
:1067900060E37EE06FCFAF92BF92CF92EF920F9304
:1067A0001F93CF93DF93CDB7DEB7C856D1090FB68D
:1067B000F894DEBF0FBECDBF5C01A2960FAFA297CB
:1067C000A3961FAFA397A4962FAFA497A5963FAF0C
:1067D000A597A6964FAFA697A7965FAFA797A8963F
:1067E0006FAFA897A9967FAFA9979E2D28E0FE01CD
:1067F000EF59FF4FDE01A75ABF4F01900D922A9526
:10680000E1F7A296EFADA297E150ED3008F0F2C0AB
:10681000EC2CF0E08827E05FFB4C8F4F0D94ED22CD
:1068200087349034EE34F834E4341D347E34FA3452
:10683000FA349934AB34D134BE34992331F0C501E4
:106840000E946317009709F449C067E0CE01875A98
:106850009F4F0E941F1B60E279E082E59DE00E944D
:1068600031F34AE050E06A966FAD6A9782E59DE0A9
:106870000E9498F165E179E082E59DE00E9431F3A4
:10688000CE01875A9F4F0E94461FAB01BC012AE0F0
:1068900030E082E59DE00E943AF282E59DE00E94B0
:1068A0007BF16A960FAD6A976B961FAD6B976C96EE
:1068B0002FAD6C976D963FAD6D976E964FAD6E9701
:1068C0006F965FAD6F97A0966FADA097A1967FADC5
:1068D000A197C5010E948B1F81E090E0C859DF4F4E
:1068E0000FB6F894DEBF0FBECDBFDF91CF911F91E1
:1068F0000F91EF90CF90BF90AF900895911105C088
:10690000C5010E946317009749F366E09FCF992362
:1069100029F0C5010E946317009701F362E096CF4A
:10692000911105C0C5010E9463170097B9F261E09B
:106930008DCF40E050E061E070E0C5010E949230F0
:10694000672B682B692B29F4C5010E9463170097F8
:1069500029F26BE07BCF40E050E061E070E0C501E0
:106960000E949230672B682B692B31F0C5010E9481
:106970006317009709F4B2CF6AE068CF40E050E0B7
:1069800062E070E0C5010E949230672B682B692B92
:1069900031F0C5010E946317009709F49FCF6CE0A6
:1069A00055CF40E050E062E070E0C5010E949230B7
:1069B000672B682B692B31F4C5010E946317009780
:1069C00009F48CCF6DE042CF911106C0C5010E9441
:1069D0006317009709F482CF63E038CF992331F031
:1069E000C5010E946317009709F478CF65E02ECFA8
:1069F00064E02CCF90E080E071CFCF93C62F63E0AE
:106A0000FC01808191810E949FC1FC01892B21F1B1
:106A10009085892F8D7001F5907F92609087818598
:106A20009285A385B4858827BB278C2B8187928785
:106A3000A387B48761E079E082E59DE00E9431F3AD
:106A40004AE050E06C2F82E59DE00E9498F182E5DB
:106A50009DE0CF910C947BF1CF910895CF92DF927E
:106A6000FF920F931F93CF93DF93F12C6115710564
:106A700009F499C06A01EB018C01CB010E94622DDF
:106A8000F82E882309F48FC0D2FE09C0D8018C915A
:106A90008B3009F44BC0E8F58A3009F44CC0D0FEC5
:106AA00009C0F801608186EF860F843018F0CE01AE
:106AB0000E94FD34D1FE6EC0D80114964D915D91B7
:106AC0006D917C91179711968C9182958F7087307C
:106AD00038F0893008F43EC08A50823008F46CC027
:106AE000CE010E94E915EC81FD81309709F452C076
:106AF00080858F709EEF980F923010F081114AC000
:106B0000D80111969C91907F80858F70892B80870A
:106B100041C08C30B9F040E050E062E070E08D3070
:106B200009F0BDCFCE010E946930B9CF40E050E0FE
:106B300061E070E0F7CF40E050E061E070E0CE014E
:106B40000E94403040E050E062E070E0CE010E94E0
:106B50004030A5CFEC81FD813097E1F080858F70CA
:106B60009EEF980F923010F0811114C04187528728
:106B700063877487EC81FD818085807F8360808757
:106B8000EC81FD818085982F907F8F708067903693
:106B900009F4BDCF61E970E182E59DE00E9431F327
:106BA000C8010E94CD228F2DDF91CF911F910F91AF
:106BB000FF90DF90CF900895CE010E94E915EACFB3
:106BC00063E0FC01808191810E949FC1009719F0D0
:106BD000FC01818508958FEF0895CF92DF92EF92A7
:106BE000FF920F931F93CF93DF936115710509F403
:106BF00058C06A017B018C01CB010E94622DD82F05
:106C0000882371F1D70114968D919C910097E9F139
:106C1000FC01C0852C2F2F703EEF320F323010F068
:106C2000211128C0C295CF70D0FE59C0C7010E9463
:106C3000E035F8018083CC2351F1C295C07F81817A
:106C40008F70C82BC183D7011496ED91FC9181857B
:106C50009285A385B485F80184839583A683B78341
:106C60008D2FDF91CF911F910F91FF90EF90DF90CB
:106C7000CF900895253049F460E00E949FC10097AD
:106C800021F0DC011896CC91CDCFC0E0CDCFD7015B
:106C90001496ED91FC9180858F70823021F08330C5
:106CA00081F0D0E0DDCF4185528563857485F801A0
:106CB00081818F70806A8183448355836683778363
:106CC000CFCF4185528563857485F80181818F70AE
:106CD000806781834483558366837783C1CFCC23C8
:106CE000B1F2C295C07FF801AACFAF92BF92CF9206
:106CF000DF92EF92FF920F931F93CF93DF9300D019
:106D000000D01F921F92CDB7DEB75C017B0160FF00
:106D100003C0E894E0F8F4F8F4FC0DC00F94560FAB
:106D2000663971058105910530F08091810E909151
:106D3000820E059719F5A70144275770052E000C00
:106D4000660B770BC5010E94693064E47DE082E543
:106D50009DE00E9431F38FEF9FEF28960FB6F894D5
:106D6000DEBF0FBECDBFDF91CF911F910F91FF907E
:106D7000EF90DF90CF90BF90AF90089519821A8264
:106D80001B821C821D821E821F8218868A818F7040
:106D90008A8340E053E0B501CE0101960E94ED35B3
:106DA00040E057E060E070E0C5010E949230E62AC2
:106DB000F72AD12CC12C09811A812B813C814D816C
:106DC0005E816F817885C5010E94B630C6CFCF93B2
:106DD000DF93EC0140E053E060E070E00E9492300D
:106DE000611571058105910599F02091810E309111
:106DF000820E2630310561F4CE010E94753640E0E6
:106E000053E060E070E0CE01DF91CF910C94403010
:106E1000DF91CF9108958F929F92AF92CF92EF9290
:106E2000FF920F931F93CF93DF9300D000D01F9258
:106E30001F92CDB7DEB74C0109831A832B833C83A5
:106E40004D835E836F8378876EE478E082E59DE012
:106E50000E9431F3CE0101960E94CD2289818111D9
:106E600030C00A810F70013089F140F1023019F011
:106E700010E00530F1F5D401ED91FC91068CF78D11
:106E8000E02D09811A812B813C814D815E816F81CA
:106E90007885C401199581E090E028960FB6F894A2
:106EA000DEBF0FBECDBFDF91CF911F910F91FF903D
:106EB000EF90CF90AF909F908F900895CC24C39483
:106EC000DACF813071F1823009F451C061E478E0A9
:106ED00082E59DE00E9431F34AE050E0698182E55D
:106EE0009DE00E9498F182E59DE00E947BF101E027
:106EF00010E061E378E082E59DE00E9431F34AE032
:106F000050E0B80182E59DE00E9482F282E59DE0BA
:106F10000E947BF1CE0101960E94CD2290E080E09C
:106F2000BCCFCE0101960E94AEC14497B8F46EE189
:106F300070E0CE0101960E94AB1EF4016281738164
:106F400040E052E0CE0101960E942E3560E072E1F1
:106F5000D40112968D919C910E947536D401ED91C9
:106F6000FC91068CF78DE02DCC24C3948ACF1D8232
:106F70001E821F821886D401ED91FC91068CF78D3C
:106F8000E02DCC24C39402E01A812B813C8140E0A7
:106F90007DCF8F929F92AF92BF92CF92DF92EF926E
:106FA000FF920F931F93CF93DF93CDB7DEB7609718
:106FB0000FB6F894DEBF0FBECDBF8C017B0140E061
:106FC00058E060E070E00E949230672B682B692BDC
:106FD00009F0A9C062E070E0C8010E94542E6C0163
:106FE00019861A861B861C861D861E861F86188A91
:106FF0008A858F708A87D7FC96C040E052E0B8013E
:10700000CE0109960E94ED3563E070E0C8010E9450
:10701000542EAC011816190614F04FE350E081E02D
:10702000C816D10429F4EF2CFF0CFF08FF2404C07C
:1070300082E0C816D104D4F32FEF30E0D7010F94CB
:1070400004239A01550F440B550B0F9498224901C4
:107050006901C8010E94E035E82EF12C60E0CE0104
:1070600009960E94DE1D88169906F9F4CD2841F094
:1070700082E0E816F10419F185E0E816F104F9F070
:1070800081E090E060960FB6F894DEBF0FBECDBFF2
:10709000DF91CF911F910F91FF90EF90DF90CF90F4
:1070A000BF90AF909F908F900895CD2859F186E0C2
:1070B000E816F10441F081E0E816F10421F061E006
:1070C000C8010E94FD34B401CE0109960E94851DBD
:1070D00040E052E0B801CE0109960E942E3582E0D0
:1070E000E816F10421F085E0E816F10429F460E0E7
:1070F00071E0C8010E94753660E072E0C8010E942C
:107100007536BECF85E0E816F10409F4B9CF82E008
:10711000E816F10409F4B4CF62E0C8010E94FD341E
:1071200060E071E0EBCF90E080E0ACCF81E090E0F8
:1071300008950F931F93CF93DF9300D000D01F9239
:107140001F92CDB7DEB719821A821B821C821D8264
:107150001E821F8218862A812F702A83FC010281D9
:107160001381C8010E94E035813041F020F0823067
:1071700011F0853081F490E080E002C081E090E081
:1071800028960FB6F894DEBF0FBECDBFDF91CF912A
:107190001F910F91089540E052E0B801CE01019691
:1071A0000E94ED3560E0CE0101960E94DE1DE8CF21
:1071B0008F929F92AF92BF92CF92DF92EF92FF9207
:1071C0000F931F93CF93DF93CDB7DEB767970FB6BB
:1071D000F894DEBF0FBECDBF8C017B014C018BE06C
:1071E000880E911C9F8A8E8AF8011286118613865A
:1071F000148E138E672B09F463C0A090830EB09099
:10720000840EA114B10409F45BC06FE270E0C70101
:107210000F944F276C01892B09F44AC0F701DE0156
:10722000119690E080E0BD012191222341F02F32A0
:1072300031F08431910519F02D930196F5CF860F29
:10724000971FFC011082C5010E9427C1F80191839C
:107250008083B6016F5F7F4F4FE050E0C4010F9411
:107260008827CE0146960E942C2DF801948F838F9B
:107270008E899F89892B09F41386C8010E94622D8B
:10728000882319F0C8010E94B52E67960FB6F894AE
:10729000DEBF0FBECDBFDF91CF911F910F91FF9049
:1072A000EF90DF90CF90BF90AF909F908F90089518
:1072B000B701C5010E9427C1F80191838083DDCF0A
:1072C000F80111821082D9CFDC0119968D919C9121
:1072D000009739F0DC01ED91FC910280F381E02D03
:1072E000199408958F929F92AF92BF92CF92DF929E
:1072F000EF92FF920F931F93CF93DF93CDB7DEB73B
:10730000CD55D1090FB6F894DEBF0FBECDBF8C01AD
:107310006B016115710519F041155105D1F460E754
:1073200072E182E59DE00E9431F367E672E182E559
:107330009DE00E9431F3B80182E59DE00E94CBF20E
:1073400065E672E182E59DE00E9431F382E59DE011
:1073500032C0460F571FDA011C920F94560F4B0193
:1073600063E672E182E59DE00E9431F34AE050E07D
:10737000B40182E59DE00E9482F260E672E182E55E
:107380009DE00E9431F3B80182E59DE00E94CBF2BE
:107390006DE572E182E59DE00E9431F3BAE38B1660
:1073A000B1E09B06F4F460E572E18BEA9CE00E9498
:1073B00031F38BEA9CE00E947BF1C35ADF4F0FB69A
:1073C000F894DEBF0FBECDBFDF91CF911F910F911B
:1073D000FF90EF90DF90CF90BF90AF909F908F90F5
:1073E00008956EE472E182E59DE00E9431F3B601FA
:1073F00082E59DE00E94CBF26CE472E182E59DE0C3
:107400000E9431F382E59DE00E947BF11A8219828D
:10741000FE0133968EE3DF011D928A95E9F7809194
:10742000810E9091820E059791F563E070E0C8019E
:107430000E94A1177C01892BE9F5E091D10AF09116
:10744000D20A808180FFB9CF61E070E0C8010E945C
:10745000A117892B09F4B1CF64E270E0C8010F9441
:107460009727892B09F0A9CF64E372E182E59DE0BB
:107470000E9431F3B80182E59DE00E94CBF282E5E3
:107480009DE00E947BF1C8010E9444CE96CF61E04E
:1074900070E0C8010E94A1177C01892B49F562E0C8
:1074A00070E0C8010E94A1177C0169E272E1892B9A
:1074B00009F448CFE00EF11E60E272E1C7010F94BB
:1074C000371B892BE9F4F60101900020E9F7319789
:1074D000EC19FD093297A0F0C8010E9444CEF601D4
:1074E0008081882309F469CFC6010E94F1F565CF38
:1074F0004FE350E0B801CE0101960F948827DACF10
:1075000064E270E0C8010F949727892B09F055CFEA
:10751000B701CE018F5B9F4F0E94D838CE018F5BA1
:107520009F4F0E94622D882339F1B601CE018F5BF7
:107530009F4F0E9458C818161906F4F489818823B1
:10754000D9F08091810E9091820E0597A9F068E0A4
:1075500072E182E59DE00E9431F3BE016F5F7F4FD3
:1075600082E59DE00E94CBF282E59DE00E947BF1E6
:10757000CE0101960E9444CECE018F5B9F4F0E94A8
:1075800064391BCFCF93DF93EC01798368831A862C
:1075900019861B861C8E1B8E0E94622D882329F063
:1075A000CE01DF91CF910C94B52EDF91CF9108954C
:1075B000CF93DF93EC01FB01248135814081518120
:1075C000628173810E943AF2CE01DF91CF910895DA
:1075D000CF92DF92EF92FF921F93CF93DF9300D071
:1075E00000D0CDB7DEB764E772E181EA9CE00E948B
:1075F00031F385E8E82E8CE0F82E10E090E1C92EFA
:10760000D12CF70181917F01803130F460E975E080
:1076100081EA9CE00E94CBF2153041F1F7013197ED
:10762000808190E0B0E0A0E089839A83AB83BC8343
:10763000DE82CD82BE016F5F7F4F81EA9CE00E94B7
:10764000D83A62E772E10E9431F31F5F1630C9F643
:1076500026960FB6F894DEBF0FBECDBFDF91CF9157
:107660001F91FF90EF90DF90CF90089580918A0C4A
:1076700090E0B0E0A0E089839A83AB83BC83DE8294
:10768000CD82BE016F5F7F4F81EA9CE00E94D83AB5
:107690000E947BF1DACFEF92FF920F931F93CF936B
:1076A000DF9300D000D0CDB7DEB77C018B0160EC5A
:1076B0007EE082E59DE00E9431F3D701ED91FC91DF
:1076C0006081718182E59DE00E94CBF267EB7EE0F4
:1076D00082E59DE00E9431F3012E000C220B330B5A
:1076E00009831A832B833C8380E190E09E838D8302
:1076F000BE016F5F7F4F82E59DE00E94D83A0E94F5
:107700007BF140E058E060E070E0C7010E94693022
:1077100026960FB6F894DEBF0FBECDBFDF91CF9196
:107720001F910F91FF90EF9008953F924F925F92BB
:107730006F927F928F929F92AF92BF92CF92DF9281
:10774000EF92FF920F931F93CF93DF93CDB7DEB7E6
:107750002C970FB6F894DEBF0FBECDBF5C01362E5E
:10776000972E3A01690161E27FE082E59DE00E9487
:1077700031F34AE050E0632D792D82E59DE00E94CF
:1077800082F269E17FE082E59DE00E9431F3C3016E
:10779000B0E0A0E08F839887A987BA8730E1432EB5
:1077A000512C5C864B86BE01695F7F4F82E59DE070
:1077B0000E94D83A4C0165E17FE00E9431F34AE033
:1077C00050E0B601C4010E9482F26DE07FE0C40186
:1077D0000E9431F3C701B0E0A0E089839A83AB83B4
:1077E000BC835E824D82BE016F5F7F4FC4010E94E9
:1077F000D83A0E947BF1809123099091240970E08E
:1078000060E0892B09F047C081E090E09093240963
:107810008093230926E040E855E260E070E086E0CE
:107820009AE00E943DF43092F60A86E09AE0909346
:10783000F50A8093F40A1092010C1092030C109236
:10784000020C0130110509F44EC00CF041C0012BAF
:1078500009F44EC0C114D10409F457C082E0C8161F
:10786000D10409F062C070927C0B60927B0B109285
:107870007E0B10927D0BF092800BE0927F0B86E0E6
:107880000E94F4D21092240910922309882309F44B
:1078900056C0682F70E0C5010E944B3B90E080E02D
:1078A0002C960FB6F894DEBF0FBECDBFDF91CF91FF
:1078B0001F910F91FF90EF90DF90CF90BF90AF900E
:1078C0009F908F907F906F905F904F903F90089522
:1078D0000330110581F00430110509F0BBCFFE24FF
:1078E000EF24FE24B7CFFE2CEE24EE24EA94B2CF90
:1078F000FF24FA94AFCFEF2821F492E0E92EF12C87
:10790000EECFEE24E394F12CEACF70927C0B6092E0
:107910007B0B90E080E0EE2011F080E09FEF9093F1
:107920007E0B80937D0B85E0ABCF61EF7EE082E53F
:107930009DE00E9431F3109224091092230981E006
:1079400090E0AECF2F923F924F925F926F927F92D4
:107950008F929F92AF92BF92CF92DF92EF92FF925F
:107960000F931F93CF93DF93CDB7DEB72C970FB64E
:10797000F894DEBF0FBECDBF5C0109831A832B8351
:107980003C834D835E836F837887CE0101960E948E
:10799000AEC11C01023011F0053011F4312C212C44
:1079A000F50102811381F80180858F70853009F01F
:1079B0007FC0C8010E9431C2E82EF12CF2E0EF1620
:1079C000F1040CF475C060E0C8010E949FC1FC0185
:1079D000818592859C878B8761E0C8010E949FC149
:1079E000FC01418452846384748488248A94982C92
:1079F000F2E0EF16F10459F062E0C8010E949FC165
:107A0000FC0181849284F3E0EF16F104A1F48FE38A
:107A100090E09A87898792E0C92ED12C29853A85F2
:107A2000D1010F94FC2224E630E040E050E00F94B6
:107A3000982279011CC063E0C8010E949FC1FC012B
:107A4000818592859A87898782E0C82ED12CF4E0BF
:107A5000EF16F10439F064E0C8010E949FC1FC01F7
:107A6000C184D28489859A857101892BB9F68401F4
:107A70009601A2016B857C85C5010E94953B2C96E1
:107A80000FB6F894DEBF0FBECDBFDF91CF911F912F
:107A90000F91FF90EF90DF90CF90BF90AF909F90AD
:107AA0008F907F906F905F904F903F902F900895B0
:107AB00090E080E0E4CF8F929F92AF92BF92DF92EE
:107AC000EF92FF920F931F93CF93DF93CDB7DEB763
:107AD000A5970FB6F894DEBF0FBECDBF7C010E8F09
:107AE0001F8F28A339A34AA35BA36CA37DA3CE0158
:107AF0004E960E94FF1E4B015C01D7011296ED913C
:107B0000FC9180858F70843009F0E9C0102F618569
:107B10007285CE0101960E94D838CE0101960E944E
:107B2000622D882309F44AC08985893009F046C04E
:107B300070E060E0CE0101960E94542E082FD92EED
:107B400064EE7EE082E59DE00E9431F34AE050E081
:107B5000602F7D2D82E59DE00E9482F262EE7EE044
:107B600082E59DE00E9431F3B501A40182E59DE02C
:107B70000E9433C66CED7EE082E59DE00E9431F309
:107B8000612F70E04AE050E082E59DE00E9482F2C1
:107B900082E59DE00E947BF1809123099091240968
:107BA000892B29F140E053E0B701CE014E960E94A7
:107BB0002E3570E060E0C7010E944B3B10E000E012
:107BC000CE0101960E946439C801A5960FB6F894BB
:107BD000DEBF0FBECDBFDF91CF911F910F91FF9000
:107BE000EF90DF90BF90AF909F908F90089581E0CD
:107BF00090E0909324098093230926E040E855E221
:107C000060E070E086E09AE00E943DF40093F60A9E
:107C100086E09AE09093F50A8093F40A1092010CA2
:107C20001092030C1092020CE981FA81153021F0B8
:107C30001F3011F0123011F580858F70808770E051
:107C400060E083ED97E090937C0B80937B0B109228
:107C50007E0B10927D0B7093800B60937F0B86E000
:107C60000E94F4D2109224091092230901E010E03E
:107C7000882309F4A5CF682F70E09DCF80858F7091
:107C80008061808722E538EB42E152E4C501B4010E
:107C90000F94202320E030E040E251E40F94922141
:107CA0002DEE3EE94CE35EE30F948C234B015C0127
:107CB00020E030E0A9010F94342420E030E040E0DF
:107CC0005FE387FD07C0C501B4010F9420230F9423
:107CD000FE23B7CFC501B4010F941F23F8CF10E0E6
:107CE00000E072CFCF92DF92EF92FF920F931F933B
:107CF000CF93DF9300D000D01F921F92CDB7DEB795
:107D00007C0109831A832B833C834D835E836F83BD
:107D10007887CE0101960E94AEC18C0189818823AB
:107D200059F09A819F70923008F0BAC0823011F0F9
:107D3000853011F410E000E070E060E0C7010E94BF
:107D4000542ED82EC92E64ED7EE082E59DE00E947F
:107D500031F34AE050E06D2D7C2D82E59DE00E94DC
:107D600082F262ED7EE082E59DE00E9431F34AE01E
:107D700050E0B80182E59DE00E9482F282E59DE03C
:107D80000E947BF18091230990912409892BE9F0CD
:107D900040E053E0B701CE0101960E942E3570E01D
:107DA00060E0C7010E944B3B90E080E028960FB650
:107DB000F894DEBF0FBECDBFDF91CF911F910F9121
:107DC000FF90EF90DF90CF90089581E090E0909346
:107DD00024098093230926E040E855E260E070E042
:107DE00086E09AE00E943DF4D092F60A86E09AE09E
:107DF0009093F50A8093F40A1092010C1092030CF0
:107E00001092020C80ED97E090937C0B80937B0B9B
:107E100010927E0B10927D0B01151105E1F185E0AA
:107E200090E09093800B80937F0B86E00E94F4D2C9
:107E3000D82E64E670E080E090E00E946AD1D11014
:107E40000AC06BEC7EE082E59DE00E9431F382E5A2
:107E50009DE00E947BF182ED97E090937C0B8093F4
:107E60007B0B10927E0B10927D0B24E6209FC001AD
:107E7000219F900D11249093800B80937F0B86E0BF
:107E80000E94F4D21092240910922309882359F0F9
:107E9000682F70E086CF1092800B10927F0BC5CFB9
:107EA0008FEF9FEF83CF81E090E080CF2F923F92C2
:107EB0004F925F926F927F928F929F92AF92BF92FA
:107EC000CF92DF92EF92FF920F931F93CF93DF93A6
:107ED000CDB7DEB7C75CD1090FB6F894DEBF0FBED1
:107EE000CDBF1C01CF54DF4F0883C15BD040CE54BF
:107EF000DF4F1883C25BD040CD54DF4F2883C35B74
:107F0000D040CC54DF4F3883C45BD040CB54DF4FDC
:107F10004883C55BD040CA54DF4F5883C65BD0400E
:107F2000C954DF4F6883C75BD040C854DF4F7883A4
:107F3000C85BD040C754DF4FF982E882C95BD040AC
:107F4000C254DF4FC882CE5BD040C154DF4FA882FD
:107F5000CF5BD0400F94560F6B01C054DF4F798335
:107F60006883C05CD040683C7105B4F467E97BE08D
:107F70008BEA9CE00E9431F34AE050E0B6018BEAC4
:107F80009CE00E9482F28BEA9CE00E947BF1AA2492
:107F9000AA94BA2C0C9477490E949DD1CC53DF4F00
:107FA000688379838A839B83C45CD040CE54DF4F3F
:107FB0008881C25BD0408F70282F30E0C454DF4FDF
:107FC00039832883CC5BD0408091810E9091820EC2
:107FD000CE53DF4F99838883C25CD040C754DF4FB4
:107FE000E881F981C95BD040309721F0808181110F
:107FF0000C94734ED1011B968C91882341F0C101E2
:108000000B96C754DF4F99838883C95BD040C45413
:10801000DF4FE881F981CC5BD040EF2B11F00C945D
:10802000CF4EC754DF4FE881F981C95BD04030970C
:1080300011F00C947C4ED1015B960D90BC91A02D5B
:10804000C454DF4FB983A883CC5BD040AB2B11F471
:108050000C94CF4ECE54DF4F8881C25BD0408F70DE
:1080600011F00C94CF4EC454DF4F6881CC5BD040EC
:10807000CE018F549F4F0E94F81AC756DF4F2883B6
:10808000C959D040C656DF4F3883CA59D040C5566B
:10809000DF4F4883CB59D040C456DF4F5883CC596B
:1080A000D040C356DF4F6883CD59D040C256DF4F12
:1080B0007883CE59D040C156DF4F8883CF59D04006
:1080C000C056DF4F9883C05AD0400C94CF4ED10198
:1080D0002D913C91232B09F45ACFC454DF4FE881F2
:1080E000F981CC5BD040349799F5C154DF4FE880DB
:1080F000CF5BD040CF54DF4F0881C15BD040CE541E
:10810000DF4F1881C25BD040CD54DF4F2881C35B65
:10811000D040CC54DF4F3881C45BD040CB54DF4FCC
:108120004881C55BD040CA54DF4F5881C65BD04000
:10813000C954DF4F6881C75BD040C854DF4F788196
:10814000C85BD040C1010E948B1F5C010C94774931
:1081500028E0FE01EF54FF4FDE01A755BF4F01900D
:108160000D922A95E1F7CF54DF4F1881C15BD040C3
:10817000143009F412C348F4112309F469C0912C96
:10818000812CAA24AA94BA2C8CC388EF810F823048
:10819000B0F788E0FE01EF54FF4FDE011196019029
:1081A0000D928A95E1F7CE54DF4F8881C25BD040B3
:1081B000807F09F485C3CE018F549F4F0E943E20DB
:1081C0004B015C0181149104A104B10409F478C34A
:1081D000193041F4B094A09490948094811C911C27
:1081E000A11CB11CB101CE018F549F4F0E942FC71B
:1081F00060E0CE018F549F4F0E941F1B6A962FAFE5
:108200006A976B963FAF6B976C964FAF6C976D9676
:108210005FAF6D976E966FAF6E976F967FAF6F97EC
:10822000A0968FAFA097A1969FAFA197C454DF4FA0
:10823000A881B981CC5BD040A230B10509F49AC3C2
:108240000CF044C3AB2B09F4D3C3912C812C58C53B
:1082500019821A821B821C821D821E821F8218862E
:108260002A812F702A83CE54DF4F2881C25BD040F1
:10827000207F09F484CFC454DF4F08811981CC5B7F
:10828000D0400A30110509F440C254F4011511051B
:1082900071F10230110509F4E1C0912C812C2CC23E
:1082A000C454DF4F28813981CC5BD0402B3031055D
:1082B00009F4D3C12C30310581F7B101CE0101960B
:1082C0000E942FC7CE018F549F4F0E948A20BC016D
:1082D000CE0101960E941B2388E0FE013196DE014B
:1082E000AF54BF4F01900D928A95E1F702C2892BDE
:1082F00059F064E57BE082E59DE00E9431F382E580
:108300009DE00E947BF1C9CFC1010E94EC4F8C011E
:1083100061E070E01816190614F070E060E04AE0C1
:1083200050E082E59DE00E9482F26EEF76E082E509
:108330009DE00E94CBF2CE018F549F4F0E94461FBA
:10834000AB01BC012AE030E082E59DE00E943AF2F8
:1083500082E59DE00E947BF1CE018F549F4F101665
:10836000110614F00C94614E0E94461F672B682B77
:10837000692B09F069C162E0CE018F549F4F0E94C2
:108380001F1BCF56DF4F2883C159D040CE56DF4F39
:108390003883C259D040CD56DF4F4883C359D040AF
:1083A000CC56DF4F5883C459D040CB56DF4F68833B
:1083B000C559D040CA56DF4F7883C659D040C956F8
:1083C000DF4F8883C759D040C856DF4F9883C859BC
:1083D000D04088248394982C31E0C554DF4F3883F3
:1083E000CB5BD0405524539442C061E0CE018F5402
:1083F0009F4F0E941F1BC757DF4F2883C958D0408B
:10840000C657DF4F3883CA58D040C557DF4F48831F
:10841000CB58D040C457DF4F5883CC58D040C357B7
:10842000DF4F6883CD58D040C257DF4F7883CE5896
:10843000D040C157DF4F8883CF58D040C057DF4F5F
:108440009883C059D04088248394982C81E0C554E7
:10845000DF4F8883CB5BD040512C09C0912C812CFD
:10846000C554DF4F1882CB5BD04055245A94B101DC
:10847000CE0101960E942FC78A81982F92959F70F6
:10848000945F9F70923060F4CE54DF4F9881C25B4E
:10849000D04092959F70923019F48F7080628A83D9
:1084A000D10118969C91973071F4CE54DF4F88819A
:1084B000C25BD040807E803211F0803421F48A810A
:1084C0008F7080628A83F101A185B285892F90E047
:1084D000109741F0ED91FC911197048CF58DE02DF2
:1084E000CD0119957C01CF54DF4F0881C15BD0408D
:1084F000CE54DF4F1881C25BD040CD54DF4F28816E
:10850000C35BD040CC54DF4F3881C45BD040CB54E8
:10851000DF4F4881C55BD040CA54DF4F5881C65BEE
:10852000D040C954DF4F6881C75BD040C854DF4F8B
:108530007881C85BD040CE0101960E945623CF5768
:10854000DF4F2883C158D040CE57DF4F3883C25801
:10855000D040CD57DF4F4883C358D040CC57DF4F72
:108560005883C458D040CB57DF4F6883C558D0409C
:10857000CA57DF4F7883C658D040C957DF4F88832A
:10858000C758D040C857DF4F9883C858D040CE0155
:1085900001960E94CD22C554DF4FF881CB5BD040BD
:1085A000FF2351F1CE54DF4F8881C25BD0408295CA
:1085B0008F709FE0980F9F70923020F08A5F8F70CD
:1085C0008230D0F48A8182958F7081508230A0F4FD
:1085D0002D8130E0AFEFB0E00F94CA222FEF61158C
:1085E00004E670078105910534F424E630E040E0AC
:1085F00050E00F9498222D8388E0FE013196DE0131
:10860000AF54BF4F01900D928A95E1F712E1912A84
:10861000F12CAA24AA94BA2CD10118968C911897FF
:10862000873009F08DC5C054DF4FE881F981C05C07
:10863000D040EE35F1400CF090C360E17BE08BEA76
:108640009CE00E9431F39FCC912C812C91E0C55489
:10865000DF4F9883CB5BD040C5CEB101CE010196F0
:108660000E942FC7CA54DF4F8881C65BD0409A81D1
:1086700092959F7039F0923049F0912C812CFF2413
:10868000F3943BC09A819F7090629A8390E0853604
:10869000910514F084E690E08E8388E0FE01319627
:1086A000DE01AF54BF4F01900D928A95E1F762E071
:1086B000CE018F549F4F0E94F81AEA962FAFEA9787
:1086C000EB963FAFEB97EC964FAFEC97ED965FAF25
:1086D000ED97EE966FAFEE97EF967FAFEF97C1589D
:1086E000DF4F8883CF57D040C058DF4F9883C058A2
:1086F000D040812CF2E19F2EF12CC554DF4F18821F
:10870000CB5BD04055245A9484CFB101CE01019661
:108710000E942FC7C954DF4F6881C75BD040C8543F
:10872000DF4F7881C85BD0407170CE0101960E9406
:108730009628C554DF4F8883CB5BD040912C812C89
:10874000FF24F3948823F1F288E0FE013196DE01E4
:10875000AF54BF4F01900D928A95E1F762E0CE01D0
:108760008F549F4F0E94F81AE2962FAFE297E3963C
:108770003FAFE397E4964FAFE497E5965FAFE59799
:10878000E6966FAFE697E7967FAFE797E8968FAFED
:10879000E897E9969FAFE997ACCFC454DF4F2881A3
:1087A0003981CC5BD0402930310509F461C0C10169
:1087B0000E94EC4F1816190674F562E0CE018F5432
:1087C0009F4F0E941F1BAA962FAFAA97AB963FAF51
:1087D000AB97AC964FAFAC97AD965FAFAD97AE96FB
:1087E0006FAFAE97AF967FAFAF97E0968FAFE09742
:1087F000E1969FAFE19788248394982CAA24AA94A9
:10880000BA2CF12C31E0C554DF4F3883CB5BD0401C
:108810005524539401CF61E0CE018F549F4F0E94A5
:108820001F1BA2962FAFA297A3963FAFA397A49624
:108830004FAFA497A5965FAFA597A6966FAFA697E3
:10884000A7967FAFA797A8968FAFA897A9969FAF37
:10885000A99788248394982CAA24AA94BA2CF12C42
:1088600081E0C554DF4F8883CB5BD040512CD4CE00
:1088700040E050E061E070E0C1010E949230672B5F
:10888000682B692BA9F040E050E061E070E0C10185
:108890000E9440308824839424E0922EAA24A3943A
:1088A000B12CF12CC554DF4F1882CB5BD040DDC01A
:1088B00040E050E061E070E0C1010E946930EACF21
:1088C00095E0892E912CA12CB12C82CCC454DF4F81
:1088D000E881F981CC5BD040EA30F10509F4B3C1FD
:1088E0003B9709F0B2CCCE54DF4F8881C25BD040B9
:1088F00082958F70823009F023C2C501B40124E64D
:1089000030E040E050E00F949822CA54DF4F888155
:10891000C65BD04090E0280F391F37FF02C030E01F
:1089200020E02536310514F024E630E0CA54DF4F4C
:108930002883C65BD04062E0CE018F549F4F0E94D7
:10894000F81A2A962FAF2A972B963FAF2B972C9683
:108950004FAF2C972D965FAF2D972E966FAF2E971A
:108960002F967FAF2F9760968FAF609761969FAFDE
:108970006197C3C1C554DF4F1882CB5BD040D10192
:1089800019968D919C911A97009709F038C0189606
:108990008C9190E000E5402E512C612C712C85309B
:1089A000910549F0412C512C3201449721F0412C82
:1089B000512C32014A94CE54DF4FE881C25BD04043
:1089C000E295EF70E150EB3008F02EC1F0E088271F
:1089D000E351FB4B8F4F0D94ED220745074514469D
:1089E00014461446E145A745A745A74538453845EF
:1089F000F1E0C554DF4FF883CB5BD040C0CFDC0142
:108A0000ED91FC91048CF58DE02D1995C3CFCB54DD
:108A1000DF4F1881C55BD040C501B40124E630E0CA
:108A200040E050E00F949822DA01C901810F911DB6
:108A3000A11DB11DB7FF03C080E090E0DC018F3FB6
:108A40009105A105B10529F024F08FEF90E0A0E099
:108A5000B0E0CB54DF4F8883C55BD040812C12E15E
:108A6000912EF12CAA24AA94BA2C55245A94D4CD30
:108A7000CB54DF4FC880D980EA80FB80C55BD040F3
:108A8000B4E68B169104A104B104DCF5A4E6B0E0D1
:108A9000A70196010F94B722860E971EA81EB91E35
:108AA0004114510461047104B9F0A30192010F94BF
:108AB000B722362F272FB501A40177FF03C040E06E
:108AC00050E0BA01832E922E5C01481559056A05C3
:108AD0007B0514F44A015B01CB54DF4F88829982F5
:108AE000AA82BB82C55BD040CE54DF4F8881C25B77
:108AF000D0408F708066CE54DF4F8883C25BD040F9
:108B0000ADCFC501B40124E630E040E050E00F9461
:108B10009822C20ED31EE41EF51E411451046104B6
:108B2000710461F0F7FE03C0C12CD12C76014C1406
:108B30005D046E047F0414F473016201CB54DF4FB3
:108B4000C882D982EA82FB82C55BD04087CFCB54F2
:108B5000DF4F688179818A819B81C55BD0400F940A
:108B6000FE236B017C01C501B40124E630E040E046
:108B700050E00F949822CA01B9016C0D7D1D8E1D25
:108B80009F1D411451046104710481F06B017C014B
:108B9000F7FE03C0C12CD12C7601C701B6014616E1
:108BA00057066806790614F4C301B2010F94332105
:108BB000CB54DF4F688379838A839B83C55BD04026
:108BC0004DCFCB54DF4F88819981AA81BB81C55B92
:108BD000D040880E991EAA1EBB1E41145104610488
:108BE0007104C9F0A4E6B0E0A30192010F94B7228A
:108BF000362F272FB501A40177FF03C040E050E0D6
:108C0000BA01832E922E5C01481559056A057B0531
:108C100014F44A015B01CB54DF4F88829982AA8207
:108C2000BB82C55BD0401ACF88E0FE013196DE01E1
:108C3000AF54BF4F01900D928A95E1F7912C812C92
:108C4000FF24F3940FCFCE54DF4F8881C25BD04016
:108C500082958F70823009F055C0C501B40124E6B9
:108C600030E040E050E00F949822C954DF4F8881F3
:108C7000C75BD040C854DF4F6881C85BD040962F97
:108C80009170280F391F2E36E1E03E072CF437FF94
:108C900005C02DE631E002C030E020E0C954DF4FCE
:108CA0002883C75BD040C854DF4F8881C85BD04061
:108CB00030FB80F9C854DF4F8883C85BD04062E046
:108CC000CE018F549F4F0E94F81A62962FAF629781
:108CD00063963FAF639764964FAF649765965FAFB7
:108CE000659766966FAF669767967FAF679768964A
:108CF0008FAF689769969FAF6997812CB2E19B2EE1
:108D0000F12C18C088E0FE013196DE01AF54BF4F50
:108D100001900D928A95E1F768E47BE08BEA9CE094
:108D20000E9431F38BEA9CE00E947BF1912C812C14
:108D3000FF24F394C554DF4F1882CB5BD04092CE12
:108D400088E0FE013196DE01AF54BF4F01900D92D5
:108D50008A95E1F76CE37BE0E1CFC254DF4F1881E5
:108D6000CE5BD040112309F46FC01296ED91FC91B7
:108D700080858F70853009F074C0CE53DF4FE88155
:108D8000F981C25CD040359709F46BC0C1010E94E3
:108D9000EC4F21E0181619060CF020E0522EC754B3
:108DA000DF4F48815981C95BD040C154DF4F2881D2
:108DB000CF5BD040BE016F547F4FD10112968D9191
:108DC0009C910E94254FC454DF4FE881F981CC5B10
:108DD000D040319709F045C0CE54DF4F8881C25B47
:108DE000D040807FF1F1C154DF4FC880CF5BD040CD
:108DF000E52CC755DF4F0881C95AD040C655DF4F13
:108E00001881CA5AD040C555DF4F2881CB5AD0406F
:108E1000C455DF4F3881CC5AD040C355DF4F48810D
:108E2000CD5AD040C255DF4F5881CE5AD040C1559F
:108E3000DF4F6881CF5AD040C055DF4F7881C05B8B
:108E4000D040C1010E94CB33CF54DF4F8881C15B3A
:108E5000D040853009F445C150F48330B9F1D12CAC
:108E6000C3C0C254DF4F1882CE5BD040EDCF8630F6
:108E700009F482C0873099F7C1010E94E035182FAC
:108E8000863009F066C064EE7AE082E59DE00E94DB
:108E900031F34AE050E066E070E082E59DE00E9438
:108EA00082F282E59DE00E947BF162E0CE018F5468
:108EB0009F4F0E941F1B29AF3AAF4BAF5CAF6DAF06
:108EC0007EAF8FAF21969FAF21973FC0C1010E9417
:108ED000E035853021F093E0A92EB12C08C26BEF6C
:108EE0007AE082E59DE00E9431F34AE050E065E0DF
:108EF00070E082E59DE00E9482F282E59DE00E94A2
:108F00007BF1B101CE018F549F4F0E942FC761E0CA
:108F1000CE018F549F4F0E941F1B22962FAF229786
:108F200023963FAF239724964FAF249725965FAFA4
:108F3000259726966FAF269727967FAF2797289677
:108F40008FAF289729969FAF2997689480F890F85B
:108F500086CF66EC7AE082E59DE00E9431F3612FD6
:108F600070E04AE050E082E59DE00E9482F282E5F6
:108F70009DE00E947BF1AFCF40E050E061E070E007
:108F8000C1010E949230672B682B692B09F0A6C0A3
:108F9000FFEF5F120EC0C1010E94EC4F512C18165A
:108FA00019064CF46CEA7AE082E59DE00E9431F308
:108FB00092CF5110F7CFB101CE018F549F4F0E9435
:108FC0002FC761E0CE018F549F4F0E941F1B29AB1A
:108FD0003AAB4BAB5CAB6DAB7EAB8FAB98AF6894F1
:108FE00080F890F8E6E0DE2E84010160CE54DF4F79
:108FF0008881C25BD040982F9F70923050F4CF543C
:10900000DF4F9881C15BD040992319F08401016042
:109010001160807F09F489C01260C254DF4F28813B
:10902000CE5BD04021111D7FA801B101CE018F542C
:109030009F4F0E942E354801AA24A394B12CF11011
:10904000FFC6D10119968D919C91009709F0A7C395
:1090500040E050E062E070E0C1010E949230672B76
:10906000682B692B09F4CDC368E679E08BEA9CE0B4
:109070000E9431F38BEA9CE00E947BF192FC0CC6CB
:1090800066E579E082E59DE00E9431F34AE050E038
:10909000B50182E59DE00E9482F26FE479E082E50D
:1090A0009DE00E9431F30E949DD1AB01BC01CC53E5
:1090B000DF4F088119812A813B81C45CD040401B6D
:1090C000510B620B730B2AE030E082E59DE00E94B9
:1090D00096F182E59DE00E947BF109C167E97AE0A3
:1090E00063CF0FEF50120BC0C1010E94EC4F55240B
:1090F0005394181619062CF06AE77AE055CF5520DC
:10910000D9F362E0CE018F549F4F0E941F1B29A705
:109110003AA74BA75CA76DA77EA78FA798AB6894CB
:1091200080F890F875E0D72E5FCF40E052E0B101B3
:10913000CE018F549F4F0E94ED3581116DCF6DCFC1
:109140003FEF53129DC0C1010E94EC4F5524539430
:10915000181619060CF497C0512C6CE67AE082E5DB
:109160009DE00E9431F3052D052C000C110BC0541D
:10917000DF4F19830883C05CD0404AE050E0B8015B
:1091800082E59DE00E9482F265E67AE082E59DE05C
:109190000E9431F3C554DF4F1881CB5BD040612F63
:1091A00070E04AE050E082E59DE00E9482F282E5B4
:1091B0009DE00E947BF1C754DF4F08811981C95B94
:1091C000D0400115110509F4B7C06FED7DE0C8016D
:1091D0000F94371BCC24C394D12C892B09F45DC088
:1091E00068EE7DE0C8010F94371B42E0C42ED12CFD
:1091F000892B09F452C063E07EE0C8010F94371B4D
:1092000035E0C32ED12C892B09F447C06CE07EE0F9
:10921000C8010F94371B26E0C22ED12C892BE9F10F
:1092200061E87EE0C8010F94371B892B99F16AE849
:109230007EE0C8010F94371B892B09F473C064E5E5
:109240007EE0C8010F94371BBEE0CB2ED12C892BBA
:1092500021F16DE57EE0C8010F94371BAFE0CA2E07
:10926000D12C892BD1F063E97EE0C8010F94371B24
:10927000D12CC12C892B89F4F5E1CF2ED12C0DC036
:10928000552009F46ACF81E0C554DF4F8883CB5B5A
:10929000D04063CF93E1C92ED12CC1010E94E035AB
:1092A000682E712C6114710431F4C054DF4F688052
:1092B0007980C05CD040C114D10409F486C06C141C
:1092C0007D04A1F169E47AE082E59DE00E9431F33A
:1092D0004AE050E0B30182E59DE00E9482F282E51F
:1092E0009DE00E947BF1EDEFAE2EBB24BA94C50148
:1092F000C953DF4F0FB6F894DEBF0FBECDBFDF916D
:10930000CF911F910F91FF90EF90DF90CF90BF9082
:10931000AF909F908F907F906F905F904F903F9015
:109320002F90089584E1C82ED12CB7CFC754DF4FBA
:1093300019821882C95BD040C454DF4FE881F9819B
:10934000CC5BD0403197A9F4C254DF4FF881CE5B9B
:10935000D040FF2399F0CE54DF4F8881C25BD040CC
:10936000807F01E0C254DF4F0883CE5BD040811183
:1093700005C0C254DF4F1882CE5BD040CF54DF4FC0
:10938000D880C15BD04015E11D1508F4E7C1ED2D73
:10939000F0E08827E153F64B8F4F0D94ED22284AD9
:1093A000604B464B674A284A274BED4AB24A284A47
:1093B000284A9A4BA44BC24BC24B7A4B7A4BAE4BCA
:1093C000AE4BAE4B7A4B7A4B7A4BD10119968D91BD
:1093D0009C91009709F4B0CFDC01ED91FC910488D9
:1093E000F589E02DC154DF4FA880CF5BD040C55434
:1093F000DF4FC880CB5BD0407801CF54DF4F08816E
:10940000C15BD040CE54DF4F1881C25BD040CD54F9
:10941000DF4F2881C35BD040CC54DF4F3881C45B21
:10942000D040CB54DF4F4881C55BD040CA54DF4F9A
:109430005881C65BD040C954DF4F6881C75BD040BC
:10944000C854DF4F7881C85BD04019950C94A54073
:10945000D12CC254DF4F8881CE5BD040882309F4E1
:10946000EECDC154DF4FC880CF5BD040952D9170B9
:10947000E92EC755DF4F0881C95AD040C655DF4F86
:109480001881CA5AD040C555DF4F2881CB5AD040E9
:10949000C455DF4F3881CC5AD040C355DF4F488187
:1094A000CD5AD040C255DF4F5881CE5AD040C15519
:1094B000DF4F6881CF5AD040C055DF4F7881C05B05
:1094C000D040C1010E94CB33E89491F8B8CDC101DE
:1094D0000E94E035853009F0FECC64E37AE082E555
:1094E0009DE00E9431F34AE050E065E070E082E5E3
:1094F0009DE00E9482F282E59DE00E947BF1B10135
:10950000CE018F549F4F0E942FC7D10118968C9186
:109510008530C9F46EE0CE018F549F4F0E941F1B0F
:1095200029A33AA34BA35CA36DA37EA38FA398A703
:10953000689480F890F8D12CB1E0C554DF4FB8831F
:10954000CB5BD04086CF61E0CE018F549F4F0E940D
:109550001F1B298F3A8F4B8F5C8F6D8F7E8F8F8F64
:1095600098A3E6CFC1010E94E035182F863091F50F
:109570006DE17AE082E59DE00E9431F34AE050E03F
:1095800066E070E082E59DE00E9482F282E59DE067
:109590000E947BF162E0CE018F549F4F0E941F1BFF
:1095A000298B3A8B4B8B5C8B6D8B7E8B8F8B988F43
:1095B00040E050E068E070E0C1010E9440306894F3
:1095C00080F890F8D12CE1E0C554DF4FE883CB5B05
:1095D000D0403FCF6FEF79E0BECC40E050E061E09B
:1095E00070E0C1010E949230672B682B692B61F5F6
:1095F000511027C0B101CE018F549F4F0E942FC739
:1096000061E0CE018F549F4F0E941F1B29873A872C
:109610004B875C876D877E878F87988B40E050E013
:1096200068E070E0C1010E946930689480F890F8A9
:1096300076E0D72EF1E0C554DF4FF883CB5BD04006
:1096400008CF65EE79E0B0CC60ED79E0ADCC552087
:10965000D1F062E0CE018F549F4F0E941F1B2983DF
:109660003A834B835C836D837E838F839887689472
:1096700080F890F865E0D62E01E0C554DF4F0883EE
:10968000CB5BD040E6CE63EB79E08ECCCE54DF4F9F
:109690008881C25BD0408F70D12C823068F7C101C5
:1096A0000E94E035689480F890F8853009F413CC76
:1096B000D12C11E0C554DF4F1883CB5BD040C9CE0D
:1096C000CE54DF4F8881C25BD0408F70823080F7EC
:1096D000552081F06AE979E082E59DE00E9431F34E
:1096E00061E0C1010E94FD3460E071E1C1010E94AE
:1096F0007536F1CBCE54DF4F8881C25BD040982FB6
:109700009F70923008F043C0DD2069F0807F31F413
:10971000B101CE018F549F4F0E942FC7689480F8EB
:1097200023E0922AD12C31E0C554DF4F3883CB5B44
:10973000D0408FCE689492F8D12C81E0C554DF4F91
:109740008883CB5BD04085CE689492F8D12C91E091
:10975000C554DF4F9883CB5BD0407BCECE54DF4FD8
:109760008881C25BD040807F51F4689490F8D12CFE
:10977000A1E0C554DF4FA883CB5BD0406ACEB3E0F5
:109780009B2A20CFD12C812C54E0952E53CFD12C65
:1097900021E0C554DF4F2883CB5BD0405ACEDC019B
:1097A000ED91FC91008CF18DE02DCF54DF4F0881BD
:1097B000C15BD040CE54DF4F1881C25BD040CD5446
:1097C000DF4F2881C35BD040CC54DF4F3881C45B6E
:1097D000D040CB54DF4F4881C55BD040CA54DF4FE7
:1097E0005881C65BD040C954DF4F6881C75BD04009
:1097F000C854DF4F7881C85BD0401995811128CCBF
:1098000033CCF10181859285892B09F473C08114D1
:10981000910439F0A401B101CE018F549F4F0E94F1
:109820002E35D10119968D919C91C754DF4FE88058
:10983000F980C95BD040DC01ED91FC910488F58989
:10984000E02DC154DF4FA880CF5BD040C554DF4F1F
:10985000C880CB5BD040CF54DF4F0881C15BD04084
:10986000CE54DF4F1881C25BD040CD54DF4F2881EA
:10987000C35BD040CC54DF4F3881C45BD040CB5465
:10988000DF4F4881C55BD040CA54DF4F5881C65B6B
:10989000D040C954DF4F6881C75BD040C854DF4F08
:1098A0007881C85BD04019955C01F1018185928572
:1098B000DC01ED91FC91048CF58DE02D1995059757
:1098C00011F4689480F892FC2CC1DD2021F06D2DFC
:1098D000C1010E94FD34CE53DF4F08811981C25C63
:1098E000D040B4010530110509F4CACBC1010E9472
:1098F0007536C6CB8085863009F477C008F584308C
:1099000009F417C1853009F78114910439F0A401D5
:10991000B101CE018F549F4F0E942E35C454DF4FAA
:1099200008811981CC5BD0400230110509F4FDC0DB
:109930000330110509F4D2C00130110531F6CAC057
:10994000883009F45AC1893009F0BFCF81149104DD
:1099500039F0A401B101CE018F549F4F0E942E35E2
:10996000C554DF4FE881CB5BD040EE2309F4ADCF87
:10997000552079F0CF54DF4F8881C15BD0408130D2
:1099800041F4CE54DF4F8881C25BD040807F09F420
:109990009CCFCF54DF4F0881C15BD040CE54DF4F06
:1099A0001881C25BD040CD54DF4F2881C35BD040CB
:1099B000CC54DF4F3881C45BD040CB54DF4F48815B
:1099C000C55BD040CA54DF4F5881C65BD040C954F4
:1099D000DF4F6881C75BD040C854DF4F7881C85BD8
:1099E000D040C1010E94723EF2C0CF54DF4FF880D8
:1099F000C15BD040FF2009F487CF70E060E0C10177
:109A00000E94542E8C018114910439F0A401B101FB
:109A1000CE018F549F4F0E942E350115110509F478
:109A200054CF712C612C17FF06C0119501951109B7
:109A300066246394712CC80101978634910508F05F
:109A400044CFE02E61E0802F0E9422CFEFEFEF0D98
:109A5000E53110F5F0E08827EF5CF24B8F4F0D9465
:109A6000ED22464D484D4C4D4C4D484D464D484DD0
:109A70004C4D4C4D4C4D4C4D4C4D4C4D464D464D2A
:109A80004C4D4C4D4C4D4C4D464D464DF1E06F26E6
:109A9000662D8E2D0E94F4CE63E679E082E59DE08E
:109AA0000E9431F34AE050E0B80182E59DE00E9457
:109AB00082F261E679E082E59DE00E9431F34AE0BE
:109AC00050E0B30182E59DE00E9482F282E59DE0D4
:109AD0000E947BF1689480F890F823C0C1010E9435
:109AE000F22D892B49F4D101ED91FC9160817181B6
:109AF00082E995E00E9486D2CE018F549F4F0E944A
:109B0000FF1E20E030E048EC52E40F9492210F94C5
:109B1000FE232B0188E00F94EF0DA201C1010E94EA
:109B2000B12DAA24A394B12CD0CE689480F891F8DA
:109B3000F8CF8114910439F0A401B101CE018F5402
:109B40009F4F0E942E35C554DF4FB881CB5BD0406C
:109B5000BB2309F4BACECF54DF4F8881C15BD0401C
:109B60005520B9F1813041F4CE54DF4F8881C25B7A
:109B7000D040807F09F4A9CECF54DF4F0881C15B6C
:109B8000D040CE54DF4F1881C25BD040CD54DF4F60
:109B90002881C35BD040CC54DF4F3881C45BD040B8
:109BA000CB54DF4F4881C55BD040CA54DF4F58814A
:109BB000C65BD040C954DF4F6881C75BD040C854F2
:109BC000DF4F7881C85BD040C1010E94A23C5C019C
:109BD0007CCE813089F6CE018F549F4F0E94AEC15A
:109BE000449750F66EE170E0CE018F549F4F0E9473
:109BF000AB1E689480F891F8BFCF8114910439F0BE
:109C0000A401B101CE018F549F4F0E942E35C5543F
:109C1000DF4FF881CB5BD040FF2309F456CE5520AF
:109C200079F0CF54DF4F8881C15BD040813041F45F
:109C3000CE54DF4F8881C25BD040807F09F445CE8F
:109C4000CF54DF4F0881C15BD040CE54DF4F188125
:109C5000C25BD040CD54DF4F2881C35BD040CC5491
:109C6000DF4F3881C45BD040CB54DF4F4881C55BA8
:109C7000D040CA54DF4F5881C65BD040C954DF4F33
:109C80006881C75BD040C854DF4F7881C85BD04043
:109C9000C1010E945B3D9BCFCE53DF4F28813981AC
:109CA000C25CD0402530310509F4EAC940E054E0F7
:109CB000B101CE018F549F4F0E942E3560E074E0B9
:109CC00015CE0E94461F672B682B692B11F00C9450
:109CD000F541912C812C11E0C554DF4F1883CB5BEB
:109CE000D0400C942C42C454DF4F28813981CC5B86
:109CF000D040232B09F053C08081882311F40C94A9
:109D00001B40CE0187549F4F0E942C2DC454DF4F1F
:109D100099838883CC5BD040CE54DF4F8881C25B6F
:109D2000D0408F7091F5C454DF4F6881CC5BD04038
:109D3000CE018F549F4F0E94F81ACF55DF4F2883D2
:109D4000C15AD040CE55DF4F3883C25AD040CD558E
:109D5000DF4F4883C35AD040CC55DF4F5883C45A95
:109D6000D040CB55DF4F6883C55AD040CA55DF4F2E
:109D70007883C65AD040C955DF4F8883C75AD04030
:109D8000C855DF4F9883C85AD040C454DF4FE8818C
:109D9000F981CC5BD040EF2B11F40C941B406CE8A4
:109DA0007BE082E59DE00E9431F34AE050E0B6019D
:109DB00082E59DE00E9482F265E87BE082E59DE01D
:109DC0000E9431F3D101ED91FC916081718182E5B6
:109DD0009DE00E94CBF26FE77BE082E59DE00E9470
:109DE00031F3C754DF4F68817981C95BD04082E588
:109DF0009DE00E94CBF26DE77BE082E59DE00E9452
:109E000031F3CE018F549F4F0E94CD22C754DF4FB4
:109E100088819981C95BD040009711F40C94674008
:109E2000FC012081243211F00C94674069E67BE04C
:109E300082E59DE00E9431F382E59DE00E947BF186
:109E40008CEFA82EBB24BA9452CA2F923F924F9205
:109E50005F926F927F928F929F92AF92CF92DF929A
:109E6000EF92FF920F931F93CF93DF93CDB7DEB79F
:109E70006D970FB6F894DEBF0FBECDBF009709F403
:109E8000A9C0FC0130853F70353009F0A3C0D22E47
:109E90001A014B016680778080917D0E8F5F8093E1
:109EA0007D0E6114710409F490C0F30180858F70F8
:109EB000843009F086C0618572858091830E90910F
:109EC000840E0E9427C12C01009709F47AC0FC017E
:109ED00080858F70853009F074C0B201CE01019683
:109EE0000E94C23A81149104B1F0CE0101960E9401
:109EF000622D882381F0AD2CC12C7101F401008109
:109F00001181228133814481558166817781CE011F
:109F100001960E94563F60E0C2010E949FC10097D7
:109F2000E9F1FC0120852F702230C1F581859285F1
:109F3000A385B4850797A105B10581F561E0C2014C
:109F40000E949FC12D2DA101B4010E94254F8114B3
:109F5000910499F5882389F180917D0E8150809339
:109F60007D0ECE0101960E94643981E06D960FB698
:109F7000F894DEBF0FBECDBFDF91CF911F910F913F
:109F8000FF90EF90DF90CF90AF909F908F907F9059
:109F90006F905F904F903F902F900895811491049F
:109FA00061F4CE0101960E94622D882331F0CE012A
:109FB00001960E94EC4F892B79F6CE0101960E9402
:109FC0006439F301628073806CCF80917D0E815083
:109FD00080937D0E80E0CACFDF92EF92FF920F93C5
:109FE0001F93CF93DF9300D000D01F921F92CDB765
:109FF000DEB77C0119821A821B821C821D821E829E
:10A000001F8218868A818F708A83D701ED91FC9117
:10A010006081718182E59DE00E94CBF268ED7BE07A
:10A0200082E59DE00E9431F3C7010E94622D8111FB
:10A030001BC06FEC7BE082E59DE00E9431F382E57E
:10A040009DE00E947BF10FEF1FEFC80128960FB62D
:10A05000F894DEBF0FBECDBFDF91CF911F910F915E
:10A06000FF90EF90DF900895C7010E94E035D82E51
:10A07000F70181859285009791F0DC01ED91FC91CB
:10A080000688F789E02D19958C0197FD08C081E0BD
:10A090000115110509F480E00E942C17D6CFF701B5
:10A0A0008085873009F42EC0EFEFED0DE43150F5D7
:10A0B000F0E08827E15AFF4A8F4F0D94ED2273504C
:10A0C0007C50825082507C5073508250825082501B
:10A0D00082508250825082507350825082508250FF
:10A0E00082507350735060EB7BE082E59DE00E94EC
:10A0F00031F301E010E0A9CF80E00E942C1710E0BE
:10A1000000E0A3CF40E052E0B701CE0101960E94EB
:10A11000ED35D70118968C911897873089F160F446
:10A12000833009F457C0843061F060EC7BE082E555
:10A130009DE00E9431F3E3CF883009F44BC08930B1
:10A14000A1F760E0CE0101960E94DE1D8C0165EB57
:10A150007BE082E59DE00E9431F34AE050E0B801E7
:10A1600082E59DE00E9482F282E59DE00E947BF103
:10A1700091E080E0012B09F490E0092F182F65CFC2
:10A180001296ED91FC9180858F7010E000E0853093
:10A19000F1F66DEC7BE082E59DE00E9431F320E07A
:10A1A00050E040E070E060E0F701828193810E941E
:10A1B000254FF82E082F10E06AEC7BE082E59DE049
:10A1C0000E9431F38F2D0E942C1782E59DE00E94A2
:10A1D0007BF13BCFCE0101960E94461F8B01B7CF8A
:10A1E000AF92CF92EF92FF920F931F93CF93DF9393
:10A1F00000D000D01F921F92CDB7DEB719821A820D
:10A200001B821C821D821E821F8218861A811F706B
:10A21000A12CCC24C394F12CE12C02E02B813C81B5
:10A2200040E05E816F8178850E94563F28960FB688
:10A23000F894DEBF0FBECDBFDF91CF911F910F917C
:10A24000FF90EF90CF90AF9008952F923F924F9252
:10A250005F926F927F928F929F92AF92BF92CF92B6
:10A26000DF92EF92FF920F931F93CF93DF93CDB7BF
:10A27000DEB7C255D1090FB6F894DEBF0FBECDBF11
:10A280004C013B0140E058E060E070E00E949230F9
:10A29000672B682B692B09F45CC019821A821B8218
:10A2A0001C821D821E821F8218868A818F708A837B
:10A2B00040E053E0B401CE0101960E94ED35D40197
:10A2C00019968D919C91892B09F4FBC040E058E0D0
:10A2D00060E070E0C4010E94403065E27CE082E50D
:10A2E0009DE00E9431F3F40181859285DC01ED91BE
:10A2F000FC910488F589E02DA12CCC24C394F12C89
:10A30000E12C09811A812B813C814D815E816F8115
:10A3100078851995D401ED91FC918F3F9807C9F08C
:10A3200060817181892B09F036C182E59DE00E9430
:10A33000CBF268EE7BE082E59DE00E9431F360EEB7
:10A340007BE082E59DE00E9431F382E59DE00E9482
:10A350007BF165E0F401808191810E949FC15C01E5
:10A36000009709F450C1DC011896BC916196BFAF0B
:10A370006197B295BF706096BFAF6097FC01218472
:10A380003284438454840E949DD16096FFAD6097CF
:10A39000FF2309F438C1261A370A480A590A19A2B4
:10A3A0001AA21BA21CA2F9A31AA11F70106A1AA359
:10A3B0002DA23EA24FA258A624E06216710449F5D0
:10A3C000D12CC12CE12C50E2F52E0F2F2BA13CA15A
:10A3D0004DA15EA16FA178A5C4010E94B630C20153
:10A3E000B10128EE33E040E050E00F949822BA012A
:10A3F000A9012AE030E082E59DE00E943AF265E39F
:10A400007DE082E59DE00E9431F382E59DE00E94BF
:10A410007BF157FEF8C082E028163104410480E841
:10A4200058060CF4F0C00F94560F1B0163967FAFD3
:10A430006EAF6397D12CC12CE12C40E2F42E09A120
:10A440001AA12BA13CA14DA15EA16FA178A5C401C9
:10A450000E94B6306396AEADBFAD6397A83CB10520
:10A460000CF0A6C06CE17DE08BEA9CE00E9431F329
:10A470004AE050E0B1018BEA9CE00E9482F28BEA54
:10A480009CE00E947BF166246A94762CC301CE5A2C
:10A49000DF4F0FB6F894DEBF0FBECDBFDF91CF9177
:10A4A0001F910F91FF90EF90DF90CF90BF90AF90F2
:10A4B0009F908F907F906F905F904F903F902F90E4
:10A4C0000895F4018085883009F445C0893019F178
:10A4D000843009F03ECF8091230990912409892B83
:10A4E00009F037CF40E058E060E070E0C4010E941E
:10A4F000403060E17CE082E59DE00E9431F309811B
:10A500001A812B813C814D815E816F817885C401E8
:10A510000E94A23CFFCE8091230990912409892BAF
:10A5200009F017CF40E058E060E070E0C4010E94FD
:10A5300040306FEF7BE082E59DE00E9431F30981BE
:10A540001A812B813C814D815E816F817885C401A8
:10A550000E94723EDFCE8091230990912409892BBD
:10A5600009F0F7CE40E058E060E070E0C4010E94DE
:10A5700040306AEE7BE082E59DE00E9431F3098184
:10A580001A812B813C814D815E816F817885C40168
:10A590000E945B3DBFCE82E59DE00E94CBF26EED56
:10A5A0007BE082E59DE00E9431F36AED7BE0C9CE5D
:10A5B000F50180858F70808719821A821B821C8228
:10A5C0001D821E821F8218868A818F708A83609600
:10A5D000FFAD6097F98361968FAD61978F70AA2464
:10A5E000A394873009F0A12CCC24C394F12CE12C46
:10A5F00009811A812B813C814D815E816F81788533
:10A60000C4010E94563F21E06216710459F4D4013E
:10A6100018968C91843079F0893009F470C1C401A6
:10A620000E94E736F40181859285009709F0A0C465
:10A63000712C612C2BCF8091230990912409892BB7
:10A64000B9F4F40142805380D20118968C918F7036
:10A65000853041F4C2010E9431C2082F10E002305F
:10A66000110554F464E87CE082E59DE00E9431F33A
:10A67000C4010E94E7360ACF709224096092230930
:10A6800070E060E0C4010E94542E1C0161E070E0A3
:10A69000C4010E94542E5C01053011050CF440C029
:10A6A00064E0C2010E949FC1FC010185128526E081
:10A6B00040E855E260E070E086E09AE00E943DF4F8
:10A6C0002092F60A86E09AE09093F50A8093F40AC5
:10A6D0001092010C1092030C1092020C60E77CE0C7
:10A6E00082E59DE00E9431F3D401ED91FC916081FF
:10A6F000718182E59DE00E94CBF282E59DE00E949F
:10A700007BF10130110509F4C2C06CF4012B09F48E
:10A71000B3C064E57CE082E59DE00E9431F325C092
:10A7200002E010E0C4CF0230110579F003301105CA
:10A7300081F7B092F80AA092F70A81E090E0909336
:10A74000FA0A8093F90A84E00BC0B092F80AA0924A
:10A75000F70A81E090E09093FA0A8093F90A83E087
:10A760000E94F4D22F968FAF2F972F96BFAD2F97C1
:10A77000B11197C00091FB0A1091FC0A6FE47CE0D4
:10A7800082E59DE00E9431F3D401ED91FC9160815E
:10A79000718182E59DE00E94CBF268E47CE082E575
:10A7A0009DE00E9431F3C801012E000CAA0BBB0BE7
:10A7B00089839A83AB83BC8380E190E09E838D8301
:10A7C000BE016F5F7F4F82E59DE00E94D83A0E94F4
:10A7D0007BF1B801C4010E94C937E0911C09F091D6
:10A7E0001D0962817381CE0101960E94C23A809157
:10A7F0001C0990911D09892BB1F1CE0101960E948F
:10A80000622D882381F18985843069F570E060E0EC
:10A81000CE0101960E94542E2816390621F561E0DA
:10A8200070E0CE0101960E94542EA816B906D9F404
:10A83000B801CE0101960E94C937E0911C09F09140
:10A840001D098281938190931D0980931C09892B96
:10A8500051F4E091830EF091840E8681978190935C
:10A860001D0980931C09CE0101960E946439109243
:10A87000240910922309FCCEB092F80AA092F70A9C
:10A8800081E090E09093FA0A8093F90A69CFB09240
:10A89000F80AA092F70A1093FA0A0093F90A82E0E4
:10A8A0005FCF6BE37CE082E59DE00E9431F3D40151
:10A8B000ED91FC916081718182E59DE00E94CBF277
:10A8C00063E37CE082E59DE00E9431F32F96EFADDB
:10A8D0002F978E2F90E0B0E0A0E089839A83AB831E
:10A8E000BC8380E190E09E838D83BE016F5F7F4FCC
:10A8F00082E59DE00E94D83A0E947BF1B8CF80911A
:10A90000230990912409892B09F0B2CE7092240971
:10A91000609223090E942AF92C01009741F0DC0182
:10A9200018968C911897807F866018968C93F20108
:10A9300080858F70808730E020E043E050E060E267
:10A94000CE0101960F940D0ED401ED91FC91608122
:10A9500071814FE150E0CE0101960F946A2761EAC0
:10A9600075E0CE0101960F94442726E040E855E2B9
:10A9700060E070E086E09AE00E943DF470E060E004
:10A98000C4010E94542E8093F60A86E09AE09093C8
:10A99000F50A8093F40A1092010C1092030C1092A5
:10A9A000020C6CE07DE082E59DE00E9431F3D40171
:10A9B000ED91FC916081718182E59DE00E94CBF276
:10A9C00082E59DE00E947BF162E370E080E090E030
:10A9D0000E946AD184E398E09093F80A8093F70A82
:10A9E0008AE090E09093FA0A8093F90A83E00E944B
:10A9F000F4D2182F811154C26FEF7CE082E59DE004
:10AA00000E9431F30BEF1AE09FE0292E9BE0392ED4
:10AA100020E1A22EB12CF801819191918F01092E94
:10AA2000000CAA0BBB0B89A39AA3ABA3BCA3BEA229
:10AA3000ADA2BE016F5D7F4F82E59DE00E94D83AD6
:10AA40006DEF7CE00E9431F32016310621F782E59C
:10AA50009DE00E947BF16091FF0A7091000B90E0F5
:10AA600080E00F94332120E030E048EC52E40F9472
:10AA70008C239B01AC0165EA76E0C2010E941DCBEC
:10AA8000C090030BD090040BF12CE12CA701960190
:10AA900067EA75E0C2010E94C6C76091050B70911C
:10AAA000060B90E080E00F94332120E030E048EC8A
:10AAB00052E40F948C239B01AC016BEA75E0C20158
:10AAC0000E941DCB6091070B7091080B90E080E015
:10AAD0000F94332120E030E040E251E40F948C23C6
:10AAE0009B01AC0169EA75E0C2010E941DCB209177
:10AAF000FB0A3091FC0A50E040E06DEA75E0C201CB
:10AB00000E94C6C7CD28CE28CF2809F47AC0D40128
:10AB10001296ED91FC9190859F70953009F071C06F
:10AB200061E0CF010E949FC1009709F46AC0FC0157
:10AB300020852F70243009F064C061857285CE01B4
:10AB400081960E94D838CE0181960E94622D88237A
:10AB500009F453C022961CAE1DAE1EAE1FAE229746
:10AB600026961CAE1DAE1EAE1FAE26978FAD8F7003
:10AB700080618FAF8FEF23968FAF239724965FADC1
:10AB8000249725963FAD259726962FAD26979EAD07
:10AB90007FAD21966FAD219722964FAD2297092F59
:10ABA00027969FAF279728967FAF289729966FAF54
:10ABB00029972A964FAF2A97482F2B968FAF2B971E
:10ABC0002C965FAF2C972D963FAF2D972E962FAFDB
:10ABD0002E97A12CCC24C394F12CE12C172F262FD7
:10ABE0002A963FAD2A972D966FAD2D972E967FAD65
:10ABF0002E97CE0181960E94563FCE0181960E94EB
:10AC000064398091FB0A83FF76C162ED7CE082E5C6
:10AC10009DE00E9431F3D401ED91FC91608171813E
:10AC200082E59DE00E94CBF282E59DE00E947BF1EF
:10AC300062E370E080E090E00E946AD18EE398E0E9
:10AC40009093F80A8093F70A81E090E09093FA0AD3
:10AC50008093F90A83E00E94F4D281110BC0209105
:10AC6000FB0A3091FC0A50E040E060EB75E0C20165
:10AC70000E94C6C71092240910922309C4010E94A1
:10AC8000EC4F181619061CF4C4010E94F05081E024
:10AC900090E0909324098093230962EC7CE082E5A4
:10ACA0009DE00E9431F3D401ED91FC9160817181AE
:10ACB00082E59DE00E94CBF282E59DE00E947BF15F
:10ACC00062E370E080E090E00E946AD183E190E06E
:10ACD0009093F80A8093F70A84E090E09093FA0A40
:10ACE0008093F90A83E00E94F4D2182F811115C1D4
:10ACF00065EB7CE082E59DE00E9431F30BEF1AE00A
:10AD000083E0E82E8BE0F82EF801619171918F01BC
:10AD10004AE050E082E59DE00E9482F263EB7CE035
:10AD200082E59DE00E9431F3E016F10669F782E5C5
:10AD30009DE00E947BF10091FB0A1091FC0A011535
:10AD40001105D1F0B801012E000C880B990B0F945E
:10AD500033212DEE3EE94CE35EE30F94922122E590
:10AD600038EB42E152E40F941F239B01AC0164EBEA
:10AD700075E0C2010E941DCB6091FD0A7091FE0A30
:10AD8000072E000C880B990B0F9433212DEE3EE912
:10AD90004CE35EE30F94922122E538EB42E152E46A
:10ADA0000F941F236B017C01AC019B0165EA75E0E8
:10ADB000C2010E941DCB6091010B7091020B16160F
:10ADC00017060CF0A1C0072E000C880B990B0F94EE
:10ADD000332120E030E040E251E40F948C239B01CA
:10ADE000AC0168EB75E0C2010E941DCB20E030E0B1
:10ADF00040E252E4C701B6010F9434241816B4F4AB
:10AE0000012BA1F00E9445C1882369F08091680E52
:10AE1000811109C0D401ED91FC91608171818CEBAD
:10AE200095E00E9486D2C4010E94F05080E091E03B
:10AE30000F94FE188C01892BD9F01CA21BA21EA214
:10AE40001DA28FEF9FEF98A78FA385EA92E09AA3A8
:10AE500089A31AA619A61CA70BA780E091E098ABBE
:10AE60008FA71EA61DA6B201CE0181960E941AF7D9
:10AE70000E9445C1882349F08091680E811105C068
:10AE8000B801CE0101960E9486D2C8010F949A198A
:10AE90004114510409F4EBCCC2010E94F1CAE7CC81
:10AEA00060EF7CE082E59DE00E9431F3D401ED91FA
:10AEB000FC916081718182E59DE00E94CBF268EE99
:10AEC0007CE082E59DE00E9431F3812F90E0B0E0CC
:10AED000A0E089A39AA3ABA3BCA380E190E09EA3CA
:10AEE0008DA3BE016F5D7F4F82E59DE00E94D83A41
:10AEF0000E947BF186CE20E030E0A90160EB75E096
:10AF0000C2010E94C6C7C9CE20E030E0A90168EBAB
:10AF100075E0C2010E94C6C769CF63EA7CE082E5A2
:10AF20009DE00E9431F3D401ED91FC91608171812B
:10AF300082E59DE00E94CBF26BE97CE082E59DE03A
:10AF40000E9431F3812F90E0B0E0A0E089A39AA3A2
:10AF5000ABA3BCA380E190E09EA38DA3BE016F5D77
:10AF60007F4F82E59DE00E94D83A0E947BF15ECF40
:10AF7000DC01ED91FC910284F385E02D1995892B7C
:10AF800009F456CBF40181859285DC01ED91FC91A9
:10AF90000480F581E02DB30119953C0177CA2F9209
:10AFA0003F924F925F926F927F928F929F92AF9259
:10AFB000BF92CF92DF92EF92FF920F931F93CF93A6
:10AFC000DF93CDB7DEB7C657D1090FB6F894DEBF11
:10AFD0000FBECDBFDC0114962D913C91232B11F4B3
:10AFE0000C94E3613B014C01FC0182819B012250E6
:10AFF00031092230310508F017C6803409F4F7C250
:10B0000008F04AC0843008F085C28091D3088F5F71
:10B010008093D308A3016FEFC4010E94411BD401A8
:10B0200012960C9112970695017013961C91139726
:10B030008AEC810F803108F043C069EC75E08D9196
:10B040009C910E9427C17C010097D1F1FC01808571
:10B050008F708530A9F58091910D181324C08091CF
:10B06000920D803401F58091930D9091940D5C01C7
:10B07000990FCC08DD0860E0C7010E949FC1FC0168
:10B0800081859285A385B485A816B906CA06DB0614
:10B090000CF065C0512C3EC0823409F4A8C208F4FB
:10B0A00039C28058AFCF1093910D80E48093920DF8
:10B0B000812F0E9435D09093940D8093930DD7CF1C
:10B0C000212F30E0F901EE5BF74D8491F901E45056
:10B0D000F84D1491F901EA54F84DF490FF2009F469
:10B0E0003BC081110E948DCEEF2DF0E0EE0FFF1FCF
:10B0F000EF50F54DA591B491EC911E2331E020E085
:10B1000009F430E0832F922F552453940817190621
:10B1100009F0C0CFF3E06F16710409F488C0D401C0
:10B120001496ED91FC91E181EF70E150EC3008F064
:10B130007EC0F0E08827E056F74A8F4F0D94ED224D
:10B14000C1583D5AF7582D593D5A46593D5A7A59DA
:10B15000A759C059025A245A90E080E0D5CF61E047
:10B16000C7010E949FC155245394FC01818592859B
:10B17000A385B4858A159B05AC05BD050CF0CACF27
:10B1800089CF0E949DD19B01AC0144275527D40152
:10B190001496ED91FC916281738190E080E0AA2485
:10B1A000AA94BA2CC12CD12C18EEE12E13E0F12E6A
:10B1B00000E010E00F94EE0C8823C9F1F401008147
:10B1C00011816FE175E0C8010E9427C1892B41F40C
:10B1D00064E275E0C8010E9427C1892B09F40EC101
:10B1E00042E050E063E0C4010E94411B20C00E9485
:10B1F0009DD19B01AC0144275527D4011496ED91B4
:10B20000FC916281738190E080E0AA24AA94BA2C18
:10B21000C12CD12C1CE2E12EFF24F39400E010E0BD
:10B220000F94EE0C42E050E064E0811184C0D40140
:10B230001496ED91FC91808183FB992790F99515E7
:10B2400009F4D2C1982F907E09F439C1982F907ECD
:10B2500090528F71892B808358C10E949DD19B0190
:10B26000AC0144275527D4011496ED91FC916281DD
:10B27000738190E080E0AA24AA94BA2CC12CD12C2E
:10B2800016E9E12EF12C00E010E0CACF0E949DD11A
:10B290009B01AC0144275527D4011496ED91FC91F4
:10B2A0006281738190E080E0AA24AA94BA2CC12C18
:10B2B000D12C18EEE12E13E0F12E00E010E00F94F7
:10B2C000EE0C882309F4B3CFF401008111816AE206
:10B2D00075E0C8010E9427C1892B41F460E375E045
:10B2E000C8010E9427C1892B09F488C042E050E0C0
:10B2F00068E079CF0E949DD19B01AC01442755277E
:10B30000D4011496ED91FC916281738190E080E00C
:10B31000AA24AA94BA2CC12CD12C1CE2E12EFF2421
:10B32000F39400E010E00F94EE0C42E050E069E08E
:10B33000882309F47CCFC4010E94411B0E949DD147
:10B34000D4011496ED91FC917383628370CF0E94B7
:10B350009DD19B01AC0144275527D4011496ED9152
:10B36000FC916281738190E080E0AA24AA94BA2CB7
:10B37000C12CD12C16E9E12EF12C00E010E0D3CF46
:10B380000E949DD19B01AC0144275527D4011496FE
:10B39000ED91FC916281738190E080E0AA24AA94EF
:10B3A000BA2CC12CD12C18EEE12E13E0F12E00E0C6
:10B3B00010E00F94EE0C882309F439CFF4010081DA
:10B3C000118167E375E0C8010E9427C1892B39F418
:10B3D0006DE375E0C8010E9427C1892B21F042E08E
:10B3E00050E06BE000CF69E175E0C8010E9427C121
:10B3F00042E050E066E0892B09F4F5CE42E050E0EF
:10B400006DE0F1CE0E949DD19B01AC0144275527F0
:10B41000D4011496ED91FC916281738190E080E0FB
:10B42000AA24AA94BA2CC12CD12C1CE2E12EFF2410
:10B43000F39400E010E00F94EE0C882309F4F7CEAB
:10B4400042E050E06CE077CF0E949DD19B01AC01BF
:10B4500044275527D4011496ED91FC9162817381A4
:10B4600090E080E0AA24AA94BA2CC12CD12C16E931
:10B47000E12EF12C00E010E0DECF0E949DD19B0177
:10B48000AC0144275527D4011496ED91FC916281BB
:10B49000738190E080E0AA24AA94BA2CC12CD12C0C
:10B4A00018E5E12E12E0F12E00E010E00F94EE0C12
:10B4B000882309F4BCCE42E050E060E094CE0E94C4
:10B4C0009DD1D4011496ED91FC91159773836283FD
:10B4D000E181EF70552009F445C0E230F1F050F4FD
:10B4E000EE23E9F1D4011496ED91FC91808150FA9C
:10B4F00083F9B1CEE53089F0A3016AE0E73091F736
:10B50000C4010E94411B8111EDCF8091D30881506D
:10B510008093D30890E080E058C7F4010081118146
:10B5200063E175E0C8010E9427C1892BA9F46AE292
:10B5300075E0C8010E9427C1892B71F460E375E0B2
:10B54000C8010E9427C1892B39F46BEF74E0C80150
:10B550000E9427C1892B19F0A30166E0D1CFA30176
:10B5600061E0CECFE150ED3008F0BCCFF0E08827AD
:10B57000E354F54A8F4F0D94ED22CA5A725ACD5AB0
:10B58000CD5A725AD05A725AF15AF15AF15AF15AA6
:10B59000F15ACD5AA30162E0B3CFA30165E0B0CF69
:10B5A0000D911C9163E175E0C8010E9427C1892BB0
:10B5B000A9F46AE275E0C8010E9427C1892B71F4E1
:10B5C00060E375E0C8010E9427C1892B39F46BEF55
:10B5D00074E0C8010E9427C1892B19F0A30167E01C
:10B5E0008FCFA30160E08CCF8F71806434CEB3E045
:10B5F0006B16710409F48ECF69EC75E0F40180815B
:10B6000091810E9427C18C01D40113968C91909155
:10B61000910D8913E5C09091920D903409F0E0C02E
:10B620008091930D9091940D3C010115110509F441
:10B6300004C1F80120852F70253009F0FEC0C80133
:10B640000E9431C2A7968FAFA797843008F4D4C068
:10B6500063E0C8010E949FC1DC0119968D919C9105
:10B660002AE0F22EF89E5001F99EB00C112462E0FF
:10B67000C8010E949FC1FC0181859285F89E10013E
:10B68000F99E300C11246101032C000CEE08FF0818
:10B69000E796CCAEDDAEEEAEFFAEE79761E0C80157
:10B6A0000E949FC12C0160E0C8010E949FC1DC0183
:10B6B0001996CD90DD90ED90FC901C97AB96CCAE9A
:10B6C000DDAEEEAEFFAEAB979301072C000C440B42
:10B6D000550B2C193D094E095F09B5010B2C000CC7
:10B6E000880B990BE796CCACDDACEEACFFACE797E2
:10B6F0006C197D098E099F090F946622D201199653
:10B700002D913D914D915C911C97AB96CCACDDACED
:10B71000EEACFFACAB972C193D094E095F09AB9617
:10B720002CAF3DAF4EAF5FAFAB970F949822E7962B
:10B73000CCACDDACEEACFFACE797C20ED31EE41E82
:10B74000F51EA7962FADA797253009F465C081E0B7
:10B7500090E0A5010B2C000C660B770B4C155D05DA
:10B760006E057F050CF461C0B701A6016101032CD1
:10B77000000CEE08FF084C155D056E057F050CF406
:10B7800059C06A017B01A796BFADA797B23009F0F7
:10B7900065C06301770CEE08FF0860E0C8010E94F5
:10B7A0009FC1FC0181859285A385B485C816D90601
:10B7B000EA06FB060CF423C661E0C8010E949FC1A3
:10B7C000FC0181859285A385B4858C159D05AE0508
:10B7D000BF050CF09FCE81E090E0A0E0B0E012C683
:10B7E0008093910D90E49093920D0E9435D09093A8
:10B7F000940D8093930D18CF8AE0869D6001879DFC
:10B80000D00C11240D2C000CEE08FF08312C212C3B
:10B81000A12C88E2B82E9BCF64E0C8010E949FC192
:10B82000DC0119968D919C9194CF66246A94B3E0C3
:10B830007B2E9CCF712C612CA6CF2AE0289F600123
:10B84000299FD00C11240D2C000CEE08FF08312C80
:10B85000212CA12CA8E2BA2E81E090E0D40114960C
:10B86000ED91FC9162817381A301461B570B57FF39
:10B8700003C0519541955109841795070CF4C0C038
:10B880008081982F929596959770963008F0BBC05E
:10B890009F5F9295990F907E8F71892BB3C0F201B3
:10B8A00061857285DB018C9181113DC60115110501
:10B8B00009F457C0D80118968C9118978F7084306E
:10B8C00009F04FC019966D917C91CE0101960E94AE
:10B8D000D838CE0101960E94622D8823F1F12114FF
:10B8E000310409F460C04114510431F0F201808543
:10B8F0008F70843009F44CC025961CAE1DAE1EAE70
:10B900001FAE259729961CAE1DAE1EAE1FAE299701
:10B9100023961FAD23971F7023961FAF239781E0B7
:10B9200022968FAF2297A12CCC24C394F12CE12C2A
:10B9300001E024962FAD249725963FAD259740E052
:10B9400027965FAD279728966FAD289729967FADEC
:10B950002997CE0101960E94563FCE0101960E9482
:10B960006439D4011496ED91FC9133822282D2CDB8
:10B970006114710429F0F30180858F70843019F00F
:10B9800067E876E0D0C561857285FB0180818CCF48
:10B9900061857285FB0180818823F9F2CE010196D1
:10B9A0000E9458C8DACF6114710431F0D30118969F
:10B9B0008C918F708430F1F025961CAE1DAE1EAEBA
:10B9C0001FAE259729961CAE1DAE1EAE1FAE299741
:10B9D00023961FAD23971F7023961FAF239782E0F6
:10B9E00022968FAF2297A12CCC24C394F12CE12C6A
:10B9F00002E09FCFF30161857285DB018C91CCCF92
:10BA000080818F7180838081803A98F0C101330CEE
:10BA1000AA0BBB0B8C159D05AE05BF0551F0C501EA
:10BA2000BB0CAA0BBB0B8C159D05AE05BF0509F021
:10BA300071CD6615770509F46DCDA2961CAE1DAECD
:10BA40001EAE1FAEA297A0968FADA0978F70806696
:10BA5000A0968FAFA097A2968CAD9DADAEADBFADB9
:10BA6000A29768968CAF9DAFAEAFBFAF6897AAE0C4
:10BA7000B0E0A70196010F94B7226C966CAF7DAF32
:10BA80008EAF9FAF6C9764E678E082E59DE00E9400
:10BA900031F34AE050E0F401638182E59DE00E94C9
:10BAA00098F162E678E082E59DE00E9431F3CE01F4
:10BAB0008C5A9F4F0E94CD226DEC75E0D4018D9180
:10BAC0009C910E9427C1B12CA12CD12CC12C659630
:10BAD000EFAC65976696FFAC669767960FAD679774
:10BAE00068961FAD689769962FAD69976A963FADC6
:10BAF0006A976B964FAD6B976C965FAD6C976FEFD7
:10BB00000F941211F4010081118164E475E0C80101
:10BB10000E9427C17C0169E475E0C8010E9427C129
:10BB20008C010097F1F1DC0118968C9118978F70B9
:10BB30008430B9F519966D917C9140E450E0CE01C6
:10BB400001960F9488276FE270E0CE0101960F9462
:10BB50004F27892B51F4F8012185328543E050E0CD
:10BB600060E4CE0101960F940D0E00E020E032E07B
:10BB700040E150E0BE016F5B7F4FCE018C5A9F4F7A
:10BB80000E94AC200E9445C1882359F08091680E24
:10BB9000811107C0BE016F5B7F4FCE0101960E94ED
:10BBA0006BD2E114F104C9F1D70118968C91189762
:10BBB0008F70843091F519966D917C91CE0101962C
:10BBC0000E94D838CE0101960E94622D882309F187
:10BBD000A12CCC24C394F12CE12C65960FAD659774
:10BBE00066961FAD669767962FAD679768963FADCF
:10BBF000689769964FAD69976A965FAD6A976B963D
:10BC00006FAD6B976C967FAD6C97CE0101960E94DD
:10BC1000563FCE0101960E946439D4011496ED91ED
:10BC2000FC917382628276CC883009F49BC28031A9
:10BC300009F488C3843009F06DCC0E949DD12B019A
:10BC40003C01C4010E943A16A12CB12C650118E9EF
:10BC5000E12E1AE3F12E00E010E0A30192010F940F
:10BC6000EE0C882309F456CCF401838127968FAF1C
:10BC7000279796E128969FAF2897282F30E0F90163
:10BC8000E450F84DE4912996EFAF2997F901EA5471
:10BC9000F84DE4912A96EFAF2A9740E85EE360E022
:10BCA00070E062964CAF5DAF6EAF7FAF629762E0BF
:10BCB0000E9422CF0E949DD1605D77408109910949
:10BCC0002E966CAF7DAF8EAF9FAF2E9787E36496B5
:10BCD0008FAF6497CE018F5B9F4F0E94F7D488236C
:10BCE00049F028968FAD28978C3009F46FC048F43E
:10BCF0008B3011F1412C512C60EC662E6FE7762EC3
:10BD000047C085518230B0F724961FAD2497612F2C
:10BD100070E0762F662766277F7725968FAD25976B
:10BD2000682B90E080E00F9431212DEC3CEC4CEC42
:10BD30005DE30F94922168C024966FAD249770E064
:10BD400090E080E00F9431216B017C0125961FADBE
:10BD5000259717FF0AC0AC019B0160E070E080E806
:10BD60009FEB0F941F236B017C011F70612F70E00C
:10BD700090E080E00F9433212DEC3CEC4CEC5DE343
:10BD80000F949221A70196010F9420232B013C01CF
:10BD9000CE018F5B9F4F0E94F7D4882309F4D7C14F
:10BDA00028968FAD28978B3030F08D30B0F18551CB
:10BDB000823008F4BAC1312C212C30ECA7963FAF69
:10BDC000A7974FE7A8964FAFA8974DC024961FADF1
:10BDD0002497612F70E090E080E00F9431216B0197
:10BDE0007C0125966FAD25976F7070E090E080E044
:10BDF0000F9433212DEC3CEC4CEC5DE30F9492213D
:10BE0000A70196010F9420232B013C0117FFC0CFFF
:10BE100077FA709477F87094BBCF23966FAD239721
:10BE200070E090E080E00F9433212DEC3CEC4CEC82
:10BE30005DE30F9492216B017C0122966FAD2297F6
:10BE400070E090E080E00F9433219B01AC01C701CA
:10BE5000B6010F942023362E272EA7968FAFA797D3
:10BE6000A8969FAFA8976EE878E082E59DE00E94D3
:10BE700031F34AE050E0D40113966C9182E59DE0E5
:10BE80000E9498F16EE778E082E59DE00E9431F330
:10BE9000B301A20182E59DE00E9433C667E778E026
:10BEA00082E59DE00E9431F3432D522DA7966FADA0
:10BEB000A797A8967FADA89782E59DE00E9433C61C
:10BEC00065E778E082E59DE00E9431F382E59DE040
:10BED0000E947BF1F4010081118161ED75E0C801E0
:10BEE0000E9427C1AD969FAF8EAFAD9766ED75E00E
:10BEF000C8010E9427C1AF969FAF8EAFAF97A30135
:10BF00009201C301B2010F94942481111FC01982C0
:10BF10001A821B821C828A818F708067F82E8A8326
:10BF2000242D4D825E826F827886B12CA12CD12C7B
:10BF3000C12CE9800B811C813E814F8158856FEFB8
:10BF4000AD968EAD9FADAD970F941211232D322D6E
:10BF5000A7964FADA797A8965FADA897632D722DB2
:10BF6000A7968FADA797A8969FADA8970F949424F6
:10BF7000811127C019821A821B821C828A818F70CC
:10BF80008067F82E8A83232D832D922DA796AFAD3F
:10BF9000A797A896BFADA8978D839E83AF83B887D8
:10BFA000B12CA12CD12CC12CE9800B811C813E81AC
:10BFB0004F8158856FEFAF968EAD9FADAF970F94C1
:10BFC000121169E475E0D4018D919C910E9427C102
:10BFD0007C01009709F4A1C0FC0180858F7084303A
:10BFE00009F09BC020E030E0A901C301B2010F9429
:10BFF0002C21882309F491C020E030E0A901632DB1
:10C00000722DA7968FADA797A8969FADA8970F946E
:10C010002C21882309F481C0A3019201C301B2013C
:10C020000F942C21811179C0232D322DA7964FAD6D
:10C03000A797A8965FADA897632D722DA7968FAD91
:10C04000A797A8969FADA8970F942C21811165C042
:10C050001A821982FE0133968EE3DF011D928A95C2
:10C06000E9F7F7016185728540E450E08E010F5FCA
:10C070001F4FC8010F9488276FE270E0C8010F942A
:10C080004F27892B51F4D70119962D913C9143E00C
:10C0900050E060E4C8010F940D0E6AED75E0C80130
:10C0A0000F944427B301A201CE018C5A9F4F0F94E5
:10C0B000FD0E0E9445C1882351F08091680E8111C8
:10C0C00006C0BE016C5A7F4FC8010E9486D2F8019B
:10C0D00001900020E9F73197E01BF10BEC0FFD1FF9
:10C0E00088E48083432D522DA7966FADA797A8961D
:10C0F0007FADA897CE018C5A9F4F0F94FD0E0E94E2
:10C1000045C1882351F08091680E811106C0BE019F
:10C110006C5A7F4FC8010E9486D20E949DD1AB010C
:10C12000BC01C4010E941316F5C923966EAD7FAD04
:10C13000239776276727762790E080E00F943121B8
:10C140002DEC3CEC4CEC5DE30F94922184CE312C31
:10C15000212CF0ECA796FFAFA7972FE7A8962FAF5B
:10C16000A89781CE0E949DD12B013C01C4010E9461
:10C170003A16A12CB12C650118E9E12E1AE3F12E33
:10C1800000E010E0A30192010F94EE0C882309F463
:10C19000C1C9D4011496ED91FC9115978181139634
:10C1A0001C91811157C0163008F03FC08CE0EAE2C4
:10C1B000F2E0DE01119601900D928A95E1F7E12FF0
:10C1C000F0E0EE0FFF1FCC24C394D12CCC0EDD1E6B
:10C1D000EC0DFD1D60E080810E9422CF6AE876E1CF
:10C1E00083E01330C9F070F462E976E181E0113048
:10C1F00099F06EE876E182E0123071F066E976E15E
:10C2000080E00AC066E876E184E0143029F062E854
:10C2100076E185E0153091F70E9403C8D4011496A9
:10C22000ED91FC9181E0818375C966EE78E082E54D
:10C230009DE00E9431F34AE050E0F401638182E521
:10C240009DE00E9498F169EB78E082E59DE00E9414
:10C2500031F360C924E0129FF0011124EC52F74F32
:10C26000C080D180E280F38065EB78E082E59DE0DC
:10C270000E9431F34AE050E0D40113966C9182E5BC
:10C280009DE00E9498F161EA78E082E59DE00E94DD
:10C2900031F32AE030E0B701A60182E59DE00E947B
:10C2A0003AF269E475E0F401808191810E9427C12E
:10C2B0008C01009709F443C0DC0118968C91189703
:10C2C0008F708430E1F519966D917C9140E450E0D7
:10C2D000CE0101960F9488276FE270E0CE0101969F
:10C2E0000F944F27892B51F4F8012185328543E0C3
:10C2F00050E060E4CE0101960F940D0EFF92EF9294
:10C30000DF92CF9285E595E09F938F938E010F5B2F
:10C310001F4F1F930F930F94DF270E9445C10FB645
:10C32000F894DEBF0FBECDBF882309F4F6CE80910E
:10C33000680E8111F2CEB801CE010196ECCE62E911
:10C3400078E083CF0E949DD12B013C01C4010E9463
:10C350003A16A12CB12C650110E3E12E15E7F12E60
:10C3600000E010E0A30192010F94EE0C882309F481
:10C37000D1C869E475E0D4018D919C910E9427C1D8
:10C380008C01009709F4C9CEFC0180858F70843040
:10C3900009F0C3CE0E949DD12AE0AE014F5F5F4FEE
:10C3A0000F94DB1B0E9445C1882309F4B6CE80910F
:10C3B000680E8111B2CEBE016F5F7F4FD801199612
:10C3C0008D919C91A8CE8FEF9FEFCA58DF4F0FB68B
:10C3D000F894DEBF0FBECDBFDF91CF911F910F91BB
:10C3E000FF90EF90DF90CF90BF90AF909F908F9095
:10C3F0007F906F905F904F903F902F90089580E0D6
:10C4000090E0DC01F40124813581F90142815381FE
:10C41000052E000C660B770B481759076A077B0738
:10C4200009F478C81C01D4016D907C9064E475E037
:10C43000C3010E9427C18C0169E475E0C3010E9419
:10C4400027C17C010115110519F4892B09F489CA4A
:10C450006EE075E0C3010E9427C12C0169E075E020
:10C46000C3010E9427C13C016AE678E082E59DE0B5
:10C470000E9431F34AE050E0F401638182E59DE0DF
:10C480000E9498F168E678E082E59DE00E9431F331
:10C490004AE050E0B10182E59DE00E9482F282E52F
:10C4A0009DE00E947BF1E114F10409F4FFC9D7017A
:10C4B00018968C9118978F70843009F0F7C91996E7
:10C4C0006D917C9140E450E0CE0101960F94882755
:10C4D0000E9445C1882309F4E9C98091680E811141
:10C4E000E5C96FE270E0CE0101960F944F27892BCA
:10C4F00051F4F7012185328543E050E060E4CE013C
:10C5000001960F940D0E2114310409F431CA41141F
:10C51000510439F0D20118968C918F70843009F44F
:10C52000BEC96CE776E0CE0101960E946BD2BEC90F
:10C53000EF92FF920F931F93CF93DF93EC018B0148
:10C540001D821C821A821B82E880F980E114F104AA
:10C5500009F45DC080911E0990911F09892B09F48F
:10C5600056C0672B09F48701F80180858F708630EB
:10C57000A9F46AED75E0C8010E9427C1009719F07F
:10C58000FC0181858A8361E376E0C8010E9427C1AE
:10C59000009709F443C0FC0181858B836CED75E045
:10C5A000C7010E9427C1009779F56DE578E082E523
:10C5B0009DE00E9431F34AE050E06B8182E59DE00E
:10C5C0000E9498F16BE578E082E59DE00E9431F3EE
:10C5D0004AE050E06A8182E59DE00E9498F182E5A0
:10C5E0009DE00E947BF120E030E0A9016CED75E058
:10C5F000888199810E94C6C76CED75E08881998118
:10C600000E9427C1009719F009969D838C83DF91C2
:10C61000CF911F910F91FF90EF900895F8018081C5
:10C6200091810F94CB1AB9CFAF92BF92CF92DF9284
:10C63000EF92FF920F931F93CF93DF93CDB7DEB7A7
:10C64000C554D1090FB6F894DEBF0FBECDBF80919F
:10C65000CF089091D008A091D108B091D208892B31
:10C660008A2B8B2B09F4CCC00E949DD19B01AC017D
:10C670006091CF087091D0088091D1089091D20834
:10C68000A12CB12C65011CE2E12EFF24F39400E003
:10C6900010E00F94EE0C882309F4B2C01092CF087A
:10C6A0001092D0081092D1081092D20880911309EC
:10C6B00090E0959587959595879510E000E0E1E0ED
:10C6C000F0E08017910709F49BC09F01002E02C083
:10C6D000220F331F0A94E2F7C090CB08D090CC0809
:10C6E000E090CD08F090CE08A901032E000C660B57
:10C6F000770B4C215D216E217F21452B462B472B4B
:10C7000009F4DCC04091CB085091CC086091CD0871
:10C710007091CE0820953095C901330FAA0BBB0B41
:10C7200084239523A623B7238093CB089093CC082A
:10C73000A093CD08B093CE08809116099091170967
:10C74000009709F45DC0FC0120852F70253009F0A9
:10C7500057C0602F0E949FC1FC0190859F7094304C
:10C7600009F04EC0618572856115710509F448C0F4
:10C77000E0911409F0911509000F111F000F111F0E
:10C78000E00FF11F13810281F180E080CE0101965C
:10C790000E94D838E11046C0F11044C0011142C0D7
:10C7A000111140C01EA21FA218A619A61AA61BA6E8
:10C7B0001CA61DA68FA18F708FA362E0CE01869666
:10C7C0000E941F1B2E8F3F8F48A359A36AA37BA3F0
:10C7D0008CA39DA361E0CE014E960E94F81AA12C75
:10C7E000CC24C394F12CE12C89019A01AB01BC014A
:10C7F000CE0101960E94563FCE0101960E946439F7
:10C80000CB5BDF4F0FB6F894DEBF0FBECDBFDF911D
:10C81000CF911F910F91FF90EF90DF90CF90BF903D
:10C82000AF9008951EA21FA218A619A68FA18F70FF
:10C8300080658FA3ECA6FBA60AA71DA78AA59BA5CA
:10C84000ACA5BDA54EA15FA168A579A54E8F5F8F50
:10C8500068A379A38AA39BA3ACA3BDA362E0CE0186
:10C860004E960E94F81AA12CCC24C394F12CE12CF2
:10C8700089019A01AB01BC01CE0101960E94563F8D
:10C880001EA21FA218A619A61AA61BA61CA61DA6A4
:10C890008FA18F708FA361E0CE0186960E941F1B2F
:10C8A0002E8F3F8F48A359A36AA37BA38CA39DA37C
:10C8B00061E0CE014E960E94F81A96CF0F5F1F4F8F
:10C8C00000CF4F925F926F927F92AF92BF92CF92C2
:10C8D000DF92EF92FF920F931F93CF93DF93CDB729
:10C8E000DEB76D970FB6F894DEBF0FBECDBF2091B7
:10C8F0001E0930911F09FF24F394232B09F420C152
:10C90000811149C0FF24F3946AEB71E182E59DE057
:10C910000E9431F382E59DE00E947BF180910A093B
:10C920008F5F80930A09E091830EF091840E309717
:10C9300009F48DC0068117810115110509F491C014
:10C94000D80118968C918F70853009F5C8010E9426
:10C9500031C28823E1F0F80160817181CE01019636
:10C960000E94D838CE0101960E94622D882359F08A
:10C970008A859B85009739F0DC01ED91FC9100845C
:10C98000F185E02D1995CE0101960E946439F801D8
:10C9900002811381D1CF63EF71E182E59DE00E94B6
:10C9A00031F382E59DE00E947BF10E949DD12B0135
:10C9B0003C0180917D0E882381F10E949DD19B01D5
:10C9C000AC01A12CB12C650110E1E12E17E2F12E92
:10C9D00000E010E0C301B2010F94EE0C81111DC004
:10C9E0000E945DF68091870E811128C00E94146319
:10C9F0008091810E9091820E059741F08091830E77
:10CA00009091840E892B11F00E94B3AB0E947FACF1
:10CA100082E090E00E94D2A4CCCF80917D0E88234A
:10CA200009F470CF60ED71E18BEA9CE00E9431F374
:10CA30008BEA9CE00E947BF1F12C66CF8091850E01
:10CA40009091860E892B91F20E94F9A1CFCF6AEACC
:10CA500071E182E59DE00E9431F382E59DE00E9454
:10CA60007BF110921D0910921C0962EA71E182E5C6
:10CA70009DE00E9431F382E59DE00E947BF164E637
:10CA800070E080E090E00E946AD110922509109237
:10CA90001B096AE871E182E59DE00E9431F30F9481
:10CAA000560FAB01BC012AE030E082E59DE00E9418
:10CAB00096F180911E0990911F09009711F00E9434
:10CAC000F1CA10921F0910921E091092800E109246
:10CAD0007F0E1092840E1092830E1092670E1092A9
:10CAE000660E10921909109218091092650E109294
:10CAF000640E10921709109216091092860E109269
:10CB0000850E109222091092210965E871E182E5F3
:10CB10009DE00E9431F30F94560FAB01BC012AE057
:10CB200030E082E59DE00E9496F182E59DE00E9462
:10CB30007BF110921A0980910A09815080930A09A9
:10CB40008F2D6D960FB6F894DEBF0FBECDBFDF916F
:10CB5000CF911F910F91FF90EF90DF90CF90BF90FA
:10CB6000AF907F906F905F904F900895FC0161159A
:10CB7000710519F4848195810895868197816817DC
:10CB800079072CF084819581860F971F0895828103
:10CB900093810C94542E4F925F926F927F928F925A
:10CBA0009F92AF92BF92CF92DF92EF92FF920F933C
:10CBB0001F93CF93DF93CDB7DEB7CD52D1400FB6E1
:10CBC000F894DEBF0FBECDBF2091810E3091820E52
:10CBD000F9013B96EB31F10508F0A0C68827EC502F
:10CBE000FA498F4F0D94ED2247733A738E6C8E6C19
:10CBF0008E6C8E6C8E6C8E6C8E6C8E6C8E6C0F66EA
:10CC00001F6E266E326E806E367235738E6C8E6C31
:10CC10008E6C8E6C8E6C6673C273E973DC7380915C
:10CC2000BE0A8093B10A8091010281110E9469FAC3
:10CC300060E08EE290E00E944AFA80FF6FC685ECC9
:10CC400094E0CC5DDE4F99838883C452D140CA5DA5
:10CC5000DE4F188219821A821B82C652D140C25EF0
:10CC6000DE4F99838883CE51D140C05EDE4F18825B
:10CC700019821A821B82C052D140C85EDE4F99834E
:10CC80008883C851D140C65EDE4F188219821A824D
:10CC90001B82CA51D140CE5EDE4F99838883C25138
:10CCA000D140CC5EDE4F188219821A821B82C45199
:10CCB000D14067EA73E181EA9CE00E9431F381EAA6
:10CCC0009CE00E947BF180917D0C90917E0C8E0106
:10CCD0000F571F4F892B09F46FC00E945FC2882332
:10CCE00009F46AC0A0917D0CB0917E0C52961C9202
:10CCF0001E92519754961C921E92539784E890E08E
:10CD00001D969C938E931C971E961C921E9782E7ED
:10CD100055968C935597ED91FC9111970088F18968
:10CD2000E02D60E170E0CD011995BE016F5F7F4F8E
:10CD300080917D0C90917E0C0E9441C289819A81E4
:10CD4000AB81BC81CA5DDE4F88839983AA83BB8394
:10CD5000C652D14080917D0C90917E0CDC01ED910A
:10CD6000FC910488F589E02D1995CA5DDE4F888114
:10CD7000C652D140882301F18F3FA9F4C95DDE4F2F
:10CD80008881C752D1408F3F71F4C85DDE4F8881E2
:10CD9000C852D1408F3F39F4C75DDE4F8881C952F8
:10CDA000D1408F3F49F00E9444C570FFA7C18091D8
:10CDB0000C09833008F0A2C16BE973E181EA9CE0C1
:10CDC0000E9431F30FB6F894A895809160008861B5
:10CDD00080936000109260000FBE8091BC0A909119
:10CDE000BD0A009711F00F949A1986E690E00F940F
:10CDF000FE1826E6FC0111922A95E9F7FC01E55B95
:10CE0000FF4F1382128248EE53E060E070E04483EB
:10CE10005583668377832DE934E03183208328E0CE
:10CE200024873F9625EC34E03183208312821382DD
:10CE3000148215829093BD0A8093BC0A8091BE0A29
:10CE40008093B10A8091010281110E9469FA26E063
:10CE500030E045E85CE064E089E090E00E94D1FACF
:10CE600085EC94E09A8389831B821C821D821E823A
:10CE7000CE0103960F94EC0660E08EE290E00E94F3
:10CE80004AFAF12CE12C80FF9BC08091BC0A909162
:10CE9000BD0ADC0196961D921D921D921C929997D7
:10CEA000FC0112A613A614A615A69E961D921D920D
:10CEB0001D921C92D19712AE13AE14AE15AEFE9613
:10CEC00040EE5EE260E070E04083518362837383F2
:10CED000349640EA5FE060E070E040835183628313
:10CEE0007383189626E0FD01322F11923A95E9F7E7
:10CEF000AC01425F5F4F34E1FA0111923A95E9F7D4
:10CF0000E5E8FCE001900D922A95E1F7FC01E65B73
:10CF1000FF4F10820F9443037C01019709F050C02A
:10CF20006091BC0A7091BD0A625F7F4FCE0101968D
:10CF30000E9471F3CE0103960F94EC066091BC0A37
:10CF40007091BD0A665E7F4FCE0101960E9471F31B
:10CF5000CE0103960F94FC066091BC0A7091BD0A45
:10CF60006A5E7F4FCE0101960E9471F3CE01039657
:10CF70000F94F4066091BC0A7091BD0A6E5D7F4FFC
:10CF8000CE0101960E9471F38B819C81AD81BE819F
:10CF90008093B40A9093B50AA093B60AB093B70AE7
:10CFA000E091BC0AF091BD0A828993899093B90AF5
:10CFB0008093B80A848995899093BB0A8093BA0AB2
:10CFC00088E199E20FB6F894A895809360000FBEAF
:10CFD00090936000A895EF2809F41FC362EF72E1F7
:10CFE00081EA9CE00E9431F335ECE32E34E0F32E2D
:10CFF000FA82E9821B821C821D821E82CE01039668
:10D000000F94E4068B819C81AD81BE81CA5DDE4FA9
:10D0100088839983AA83BB83C652D140FA82E9826E
:10D02000CE0101960F94A10E81EA9CE00E947BF153
:10D03000CE018C5D9E4F0E94A0C38091B40A909156
:10D04000B50AA091B60AB091B70A8B839C83AD83D1
:10D05000BE83C05EDE4F88839983AA83BB83C052A0
:10D06000D140CE01825E9E4F0E9472C4FA82E98254
:10D070001B821C821D821E8224E030E0AE014D5FC7
:10D080005F4F60E081E090E00E9413FA8B819C8109
:10D09000AD81BE81C65EDE4F88839983AA83BB8340
:10D0A000CA51D140CE01885E9E4F0E94DBC4FA82F5
:10D0B000E9821B821C821D821E8224E030E0AE01C8
:10D0C0004D5F5F4F60E085E090E00E9413FA8B8136
:10D0D0009C81AD81BE81CC5EDE4F88839983AA831B
:10D0E000BB83C451D140CE018E5E9E4F0E9409C4C5
:10D0F00081E00E9400C610920C0910C265E873E13D
:10D1000081EA9CE00E9431F385EC94E09A83898364
:10D11000CA5DDE4F88819981AA81BB81C652D14008
:10D120008B839C83AD83BE83CE0101960F94A10EA9
:10D1300080917D0C90917E0C892B09F459C20E943C
:10D140005FC2882309F454C2A0917D0CB0917E0C7B
:10D1500052961C921E92519754961C921E9253976F
:10D1600084E890E01D969C938E931C971E961C92CB
:10D170001E9782E755968C935597ED91FC911197E8
:10D180000088F189E02D64E170E0CD011995BE01C0
:10D190006F5F7F4F80917D0C90917E0C0E9441C209
:10D1A00089819A81AB81BC81C05EDE4F888399837F
:10D1B000AA83BB83C052D14080917D0C90917E0C9C
:10D1C000DC01ED91FC910488F589E02D1995C05E94
:10D1D000DE4F8881C052D140882309F409C28F3FB5
:10D1E000B1F4CF5DDE4F8881C152D1408F3F79F4D9
:10D1F000CE5DDE4F8881C252D1408F3F41F4CD5D7C
:10D20000DE4F8881C352D1408F3F09F4F1C16FE7EF
:10D2100073E181EA9CE00E9431F385EC94E09A830B
:10D220008983C05EDE4F88819981AA81BB81C0520B
:10D23000D1408B839C83AD83BE83CE0101960F9436
:10D24000A10E80917D0C90917E0C892B09F4A9C1CF
:10D250000E945FC2882309F4A4C1A0917D0CB09103
:10D260007E0C52961C921E92519754961C921E92BE
:10D27000539784E890E01D969C938E931C971E967E
:10D280001C921E9782E755968C935597ED91FC91D1
:10D2900011970088F189E02D68E170E0CD011995C2
:10D2A000BE016F5F7F4F80917D0C90917E0C0E943C
:10D2B00041C289819A81AB81BC81C65EDE4F888381
:10D2C0009983AA83BB83CA51D14080917D0C9091F0
:10D2D0007E0CDC01ED91FC910488F589E02D199517
:10D2E000C65EDE4F8881CA51D140882309F459C1F6
:10D2F0008F3FB1F4C55EDE4F8881CB51D1408F3F67
:10D3000079F4C45EDE4F8881CC51D1408F3F41F427
:10D31000C35EDE4F8881CD51D1408F3F09F441C1BA
:10D320006AE773E181EA9CE00E9431F385EC94E0C6
:10D330009A838983C65EDE4F88819981AA81BB81E9
:10D34000CA51D1408B839C83AD83BE83CE010196AD
:10D350000F94A10E80917D0C90917E0C892B09F485
:10D36000E0C00E945FC2882309F4DBC0A0917D0C5D
:10D37000B0917E0C52961C921E92519754961C921C
:10D380001E92539784E890E01D969C938E931C9771
:10D390001E961C921E9782E755968C935597ED9199
:10D3A000FC9111970088F189E02D6CE170E0CD01CE
:10D3B0001995BE016F5F7F4F80917D0C90917E0C1F
:10D3C0000E9441C289819A81AB81BC81CC5EDE4FD3
:10D3D00088839983AA83BB83C451D14080917D0CFB
:10D3E00090917E0CDC01ED91FC910488F589E02D93
:10D3F0001995CC5EDE4F8881C451D140882309F451
:10D4000090C08F3FB1F4CB5EDE4F8881C551D140D3
:10D410008F3F79F4CA5EDE4F8881C651D1408F3F7D
:10D4200041F4C95EDE4F8881C751D1408F3F09F476
:10D4300078C063E773E181EA9CE00E9431F345EC38
:10D44000E42E44E0F42EFA82E982CC5EDE4F88813D
:10D450009981AA81BB81C451D1408B839C83AD83C8
:10D46000BE83CE0101960F94A10EFA82E982CC5EB2
:10D47000DE4F88819981AA81BB81C451D1408B83C1
:10D480009C83AD83BE83F801F182E082C65EDE4FED
:10D4900088819981AA81BB81CA51D14082839383BB
:10D4A000A483B583CE53DF4FF982E882C25CD040BB
:10D4B000C05EDE4F88819981AA81BB81C052D14074
:10D4C000CC53DF4F88839983AA83BB83C45CD0404D
:10D4D000CE5FDE4FF982E882C250D140CA5DDE4F96
:10D4E00088819981AA81BB81C652D140CC5FDE4F31
:10D4F00088839983AA83BB83C450D1409E012F5F48
:10D500003F4FA801BE016E537F4FCE018E5F9E4FED
:10D510000E9431CD81EA9CE00E947BF182E090E0A4
:10D520008FC085EC94E09A838983C65EDE4F488184
:10D5300059816A817B81CA51D1404B835C836D8361
:10D540007E83D8018D939C93C05EDE4F48815981C4
:10D550006A817B81C052D140F80142835383648346
:10D560007583CE53DF4F99838883C25CD040CA5DF8
:10D57000DE4F88819981AA81BB81C652D140CC53AC
:10D58000DF4F88839983AA83BB83C45CD040AE01FC
:10D590004F5F5F4FB801CE018E539F4F0E9470CDF9
:10D5A000B9CF85EC94E09A838983C05EDE4F4881D1
:10D5B00059816A817B81C052D1404B835C836D83EA
:10D5C0007E83D8018D939C93CA5DDE4F88819981BB
:10D5D000AA81BB81C652D140F80182839383A48380
:10D5E000B583BE016F5F7F4FC8010E94C2CD92CF4D
:10D5F00085EC94E09A838983CA5DDE4F88819981A6
:10D60000AA81BB81C652D1408B839C83AD83BE83EC
:10D61000CE0101960E940DCE7DCF61E373E18BEACE
:10D620009CE00E9431F362E073E18BEA9CE00E948F
:10D6300031F380910C098F5F80930C0986EF9FEF87
:10D640009093820E8093810E89E0E6E3F2E0D801A8
:10D6500001900D928A95E1F787E1F8013996DF0193
:10D660001D928A95E9F789E89CE0009731F0A801BE
:10D67000485F5F4F62E00F94500D85EC94E0CE530D
:10D68000DF4F99838883C25CD040CC53DF4F188230
:10D6900019821A821B82C45CD04082EC90E08C0F0D
:10D6A0009D1F02960F94E4060E949DD1683B7B402B
:10D6B0008105910538F464E670E080E090E00E9416
:10D6C0006AD1F2CFCC53DF4F88819981AA81BB8187
:10D6D000C45CD0408093170C9093180CA093190C45
:10D6E000B0931A0CC8010E94E1CC892BC9F0E090DC
:10D6F000130CF090140CD701ED91FC91C088D188E7
:10D7000062E072E0CE0101960E9471F349EE54E1AD
:10D71000BE016F5F7F4FC701F6011995811169C284
:10D7200061ED72E18BEA9CE00E9431F38BEA9CE0B0
:10D730000E947BF127E2A22E2CE0B22E7501D12CA3
:10D74000C12CD7018D919C91892B49F1960143E021
:10D7500050E060E070E0CB010E943BDAD701ED9130
:10D76000FC9180859185009711F00F949A19D7014B
:10D77000ED91FC9186819781009711F00F949A1991
:10D78000D701ED91FC91848195810F949A19F7014D
:10D79000808191810F949A19D7011D921C92BFEF3D
:10D7A000CB1ADB0AE2E0EE0EF11CF8E0CF16D10452
:10D7B00041F686E0E6E5F2E09E012F5F3F4F49012A
:10D7C000D90101900D928A95E1F7FE0137968AE121
:10D7D000DF011D928A95E9F785E89CE0009731F01A
:10D7E000AE014A5F5F4F66E00F94500D6FED75E03C
:10D7F000C8010F944427D12CC12CF501819191913E
:10D800005F01892B09F0FEC18AE090E00F94FE18B9
:10D810007C01009709F4F6C1DC0119961C921E9256
:10D82000189715961C921E921497F80101900020EB
:10D83000E9F7CF010197801B910B0F94FE185C0153
:10D84000D70115969C938E931497892B11F40C9401
:10D850007774F40101900020E9F7CF01019788194E
:10D8600099090F94FE18D70119969C938E931897D7
:10D87000009711F40C947474B4010F94632780E53D
:10D8800090E0F7019183808313821282B801C50171
:10D890000F946327F50101900020E9F73197AE1648
:10D8A000BF0620F4319781818E32C9F75F0122E0F3
:10D8B000A20EB11CD5010D900020E9F7CD018A1907
:10D8C0009B090B960F94FE184C01F70197838683F2
:10D8D000009741F0B5010F94632766EE75E0C4012F
:10D8E0000F944427F601EE0FFF1FE95DF34FF1821D
:10D8F000E082960142E050E060E070E0CB010E94DF
:10D900003BDA019709F487C162EF75E08BEA9CE08E
:10D910000E94CBF28BEA9CE00E947BF10FB6F89458
:10D92000A8958091600088618093600010926000EB
:10D930000FBE8091810E9091820E02970CF432C13D
:10D9400080910C0981112EC160E08EE290E00E946E
:10D950004AFA80FF99C70091BC0A1091BD0A0115CF
:10D96000110509F41FC10E949DD14B015C01F80112
:10D9700082AD93ADA4ADB5AD98012A5B3F4F79015F
:10D98000892B8A2B8B2B09F466C7F9018081918141
:10D99000A281B381A5019401281B390B4A0B5B0BB3
:10D9A000CA01B90197FD52C028EE33E040E050E0D3
:10D9B0000F949822C65DDE4F688379838A839B83A8
:10D9C000CA52D1402401350188EE480E83E0581E2A
:10D9D000611C711CC65DDE4F88819981AA81BB8163
:10D9E000CA52D140481A590A6A0A7B0AD7014D9295
:10D9F0005D926D927C921397BA01A9014F5F5F4FC0
:10DA00006F4F7F4FF80182A993A9A4A9B5A96A0114
:10DA10007B01CC0CDD1CEE1CFF1C8C159D05AE059E
:10DA2000BF050CF003C712AA13AA14AA15AAF8017D
:10DA300086A997A9A0ADB1AD8C159D05AE05BF0512
:10DA40000CF0FDC616AA17AA10AE11AE6801FAE4D2
:10DA5000CF0ED11CD6018C91833009F0F9C6F801A4
:10DA600082A993A9A4A9B5A9181619061A061B0616
:10DA70000CF4EEC684E0D6018C93C8010F944303E6
:10DA800001967C01F6018081833011F0811117C06D
:10DA9000F80186A997A9A0ADB1AD181619061A0606
:10DAA0001B066CF0D6011C9284E13E96DF011D92AC
:10DAB0008A95E9F7C8010F94430303967C01D801C6
:10DAC000DA968D929D92AD92BC92DD97B2E0EB1604
:10DAD000F10429F0E4E0EE16F10409F050C0609181
:10DAE000BC0A7091BD0A625F7F4FCE0101960E9411
:10DAF00071F3CE0103960F94EC066091BC0A70910D
:10DB0000BD0A665E7F4FCE0101960E9471F3CE0181
:10DB100003960F94FC066091BC0A7091BD0A6A5E80
:10DB20007F4FCE0101960E9471F3CE0103960F94B0
:10DB3000F4066091BC0A7091BD0A6E5D7F4FCE0104
:10DB400001960E9471F38B819C81AD81BE8180938F
:10DB5000B40A9093B50AA093B60AB093B70AE091BD
:10DB6000BC0AF091BD0A828993899093B90A809387
:10DB7000B80A848995899093BB0A8093BA0AF3E026
:10DB8000EF16F10409F494C60CF073C631E0E31605
:10DB9000F10409F48AC66BE475E142E0E416F1048D
:10DBA00009F489C688E199E20FB6F894A8958093A4
:10DBB00060000FBE909360002091810E3091820E24
:10DBC000C901C35DDE4F0FB6F894DEBF0FBECDBFF7
:10DBD000DF91CF911F910F91FF90EF90DF90CF9049
:10DBE000BF90AF909F908F907F906F905F904F907D
:10DBF000089569EB72E181EA9CE00E9431F381EAC9
:10DC00009CE096CDFFEFCF1ADF0A28E0C216D104C0
:10DC100009F0F3CD79CE68EA72E181EA9CE00E94D6
:10DC200031F3B80181EA9CE00E94CBF261EA72E133
:10DC300081EA9CE00E9431F381EA9CE06DCE82E0B3
:10DC400090E09093820E8093810E68CE80911109AE
:10DC5000811105C00E942C1A81E08093110983E094
:10DC600090E0EFCF80917D0E8111AACF0E9444C534
:10DC700063FD36C080911A0981112FC00E9479B6C8
:10DC8000883C910519F484E090E0DBCF80911B097A
:10DC9000882359F06CE176E181EA9CE00E9431F33F
:10DCA00081EA9CE00E947BF1EECF85EC94E09A83C0
:10DCB00089831B821C821D821E82CE0103960F94D3
:10DCC000E4068B819C81AD81BE81892B8A2B8B2BB5
:10DCD00009F435C28FE090E0B4CF6CE076E1DCCFA0
:10DCE00080911B09882349F084E090E09093820E94
:10DCF0008093810E62ED75E19BCF8FE090E0F6CFCF
:10DD0000A8958091180990911909009721F00E9417
:10DD100031C2823068F46FEB75E181EA9CE00E94C9
:10DD200031F381EA9CE00E947BF187E090E089CFAB
:10DD3000C85EDE4F1882C851D140FE01EE5FFE4F33
:10DD4000119211928EE0DF011D928A95E9F70E94EF
:10DD500045C1882319F085E090E073CFE090180961
:10DD6000F0901909E114F10441F0C7010E9431C299
:10DD7000082F10E0023011055CF463EB74E18BEACC
:10DD80009CE00E9431F38BEA9CE00E947BF1A2CFE1
:10DD900070E060E0C7010E944D17009709F49CC035
:10DDA0009093650E8093640E66EA74E181EA9CE0CC
:10DDB0000E9431F36091640E7091650E81EA9CE0DF
:10DDC0000E94CBF281EA9CE00E947BF18091640E7C
:10DDD0009091650E0E94E1CC892B09F080C063E12F
:10DDE00076E08BEA9CE00E94CBF28BEA9CE00E94FA
:10DDF0007BF1E0901809F090190961E070E0C7012B
:10DE00000E944D175C010230110509F47FC062E0E9
:10DE1000C7010E949FC1FC01C184D2840330110557
:10DE200009F47DC063E070E0C7010E944D177C01DA
:10DE300080917D0C90917E0C892B09F475C00E9415
:10DE40005FC2882309F470C0A0917D0CB0917E0C54
:10DE500052961C921E92519754961C921E92539762
:10DE600084E890E01D969C938E931C971E961C92BE
:10DE70001E9782E755968C935597ED91FC911197DB
:10DE80000088F189E02D60E470E0CD0119954FE044
:10DE900050E0BE016E5F7E4F80917D0C90917E0CB4
:10DEA0000E94B4C24C0180917D0C90917E0CDC01EB
:10DEB000ED91FC910488F589E02D19958114910468
:10DEC00099F1E2E0F1E0EC0FFD1FE80DF91D108281
:10DED0008E010E5F1E4F3EC08BEC93E061CF62E976
:10DEE00074E181EA9CE00E9431F36091640E7091CC
:10DEF000650E81EA9CE00E94CBF26BE874E181EA56
:10DF00009CE00E9431F381EA9CE071CF8BE5C82E42
:10DF100087E0D82E9E01285E3E4F790189CFAE0161
:10DF2000485E5E4F7A0184CF053011058CF264E0C3
:10DF300070E080911809909119090E944D178C0189
:10DF40006BE674E181EA9CE00E9431F381EA9CE097
:10DF50000E947BF1B092ED0AA092EC0AD092EF0AF7
:10DF6000C092EE0A82E799E39093E50A8093E40A6F
:10DF700040E150E06EE574E1CE018E539F4F0F9467
:10DF80006E1B30E020E041E050E060E2CE018F57B0
:10DF90009F4F0F940D0E40E250E065EF7FE1CE0100
:10DFA0008F579F4F0F94501B6EE374E181EA9CE002
:10DFB0000E9431F3B50181EA9CE00E94CBF26CE350
:10DFC00074E181EA9CE00E9431F34AE050E0B6013E
:10DFD00081EA9CE00E9482F265E374E181EA9CE0C0
:10DFE0000E9431F3B70181EA9CE00E94CBF260E32A
:10DFF00074E181EA9CE00E9431F3F7018081811194
:10E0000004C010E000E0F12CE12CA090640EB09070
:10E01000650E0E9445C18111B5C18091CF0A9091D2
:10E02000D00ADC01ED91FC910688F789E02D199565
:10E03000882309F487C081E090E09093DA0A809306
:10E04000D90A87E0E6E7F2E0DE01119601900D9231
:10E050008A95E1F7FE01319685E090E02191A0914B
:10E06000D10AB091D20AA80FB91F2C9301968C3017
:10E070009105A1F786E3E114F10429F086EB01157F
:10E08000110509F086EFC090D10AD090D20AF601AE
:10E0900084878091D60A85878091D50A868780906B
:10E0A000D30A9090D40AB401C5010F94811B419604
:10E0B0008816990608F07DC08091CF0A9091D00A09
:10E0C000DC01ED91FC910488F589E02D199569EF4B
:10E0D00073E18BEA9CE00E9431F36091F20A709147
:10E0E000F30A4AE050E08BEA9CE00E9482F261EE83
:10E0F00073E18BEA9CE00E9431F38BEA9CE00E9482
:10E100007BF10E949DD160930D0970930E0980935D
:10E110000F099093100980910B098F5F80930B0971
:10E1200083330CF4A0C164EB73E18BEA9CE00E94A2
:10E1300031F38BEA9CE00E947BF110920B0986EF91
:10E140009FEF7FCD6091EC0A7091ED0A8091CF0A2C
:10E150009091D00ADC01ED91FC914091EE0A509132
:10E16000EF0A6115710571F00088F189E02D1995AC
:10E17000019709F460CF8EEF9FEF9093F30A80939D
:10E18000F20AA5CF0684F785E02D25EC34E03A832A
:10E1900029834090E80A5090E90A6090EA0A70905A
:10E1A000EB0A4B825C826D827E82BE016F5F7F4F85
:10E1B000DECF4FE050E0B601C5010E947DC16C0189
:10E1C000A090D30AB090D40AB501CE018F579F4FCB
:10E1D0000F94811B8C0D9D1D0296A816B90608F49C
:10E1E0006BCF6091D10A7091D20AA601CE018F57F0
:10E1F0009F4F0E947DC16C01A090D30AB090D40AB9
:10E20000B501CE018E539F4F0F94811B8C0D9D1D28
:10E210000296A816B90608F44FCF6091D10A709102
:10E22000D20AA601CE018E539F4F0E947DC16C0180
:10E23000E114F104B9F1A090D30AB090D40AB50169
:10E24000C7010F94811B96012E5F3F4F820F931FD2
:10E25000A816B90608F430CF6091D10A7091D20A9D
:10E26000A601C7010E947DC16C0101151105D1F005
:10E27000E090D30AF090D40AB701C8010F94811B33
:10E2800096012E5F3F4F820F931FE816F90608F4A0
:10E2900013CF6091D10A7091D20AA601C8010E94E1
:10E2A0007DC16C01A601455051096091D10A709160
:10E2B000D20A80E10E94A9D10E949DD16093DB0A1D
:10E2C0007093DC0A8093DD0A9093DE0A6093DF0A84
:10E2D0007093E00A8093E10A9093E20A8091CF0A5A
:10E2E0009091D00ADC01ED91FC910084F185E02D44
:10E2F0001995892B21F50E949DD10091DF0A10917B
:10E30000E00A2091E10A3091E20A6B017C01C01A17
:10E31000D10AE20AF30A2091D70A3091D80AA8EE6E
:10E32000B3E00F94CA22C616D706E806F906B0F283
:10E330008CEF9FEF9093F30A8093F20ABDCECE014B
:10E340008E5E9E4F0E9446D6643071058105910510
:10E3500009F0B2CEE091D10AF091D20A838190E027
:10E360008111E8CF0E949DD16093DF0A7093E00A8B
:10E370008093E10A9093E20A1092E30A1092F30A62
:10E380001092F20A10920B0962E274E181EA9CE0B9
:10E390000E9431F36091640E7091650E81EA9CE0F9
:10E3A0000E94CBF281EA9CE00E947BF181E08093A5
:10E3B0001A0930E020E043E050E061E4CE0101962C
:10E3C0000F940D0E6DE276E0CE0101960F94442776
:10E3D000CE0101960E94A1D230E020E042E050E060
:10E3E00061E4CE0101960F940D0E61E376E0CE015B
:10E3F00001960F944427BE016F5F7F4F82E59DE039
:10E400000E947FF1CE0101960E94A1D230E020E06F
:10E4100041E050E061E4CE0101960F940D0E61E3FE
:10E4200076E0CE0101960F944427BE016F5F7F4FC7
:10E4300082E59DE00E947FF1CE0101960E94A1D26B
:10E4400085E090E09093820E8093810E0E949DD192
:10E4500060930D0970930E0980930F099093100932
:10E4600065E074E1E5CB8CE090E0EBCB0E949DD1C0
:10E470009B01AC0160910D0970910E0980910F090B
:10E4800090911009A12CB12C650110E4E12E1FE13F
:10E49000F12E00E010E00F94EE0C882309F43ECA40
:10E4A00030E020E043E050E061E4CE018F579F4F21
:10E4B0000F940D0E6DE276E0CE018F579F4F0F94B3
:10E4C00044270091D30A1091D40AB801CE018F5786
:10E4D0009F4F0F94811B09960817190790F10E940E
:10E4E00045C1882371F18091D90A9091DA0A019689
:10E4F00009F4B8C09093DA0A8093D90AE091D10A5E
:10E50000F091D20A8091DA0A8583E091D10AF091E4
:10E51000D20A8091D90A86836091D10A7091D20A79
:10E5200047E050E0CE018F579F4F0E947DC1AC0164
:10E53000455051096091D10A7091D20A82EA0E9435
:10E54000A9D1FE01EE53FF4F119211928EE3DF012C
:10E550001D928A95E9F71A821982FE0133968EE799
:10E56000DF011D928A95E9F730E020E041E050E0BC
:10E5700060E4CE018E539F4F0F940D0E4FE350E099
:10E5800065EF7FE1CE018E539F4F0F94501B4FE7F5
:10E5900050E06FEE7FE1CE0101960F946E1BBE013D
:10E5A0006F5F7F4FCE018E539F4F0E946BD230E042
:10E5B00020E041E050E060E4CE018E539F4F0F9485
:10E5C0000D0E4FE350E066E175E1CE018E539F4F93
:10E5D0000F94501B4FE750E06CE075E1CE010196BF
:10E5E0000F946E1B4FE750E069EF74E1CE01019686
:10E5F0000F94501BBE016F5F7F4FCE018E539F4F14
:10E600000E946BD230E020E041E050E060E4CE01B7
:10E610008E539F4F0F940D0E4FE350E06CE070E26D
:10E62000CE018E539F4F0F94501B4FE750E069EE81
:10E6300074E1CE0101960F946E1BBE016F5F7F4F98
:10E64000CE018E539F4F0E946BD286E090E0909354
:10E65000820E8093810E68EA75E181EA9CE00E9457
:10E6600031F35CC981E090E045CF0E9445C1811142
:10E6700055C909CB0E949DD160930D0970930E0975
:10E6800080930F099093100985EF9FEFDACA0E94DB
:10E690009DD19B01AC0160910D0970910E09809193
:10E6A0000F0990911009A12CB12C650118E8E12EF9
:10E6B00013E1F12E00E010E00F94EE0C882309F432
:10E6C0002DC91092820E1092810E28C90E9445C158
:10E6D000882309F44AC0E091D10AF091D20A80EE71
:10E6E0008083E091D10AF091D20A11828091CF0A01
:10E6F0009091D00A6091D10A7091D20ADC01ED911B
:10E70000FC910280F381E02D42E050E019958FEFFB
:10E710009FEF9093F30A8093F20A8091CF0A909131
:10E72000D00ADC01ED91FC910680F781E02D19956E
:10E730008091CF0A9091D00ADC01ED91FC91048880
:10E74000F589E02D19950E949DD16093DB0A7093A5
:10E75000DC0A8093DD0A9093DE0A6093DF0A7093EF
:10E76000E00A8093E10A9093E20A0E949DD16093AF
:10E770000D0970930E0980930F09909310098DE095
:10E7800090E05FCA0E949DD19B01AC0160910D0990
:10E7900070910E0980910F0990911009A12CB12C54
:10E7A000650110E1E12E17E2F12E00E010E00F9478
:10E7B000EE0C811168CAB2C80E949DD160930D0908
:10E7C00070930E0980930F09909310098EE090E0EA
:10E7D00038CA80917D0E811105C00E942FB5892B0A
:10E7E00009F051CA0E949DD19B01AC0160910D09B5
:10E7F00070910E0980910F0990911009A12CB12CF4
:10E80000650110E3E12E15E7F12E00E010E00F9412
:10E81000EE0C882309F482C865E875E18BEA9CE078
:10E820000E9431F3F0E0E0E0199578C8841B950B65
:10E83000A60BB70B82AB93ABA4ABB5ABF8C8841BEC
:10E84000950BA60BB70B86AB97ABA0AFB1AFFEC8CD
:10E85000F12CE12C17C9D501C40188519C4FAF4F51
:10E86000BF4FF90180839183A283B383F12CE12C04
:10E8700026C96CE175E154E0E516F104E1F085E0AC
:10E88000E816F10409F08EC96CE775E18BEA9CE0AB
:10E890000E9431F38BEA9CE00E947BF186EF9FEFB0
:10E8A0009093820E8093810E7DC968E675E1EECF6C
:10E8B00068E375E1EBCF81EA9CE00E9431F385ECDF
:10E8C00094E09A8389831B821C821D821E82CE0162
:10E8D00003960F94E406CE0101960F94A10E81EAEF
:10E8E0009CE00E947BF15EC9C5010F949A19D70183
:10E8F00016968D919C91009711F00F949A19F7013B
:10E9000080859185009711F00F949A19C7010F9493
:10E910009A190C94846CAF92BF92DF92EF92FF929F
:10E920000F931F93CF93DF9300D000D0CDB7DEB706
:10E930008C017B01D42EFB0184819581892BF9F018
:10E94000A080B1806FE370E0C5010F944F2700975E
:10E95000B1F09C012A193B0937FD11C050E040E09D
:10E96000B701CE0101960E9445EFBE016F5F7F4F58
:10E97000C7010E947BEECE0101960E9423EFF701B2
:10E9800084819581892BD9F1E080F18063E376E081
:10E99000C7010F945A27892B01F5F801128A118AB1
:10E9A00080E090E19587848784E890E0948B838B66
:10E9B00081E08687D58A81E090E026960FB6F894AC
:10E9C000DEBF0FBECDBFDF91CF911F910F91FF90A2
:10E9D000EF90DF90BF90AF90089560E476E0C701BC
:10E9E0000F945A27892B59F4F801128A118A148A34
:10E9F000138A84E890E0958784871686DBCF90E0C1
:10EA000080E0DBCF90E080E00895DC01ED91FC91A7
:10EA10000284F385E02D1994DF92EF92FF920F9319
:10EA20001F93CF93DF93EC010C891D89011511050C
:10EA300059F01D8A1C8AC801DF91CF911F910F9157
:10EA4000FF90EF90DF900895EC85FD858E859F8582
:10EA5000DF01A80FB91F2C91243209F055C011967F
:10EA60002C912B3709F050C00296E80FF91FF12CBA
:10EA7000E12CDF01D190DD2009F446C08DE7D816E6
:10EA8000E9F08FEFE81AF80AF4CF198A188A2C8572
:10EA90003D852115310579F08E859F85280F391F19
:10EAA000F9012081222321F001969F878E873EC0A5
:10EAB0001D861C86C0CF0FEF1FEFBDCFE114F10400
:10EAC00019F11C928E859F8502966C857D85680F55
:10EAD000791FE881F9810684F785E02DCE0119952B
:10EAE000998B888B1B8A1A8AEC85FD858E859F857C
:10EAF000E80FF91FEE0DFF1DD2828E859F850396CC
:10EB0000E80EF91EFF86EE86288939892115310520
:10EB100009F4BDCF8A899B89280F391FF90120810B
:10EB2000222309F4B2CF01969B8B8A8B022F220FEE
:10EB3000110B81CFDC011C96ED91FC911D971E9667
:10EB40008D919C91E80FF91F8081082E000C990B84
:10EB50000895DC0115968D919C91009739F0DC01A8
:10EB6000ED91FC910680F781E02D199408950097AE
:10EB7000D1F0DC011696ED91FC913097A1F08085E3
:10EB80008F70843021F481859285009771F406801E
:10EB9000F781E02D309739F080858F70843019F43B
:10EBA00081859285089590E080E0089583E090E06B
:10EBB0000895DC011296ED91FC9113973097B9F00E
:10EBC00016968D919C918430910541F08530910588
:10EBD00041F0039749F482E090E0089581E090E0ED
:10EBE000089581E190E00895808590E0089590E097
:10EBF00080E0089585E090E0089590E080E0089539
:10EC00008EE090E00895DC011296ED91FC9113974F
:10EC10003097B9F016968D919C918430910541F012
:10EC20008530910541F0039749F482E090E0089522
:10EC300081E090E0089581E190E00895808590E082
:10EC4000089590E080E0089584E190E00895DC016B
:10EC5000ED91FC910484F585E02D60E0199581E04B
:10EC600090E008958FE090E09093820E8093810E63
:10EC700088EC90E0089560EC7CE1811102C062ECC8
:10EC80007CE181EA9CE00C9431F367ED78E181EA64
:10EC90009CE00E9431F3F0E0E0E0199584EF91E010
:10ECA00008954F925F926F927F92AF92BF92DF92E0
:10ECB000EF92FF920F931F93CF93DF9300D000D07A
:10ECC000CDB7DEB77C01D62E80912509882309F4C3
:10ECD000BEC0D70114969C9180911E02891708F43A
:10ECE000B6C08091940990919509BAE06B13F0C079
:10ECF0008C5B964FFC011082D70118960D911C91E8
:10ED00000115110509F49FC0F8016185728561152F
:10ED1000710591F445805680678070848091A50AC2
:10ED20009091A60AA091A70AB091A80A4816590680
:10ED30006A067B0609F487C0D8011B964D915C9149
:10ED40001C974115510509F47EC0F70124815396A3
:10ED50008C91539790E0322F377002C0959587952C
:10ED60003A95E2F780FF6FC0A22EB12CC501887FD3
:10ED70009370892B39F451968D919C91887F937073
:10ED8000A82AB92AD8018D919C91DC01ED91FC91C2
:10ED90006115710509F486C00688F789E02D19957B
:10EDA000019709F050C06CE3F801808191810E94C5
:10EDB00033F2A50170E060E02AE0D8018D919C91CA
:10EDC0000E942FF1F8012281808191816CE777E226
:10EDD000222311F06AE777E20E9431F3D8011D96F1
:10EDE0006D917C911E978D919C910E94CBF260E277
:10EDF000F801808191810E9433F2D8011F966D91B4
:10EE00007C9150978D919C910E94CBF2F8012281C8
:10EE1000808191816FE677E2222311F069E677E243
:10EE20000E9431F364E479E0D8018D919C910E94B5
:10EE3000CBF2F80180819181DC01ED91FC91008C95
:10EE4000F18DE02D19951092950910929409D70132
:10EE500015968D919C911697009771F014963C91A0
:10EE600020911F02231740F0DC01ED91FC910190ED
:10EE7000F081E02D6D2D199581E090E026960FB67A
:10EE8000F894DEBF0FBECDBFDF91CF911F910F91E0
:10EE9000FF90EF90DF90BF90AF907F906F905F906A
:10EEA0004F9008950488F589E02D25EC34E03A83ED
:10EEB0002983D80115964D905D906D907C901897A0
:10EEC0004B825C826D827E82BE016F5F7F4F67CF17
:10EED0008F3491050CF0BBCFBDE06B1709F4B7CFB1
:10EEE0009C012F5F3F4F30939509209394098C5BD1
:10EEF000964FFC016083ABCFCF93DF93EC016BEABD
:10EF000074E282E59DE00E9431F382E59DE00E947B
:10EF10007BF1E881F9810484F585E02D60E0CE0184
:10EF2000199581E090E0DF91CF910895CF93DF9321
:10EF3000EC0164E371E282E59DE00E9431F3EA8135
:10EF4000FB810190F081E02D6081718182E59DE07F
:10EF50000E94CBF282E59DE00E947BF1E881F9817D
:10EF60000484F585E02D60E0CE01199581E090E004
:10EF7000DF91CF9108950D949A190D949A190D94DB
:10EF80009A190D949A190D949A190D949A190D9431
:10EF90009A190D949A19CF93C1E068EE73E080E05E
:10EFA00090E00E946AD14AE050E06C2F81EA9CE038
:10EFB0000E9498F1CF5FC43181F784EF91E0CF9147
:10EFC0000895FC01828193810E94E03521E030E0C8
:10EFD000823011F430E020E0C90108950F931F93AF
:10EFE000CF93DF938C01D0E0C0E001151105B1F0A3
:10EFF000BE01685A7E4DC8010F94371B892B51F40E
:10F00000FE01E45AFE4D849190E0DF91CF911F9173
:10F010000F9108952596C233D10539F781E090E02C
:10F02000F4CFCF92EF92FF920F931F93CF93DF9382
:10F0300000D000D01F921F92CDB7DEB77C010983AC
:10F040001A832B833C834D835E836F8378876BE1C8
:10F0500071E282E59DE00E9431F3CE0101960E94AB
:10F06000CD22898181112AC00A810F70013071F18E
:10F0700028F010E00230E9F5CC20E9F060E0CE01A4
:10F0800001960E94DE1DF70102811381892B69F030
:10F09000C8010E94F22D672B682B692B61F480E078
:10F0A0000F94EF0DAB01BC0103C040E050E0BA018A
:10F0B000C8010E94B12D81E090E02EC08031D0F5D2
:10F0C0008E30D8F58130C9F18230D9F16EE071E22D
:10F0D00082E59DE00E9431F34AE050E0698182E5DB
:10F0E0009DE00E9498F182E59DE00E947BF101E0A5
:10F0F00010E06EEF70E282E59DE00E9431F34AE09D
:10F1000050E0B80182E59DE00E9482F282E59DE038
:10F110000E947BF190E080E028960FB6F894DEBF65
:10F120000FBECDBFDF91CF911F910F91FF90EF9058
:10F13000CF9008958351833048F6F70102811381FF
:10F14000A7CF40E050E0BA01F70182819381B1CFAF
:10F15000FF920F931F93CF93DF93CDB7DEB76497E2
:10F160000FB6F894DEBF0FBECDBF8C01F62E8FE236
:10F1700090E09A838983FE01339688E0DF011D9237
:10F180008A95E9F7F8016681FF2011F081E0682790
:10F19000D80114968C910E94F4CEF8018781908555
:10F1A000A185B285883E9340A105B10508F491C0C0
:10F1B0006CEC76E282E59DE00E9431F3D801149672
:10F1C0006D917C914AE050E082E59DE00E9482F2E0
:10F1D00067EC76E282E59DE00E9431F36F2D70E0EE
:10F1E0004AE050E082E59DE00E9482F282E59DE0E7
:10F1F0000E947BF16EEE76E2CE0101960F942C1BFD
:10F20000F801828193810E94E035FF2009F46DC0EE
:10F210006FEB76E2843151F068EB76E2853131F0C4
:10F220006CEA76E28F3011F464EB76E2CE010B9655
:10F230000F94401B67E976E282E59DE00E9431F37E
:10F24000D8011296ED91FC9113970190F081E02D79
:10F2500060817181ED91FC910288F389E02D9E011E
:10F260002F5F3F4FAE01455F5F4FC80119954AE0E0
:10F2700050E0BC0182E59DE00E9482F265E976E201
:10F2800082E59DE00E9431F3D8011296ED91FC9148
:10F290000190F081E02D6081718182E59DE00E9406
:10F2A000CBF2BE016F5F7F4F82E59DE00E94CBF203
:10F2B00062E976E282E59DE00E9431F3BE01655F7E
:10F2C0007F4F82E59DE00E94CBF282E59DE00E94A7
:10F2D0007BF164960FB6F894DEBF0FBECDBFDF9111
:10F2E000CF911F910F91FF90089568EA76E28230E6
:10F2F00009F49CCF63EA76E299CFAF92BF92CF92A6
:10F30000EF92FF920F931F93CF93DF9300D000D023
:10F310001F921F92CDB7DEB75C0109831A832B833E
:10F320003C834D835E836F83788765EF76E282E569
:10F330009DE00E9431F3CE0101960E94CD22E1149E
:10F34000F10439F06EEE76E2C7010F94371B009797
:10F3500031F1F5010281138101151105F1F0898167
:10F3600081115DC08A818F70813009F460C048F1DD
:10F37000823029F1082F10E061ED76E282E59DE010
:10F380000E9431F34AE050E0B80182E59DE00E941E
:10F3900082F282E59DE00E947BF190E080E0289679
:10F3A0000FB6F894DEBF0FBECDBFDF91CF911F9196
:10F3B0000F91FF90EF90CF90BF90AF900895CC2029
:10F3C000C1F060E0CE0101960E94DE1D892B09F498
:10F3D00047C0C8010E94F22D672B682B692BE1F40E
:10F3E00080E00F94EF0DAB01BC01C8010E94B12D6C
:10F3F00013C0C8010E94E0358E3019F050F48130FE
:10F4000059F460E0CE0101960E94DE1D892B21F0A7
:10F41000E0CF83518330A8F381E090E0C0CF80310A
:10F42000D0F48E30B0F68130A1F28230C9F061EEB6
:10F4300076E282E59DE00E9431F34AE050E0698186
:10F4400082E59DE00E9498F182E59DE00E947BF1BB
:10F4500001E010E091CF8351833008F4BACFE7CFB9
:10F4600040E050E0BA01C8010E94B12D60E0C50142
:10F470000E94A878D1CF2F923F924F925F926F92C5
:10F480007F928F929F92AF92BF92CF92DF92EF9234
:10F49000FF920F931F93CF93DF93CDB7DEB76097A3
:10F4A0000FB6F894DEBF0FBECDBF6130710509F411
:10F4B00095C0DC0112966D917C916115710509F47E
:10F4C0008DC04C0119821A821B821C821D821E82F1
:10F4D0001F8218868A818F708A8340E052E0CE01B5
:10F4E00001960E94ED3560E0CE0101960E94DE1D7E
:10F4F0001C01F401828193810E94F22D2B013C01B9
:10F50000D40117962D913D914D915C911A97D1019F
:10F510000F94C2222FEF30E040E050E00F947622AB
:10F5200029873A874B875C870E949DD19B01AC015C
:10F5300089859A85AB85BC850097A105B10509F43D
:10F5400068C0A12CB12C65017C018D01C301B20101
:10F550000F94EE0C89874114510461047104F1F198
:10F56000D40117968D919D910D90BC91A02D8D8702
:10F570009E87AF87B88B0E949DD19B01AC018D8582
:10F580009E85AF85B8890097A105B10561F0A12CD2
:10F59000B12C65017C018D01C301B2010F94EE0C09
:10F5A000882309F451C0D40112966D907C9080E0BC
:10F5B0000F94EF0DAB01BC01C3010E94B12D2328B4
:10F5C00069F0F40184810F94D80DD40116969C91B2
:10F5D000891304C061E0C4010E94A87890E080E033
:10F5E00060960FB6F894DEBF0FBECDBFDF91CF910E
:10F5F0001F910F91FF90EF90DF90CF90BF90AF9051
:10F600009F908F907F906F905F904F903F902F9042
:10F61000089591E099879FCFB985BB23F1F060E011
:10F62000C4010E94A878F401828193810E94EC4F6A
:10F63000892BA1F640E050E0BA01D40112968D91D9
:10F640009C910E94B12DCACFF40184810F94D80DF2
:10F65000D40116969C918913DFCF232809F4BECFDD
:10F66000F40184810F94D80DD40116969C918913CE
:10F67000B5CFB985B111B2CFADCF60E08DE00C94BC
:10F68000F4CE61E08DE00C94F4CECF93DF93EC01E7
:10F6900066E876E282E59DE00E9431F36C817D812F
:10F6A0004AE050E082E59DE00E9482F260E876E266
:10F6B00082E59DE00E9431F382E59DE00E947BF1AE
:10F6C00060E08C810E9422CFE881F9810484F58575
:10F6D000E02D60E0CE01199581E090E0DF91CF91BF
:10F6E0000895CF93DF93EC016DE576E282E59DE02E
:10F6F0000E9431F36C817D814AE050E082E59DE01B
:10F700000E9482F26BE576E282E59DE00E9431F391
:10F71000EA81FB810190F081E02D6081718182E5B9
:10F720009DE00E94CBF265E576E282E59DE00E94D5
:10F7300031F382E59DE00E947BF1E881F981048C40
:10F74000F58DE02DCE0119958130910529F00297B4
:10F7500059F060E08C811AC063E070E0CE010E9435
:10F76000B66560E00E9422CF60E08C810E9422CFCB
:10F7700061E070E0CE010E94B66560E00E9422CF99
:10F7800062E070E0CE010E94B66560E00E9422CF88
:10F79000E881F9810484F585E02D60E0CE011995BA
:10F7A00081E090E0DF91CF910895EF92FF921F9357
:10F7B000CF93DF93192F7B01C82FD92FD7FF03C019
:10F7C000D195C195D10961E08C2F0E9422CF82E0B2
:10F7D000E816F10499F460E08C2F0E94F4CE67EEF5
:10F7E0007FE182E59DE00E9431F382E59DE0DF91BB
:10F7F000CF911F91FF90EF900C947BF1612FEF2838
:10F8000051F46095661F6627661F8C2F0E94F4CE08
:10F8100063EE7FE1E6CF661F6627661F8C2F0E948E
:10F82000F4CE6EED7FE1DDCFCF93DF93EC0164E7A3
:10F8300076E282E59DE00E9431F36C817D814AE0B1
:10F8400050E082E59DE00E9482F26EE676E282E57B
:10F850009DE00E9431F382E59DE00E947BF161E032
:10F860008C810E9422CF6E818C810E94F4CE8A818D
:10F870009B81009729F040E050E0BA010E94B12D31
:10F88000E881F9810484F585E02D62E0CE011995C7
:10F890008A819B810E94EC4F181619065CF40A803D
:10F8A000DB81C02D80E00F94EF0DAB01BC01CE01D8
:10F8B0000E94B12D81E090E0DF91CF910895CF9328
:10F8C000DF93EC016BE476E282E59DE00E9431F388
:10F8D0006C817D814AE050E082E59DE00E9482F2E9
:10F8E00069E476E282E59DE00E9431F3EA81FB81E2
:10F8F0000190F081E02D6081718182E59DE00E94A0
:10F90000CBF263E476E282E59DE00E9431F382E58A
:10F910009DE00E947BF18A819B81892B09F451C073
:10F920008C819D81892B09F04CC0E881F981048C80
:10F93000F58DE02DCE0119958130910529F00297C2
:10F9400059F061E08C811AC063E070E0CE010E9442
:10F95000B66561E00E9422CF61E08C810E9422CFD7
:10F9600061E070E0CE010E94B66561E00E9422CFA6
:10F9700062E070E0CE010E94B66561E00E9422CF95
:10F980008091A100887F8093A10080919100887F61
:10F99000809391008091A10082608093A10080916A
:10F9A0009100826080939100E881F9810484F5855B
:10F9B000E02D62E0CE01199581E090E0DF91CF91DA
:10F9C000089590E080E0FACFCF93DF93EC0165E2F9
:10F9D00071E282E59DE00E9431F3EA81FB810190B2
:10F9E000F081E02D6081718182E59DE00E94CBF283
:10F9F00082E59DE00E947BF1E881F9810484F58530
:10FA0000E02D62E0CE01199581E090E0DF91CF9189
:10FA10000895DC01ED91FC910484F585E02D62E010
:10FA2000199581E090E00895AF92BF92CF92DF9256
:10FA3000EF92FF920F931F93CF93DF93CDB7DEB773
:10FA400068970FB6F894DEBF0FBECDBFFC01098BDF
:10FA50001A8B2B8B3C8B4D8B5E8B6F8B788F8281BF
:10FA60009381009709F4A3C024813581232B09F4E5
:10FA70009EC0CC2009F49BC06F0170E060E00E9442
:10FA8000542E192FD601ED91FC91048CF58DE02DAB
:10FA9000C60119955C018230910509F47CC0039779
:10FAA00009F447C095E0F1E0AF16B10409F091E028
:10FAB00019861A861B861C861D861E861F86188A36
:10FAC0009295907F8A858F70892B8A87EE24EA949D
:10FAD000FE2C09891A892B893C894D895E896F8999
:10FAE000788DCE0109960E945623F1E0AF16B1043D
:10FAF00009F453C082E0A816B10409F049C06F852B
:10FB000070E0D60114968C910E945ECF61E070E0A7
:10FB1000C6010E94B6656E8570E00E945ECF62E00D
:10FB200070E0C6010E94B6656D8570E00E945ECFF0
:10FB30002FC0612F661F6627661FCE0141960E9467
:10FB4000DE1D5C01BC01D60114968C910E945ECF33
:10FB500069E676E282E59DE00E9431F3F601648178
:10FB600075814AE050E082E59DE00E9482F267E6FE
:10FB700076E282E59DE00E9431F34AE050E0B50173
:10FB800082E59DE00E9482F282E59DE00E947BF189
:10FB900081E090E00EC094E08BCF63E070E0C6019E
:10FBA0000E94B665688970E00E945ECFA8CF90E0A1
:10FBB00080E068960FB6F894DEBF0FBECDBFDF9130
:10FBC000CF911F910F91FF90EF90DF90CF90BF905A
:10FBD000AF900895CF92DF92FF920F931F93CF9330
:10FBE000DF9300D000D01F921F92CDB7DEB76C011B
:10FBF000F02E012F1A830F7010E0FF2029F001155D
:10FC0000110511F401E010E040E050E460E070E024
:10FC1000F601828193810E9469300130110591F1D2
:10FC20000230110541F0012B99F56CE674E282E592
:10FC30009DE00E9431F38A81807FA1F1F60102816B
:10FC40001381C8010E94F22D672B682B692B89F460
:10FC500001E010E0C80128960FB6F894DEBF0FBE91
:10FC6000CDBFDF91CF911F910F91FF90DF90CF908B
:10FC7000089580E00F94EF0DAB01BC01C8010E9414
:10FC8000B12DE6CFF1E0FF1681F082E0F81669F0C1
:10FC900060E674E282E59DE00E9431F382E59DE03A
:10FCA0000E947BF110E000E0D5CFF601C280D38046
:10FCB000C6010E94F22D672B682B692B49F280E068
:10FCC0000F94EF0DAB01BC01C6010E94B12DC2CF54
:10FCD000CF92DF92EF92FF920F931F93CF93DC01AD
:10FCE0001296ED91FC9160E0828193810E949FC108
:10FCF0008C01009729F0FC0180858F708530D1F050
:10FD000061EB75E28BEA9CE00E9431F38BEA9CE0A8
:10FD10000E947BF1C12CD12C90E8E92E9FEBF92EAB
:10FD2000C701B601CF911F910F91FF90EF90DF9027
:10FD3000CF900895C8010E9431C2813040F18630D1
:10FD4000A8F1893020F565E0C8010E949FC1FC013F
:10FD500090859F709330F9F4C184D284E384F48455
:10FD6000C1E060E0C8010E949FC1FC0190859F70C6
:10FD7000933009F5618572858385948520E030E0B4
:10FD8000A9010F942C2187FF1FC0C111C9CFC12C1D
:10FD9000D12C7601C5CF923049F461857285838577
:10FDA00094850F9433216B017C01DACFC0E0C12C24
:10FDB000D12C7601D6CF923039F461857285838556
:10FDC00094850F943321DACFC111AACFC12CD12C45
:10FDD0008FE7E82E83E4F82EA3CFAF92BF92CF92A5
:10FDE000DF92EF92FF920F931F93CF93DF9300D098
:10FDF00000D01F921F92CDB7DEB7DC011296ED91B5
:10FE0000FC91309709F466C022813381232B09F4D9
:10FE100061C08C01662309F46EC00E94687EE62EE4
:10FE2000B72E6C01D8011296ED91FC910190F081F2
:10FE3000E02D608171818BEA9CE00E94CBF267ED3E
:10FE400075E28BEA9CE00E9431F38BEA9CE00E9411
:10FE50007BF120E030E0A9016E2D7B2DC6010F94CF
:10FE6000342487FD37C06BEC75E28BEA9CE00E947E
:10FE700031F34E2D5B2DB6018BEA9CE00E9433C618
:10FE80008BEA9CE00E947BF1D8011296ED91FC91E7
:10FE900061E0828193810E949FC119821A821B8234
:10FEA0001C822A812F702067F22E2E2D4E2D5B2D65
:10FEB000B6014D835E836F837887B12CA12CD12C42
:10FEC000C12CE9800B811C813E814F8158856FEFE9
:10FED0000F94121128960FB6F894DEBF0FBECDBF57
:10FEE000DF91CF911F910F91FF90EF90DF90CF9016
:10FEF000BF90AF9008950190F081E02D60817181F5
:10FF000081EA9CE00E94CBF264EE75E281EA9CE01B
:10FF10000E9431F381EA9CE028960FB6F894DEBF88
:10FF20000FBECDBFDF91CF911F910F91FF90EF904A
:10FF3000DF90CF90BF90AF900C947BF16F927F9247
:10FF40008F929F92AF92BF92CF92DF92EF92FF92E9
:10FF50000F931F93CF93DF93CDB7DEB7A8970FB65C
:10FF6000F894DEBF0FBECDBF09A31AA32BA33CA3F9
:10FF70004DA35EA36FA378A7DC011496ED91FC91CD
:10FF8000309719F490E080E0C3C020813181232BA9
:10FF9000C9F34C01DC01ED91FC910284F385E02D65
:10FFA0001995029779F78AA1982F9F70E92EF12C65
:10FFB00019A1112321F0E114F10409F424C19230B4
:10FFC00009F4CDC0B8F4992309F4C9C09130B9F04F
:10FFD00067EF75E282E59DE00E9431F34AE050E070
:10FFE000B70182E59DE00E9482F282E59DE00E94D9
:10FFF0007BF1C8CF933009F43EC0993049F7D40162
:020000021000EC
:100000001296ED91FC9161E0828193810E949FC1E3
:100010003C01198E1A8E1B8E1C8E1D8E1E8E1F8EFD
:1000200018A28A8D8F708A8F198F61E0CE01499650
:100030000E94F81A1150153108F056C1E12FF0E076
:100040008827EA5DFF478F4F0D94ED2207810781D6
:1000500074817481748174817481748174814B8121
:1000600065817481748107810781748174817481D1
:10007000078107810781807F09F484CFCE018196B3
:100080000E94FF1ED4011496ED91FC916683778344
:10009000808791876DE376E282E59DE00E9431F3EF
:1000A000D4011296ED91FC910190F081E02D6081D8
:1000B000718182E59DE00E94CBF26FE276E282E5FB
:1000C0009DE00E9431F3D4011496ED91FC9146819C
:1000D00057816085718582E59DE00E9433C682E587
:1000E0009DE00E947BF1F401E480F5800E949DD1A7
:1000F000D70152966D937D938D939C935597D40120
:100100001496ED91FC918689811117C081E090E0F1
:10011000A8960FB6F894DEBF0FBECDBFDF91CF918A
:100120001F910F91FF90EF90DF90CF90BF90AF9015
:100130009F908F907F906F900895168A60E0C40121
:100140000E94ED7ED4011496ED91FC9180E090E048
:10015000A0E0B0EC86879787A08BB18BD7CF807F4C
:1001600009F410CFCE0181960E94FF1ED40114968F
:10017000ED91FC91628773878487958769E276E2C7
:1001800082E59DE00E9431F3D4011296ED91FC913D
:100190000190F081E02D6081718182E59DE00E94F7
:1001A000CBF26EE176E282E59DE00E9431F3D4016C
:1001B0001496ED91FC91428553856485758582E5A1
:1001C0009DE00E9433C682E59DE00E947BF1D40150
:1001D0001296ED91FC9162E0828193810E949FC111
:1001E000009709F493CFB12CA12CD12CC12CE9A0FC
:1001F000FAA00BA11CA12DA13EA14FA158A56FEF04
:100200000F94121183CFEE24E394F12CF8CEB12C8D
:10021000A12CD12CC12CE98CFA8C0B8D1C8D2D8D31
:100220003E8D4F8D58A16FEFC3010F9412111986A7
:100230001A861B861C861D861E861F86188A8A853E
:100240008F708A8740E050E061E070E0F4018281C5
:1002500093810E949230672B682B692BD1F46AE05E
:10026000CE0109960E941F1BB12CA12CD12CC12CB0
:1002700079018A019B01AC016FEFC3010F94121148
:1002800060E074E0D40112968D919C910E947536C5
:100290003DCF6BE0E5CF40E050E460E070E0F4017A
:1002A000828193810E946930B12CA12CD12CC12C68
:1002B000E98CFA8C0B8D1C8D2D8D3E8D4F8D58A1A8
:1002C0006FEFC3010F9412113DCFB12CA12CD12C93
:1002D000C12CE98CFA8C0B8D1C8D2D8D3E8D4F8D94
:1002E00058A16FEFC3018CCF6CE076E282E59DE010
:1002F0000E9431F34AE050E069A182E59DE00E944E
:1003000098F182E59DE00E947BF162CE2F923F92B0
:100310004F925F926F927F928F929F92AF92BF9215
:10032000CF92DF92EF92FF920F931F93CF93DF93C1
:10033000CDB7DEB7A9970FB6F894DEBF0FBECDBF1D
:100340006130710509F439C3DC011496ED91FC911B
:100350003097D9F481E090E0A9960FB6F894DEBF0B
:100360000FBECDBFDF91CF911F910F91FF90EF9006
:10037000DF90CF90BF90AF909F908F907F906F90C5
:100380005F904F903F902F90089520813181232BD3
:1003900009F31C01DC01ED91FC910284F385E02D51
:1003A00019950297B9F6F101028113810115110522
:1003B00089F2C8010E94E035823061F240E050E0ED
:1003C00061E070E0C8010E949230672B682B692BB6
:1003D00009F6D1011496ED91FC9100811181F8018B
:1003E00082AD882309F495C20E949DD169A37AA3A6
:1003F0008BA39CA3F80182A193A1A4A1B5A149A1BB
:100400005AA16BA17CA1481B590B6A0B7B0B86A5DB
:1004100097A5A0A9B1A9481759076A077B0708F44F
:1004200078C2048CF58DE02D80819181A281B38109
:100430008D8F9E8FAF8FB8A3D8019096ED91FC91D0
:100440002D8D3E8D4F8D58A1608171818281938168
:100450000F941F234B015C01F80122A533A544A58D
:1004600055A56D8D7E8D8F8D98A10F941F236B01E7
:100470007C01D80150962D913D914D915C915397FF
:10048000C501B4010F949221F80126A137A140A51E
:1004900051A50F9420232B013C01D80196964D9233
:1004A0005D926D927C929997DB96BC91BDA3B11140
:1004B00016C0F8012485358546855785C701B601E4
:1004C0000F9492219B01AC01C301B2010F941F2331
:1004D000D80196966D937D938D939C939997F8018F
:1004E00046A057A060A471A4F6A9F98FD801D796A9
:1004F000BC91BA8FF801F0ADFB8FD801D996BC91B1
:10050000BC8F298D3A8D4F2F5B2FC301B2010F9401
:10051000342418160CF035C2898D9A8DAB8DBC8DA4
:10052000F80186A397A3A0A7B1A7FDA1FF2309F413
:1005300040C2D8011C962D913D914D915C911F9721
:10054000C501B4010F9492214B015C01F80124898B
:10055000358946895789C701B6010F9492219B01BD
:10056000AC01D80196966D917D918D919C91999752
:100570000F941F23A50194010F9420236B017C018C
:100580009B01AC01698D7A8D8B8D9C8D0F942C21F4
:1005900087FD1CC0F801F2A9F98FD801D396BC9150
:1005A000BA8FF801F4A9FB8FD801D596BC91BC8F06
:1005B000298D3A8D4F2F5B2FB601C7010F942C2147
:1005C00087FD04C0C98EDA8EEB8EFC8ED8015E9654
:1005D000ED91FC91898D9A8DAB8DBC8D808391833B
:1005E000A283B3838D8D9E8DAF8DB8A1F80182A7B4
:1005F00093A7A4A7B5A789A19AA1ABA1BCA182A3E7
:1006000093A3A4A3B5A3D1011496ED91FC9186897F
:100610008823A1F0C1010E94687E6B017C0120E06B
:1006200030E0A9010F94342487FD08C0D10114964D
:10063000ED91FC91C282D382E482F5826BEA75E28D
:1006400082E59DE00E9431F3D1011296ED91FC917B
:100650000190F081E02D6081718182E59DE00E9432
:10066000CBF265EA75E282E59DE00E9431F3D101AB
:100670001496ED91FC91428553856485758582E5DC
:100680009DE00E9433C660EA75E282E59DE00E942B
:1006900031F3D1011496ED91FC914681578160852B
:1006A000718582E59DE00E9433C66CE476E082E5C8
:1006B0009DE00E94CBF2D1011496ED91FC91428114
:1006C00053816481758182E59DE00E9433C66CE9A7
:1006D00075E282E59DE00E9431F3D1011496ED911F
:1006E000FC910190F081E02D408151816281738104
:1006F00082E59DE00E9433C668E975E282E59DE0EF
:100700000E9431F3D1011496ED91FC910190F0819A
:10071000E02D448155816681778182E59DE00E94CC
:1007200033C664E975E282E59DE00E9431F3D101B0
:100730001496ED91FC910190F081E02D408551855A
:100740006285738582E59DE00E9433C6D1011496CF
:10075000ED91FC918689882331F06DE875E282E5A0
:100760009DE00E9431F382E59DE00E947BF1F10162
:1007700004811581D8011296CD90DD90ED90FC900A
:1007800015971E964D905D906D907C905197A301AA
:100790009201C701B6010F941F234B015C0120E0B9
:1007A00030E0A9010F943424181624F0B7FAB0945D
:1007B000B7F8B09420E030E040E85FE3C501B40151
:1007C0000F943424181674F040E050E460E070E0B8
:1007D000F101828193810E949230672B682B692BF3
:1007E00009F497C0D80156968C918111B3CDF101CF
:1007F0000281138161E0D80112968D919C910E9433
:100800009FC14C0120E030E0A901C301B2010F9467
:100810002C21811109C020E030E0A901C701B601F7
:100820000F94342418165CF040E050E460E070E06F
:10083000C8010E949230672B682B692B21F1198225
:100840001A821B821C821D821E821F8218868A8148
:100850008F708A8361E0CE0101960E941F1B298759
:100860003A874B875C876D877E878F87988BB12C03
:10087000A12CD12CC12C79018A019B01AC016FEF15
:10088000C4010F94121140E050E460E070E0F10107
:10089000828193810E944030D1011496ED91FC91A8
:1008A0004281538164817581198A1A8A1B8A1C8A44
:1008B0008A898F7080678A8B4D8B5E8B6F8B788F68
:1008C00062E0CE0141960E94F81A29833A834B8355
:1008D0005C836D837E838F839887B12CA12CD12C70
:1008E000C12CE988FA880B891C892D893E894F899A
:1008F000588D6FEFC4010F941211D1011496ED9130
:10090000FC9182819381A481B58186879787A08B92
:10091000B18BD1011496ED91FC91868981111ACD8C
:100920008789908D009709F415CD28EE33E0829FDA
:100930007001839FF00C929FF00C11240E949DD1B6
:100940009B01AC01F10184809580E114F10489F0F0
:1009500010E000E0D40152966D917D918D919C91B3
:100960005597A12CB12C65010F94EE0C882309F446
:10097000F1CC81E0F401868B61E0C1010E94ED7E43
:10098000E9CCD801D2968D919D910D90BC91A02D6E
:100990008EA39FA3A8A7B9A79C01AD01C301B20173
:1009A0000F942C2187FFC1CD8EA19FA1A8A5B9A529
:1009B000B7CD812C912C5401C9CD90E080E0CCCCF6
:1009C000CF93DF93EC016FE775E282E59DE00E9433
:1009D00031F3EA81FB810190F081E02D608171812A
:1009E00082E59DE00E947FF1EC81FD81309721F04E
:1009F000808191810F949A198C819D810F949A190D
:100A000070E060E08A819B810E946E2D1D821C82B5
:100A100081E090E0DF91CF910895CF93DF93EC01D7
:100A200062E576E082E59DE00E947FF140E050E0E3
:100A3000BA018A819B810E94B12DE881F9810484E9
:100A4000F585E02D60E0CE0119956D858C810E94C1
:100A5000F4CE6D858D810E94F4CE81E090E0DF912F
:100A6000CF910895CF93DF93EC0161E676E082E5C4
:100A70009DE00E94CBF2EA81FB810190F081E02DA4
:100A80006081718182E59DE00E947FF18C819D8172
:100A9000009711F00F949A1970E060E08A819B81B1
:100AA0000E946E2D1D821C8281E090E0DF91CF912B
:100AB00008952F923F924F925F926F927F928F9202
:100AC0009F92AF92BF92CF92DF92EF92FF920F93DD
:100AD0001F93CF93DF93CDB7DEB765970FB6F8942A
:100AE000DEBF0FBECDBF1C01DC0114968D919C9121
:100AF0001597892B99F41296ED91FC91FA83E9836D
:100B000089E190E00F94FE18BC0189819A810E94CE
:100B10006E2DD10115969C938E931497F10104814B
:100B200015810115110569F46CE675E28BEA9CE00C
:100B30000E9431F38BEA9CE00E947BF190E080E020
:100B4000FCC4D8011D921C920280F381E02DFD8B24
:100B5000EC8B309791F0828193819A8389830097FF
:100B600061F0DC0118968C9118978F70853029F40C
:100B7000CD010E9431C2811190C062E375E28BEA1F
:100B80009CE00E9431F361E070E0F1018481958185
:100B9000892B11F470E060E04AE050E08BEA9CE0C1
:100BA0000E9482F260E375E28BEA9CE00E9431F3DE
:100BB00061E070E0D10112968D919C91892B11F426
:100BC00070E060E04AE050E08BEA9CE00E9482F234
:100BD0006EE275E28BEA9CE00E9431F3D10112963D
:100BE000ED91FC9161E070E082819381892B11F499
:100BF00070E060E04AE050E08BEA9CE00E9482F204
:100C00006CE275E28BEA9CE00E9431F3D10112960E
:100C1000ED91FC910280F381E02D80858F7061E081
:100C200070E0853011F470E060E04AE050E08BEA5B
:100C30009CE00E9482F26AE275E28BEA9CE00E94EC
:100C400031F3D1011296ED91FC91828193810E9442
:100C500031C261E070E0823010F070E060E04AE0A4
:100C600050E08BEA9CE00E9482F28BEA9CE00E94BA
:100C70007BF166E475E28BEA9CE00E9431F38BEA3B
:100C80009CE00E947BF1D101ED91FC910484F585FB
:100C9000E02D61E0C101199551CF60E089819A8111
:100CA0000E949FC19B8B8A8B009729F0FC01808555
:100CB0008F70853039F060E175E28BEA9CE00E942C
:100CC00031F3D3CF8A899B890E9431C28150883009
:100CD00008F0AEC1E82FF0E08827EE58F9478F4FB3
:100CE0000D94ED22E487B7878A871487F286F2860F
:100CF000D9867A8667E08A899B890E949FC1FC0118
:100D000090859F70933009F045C081859285A385B9
:100D1000B48589839A83AB83BC8391E09D8366E02D
:100D20008A899B890E949FC1FC0190859F709330A6
:100D300009F049C081859285A385B4858E839F8300
:100D4000A887B98791E09D8364E08A899B890E9486
:100D50009FC1FC0180858F70833009F056C061858A
:100D60007285838594850F9405244B0163E08A89FD
:100D70009B890E949FC1FC0180858F70833009F0A0
:100D800068C081859285A385B4858E879F87A88B4F
:100D9000B98B6CC0923069F46185728583859485C6
:100DA0000F94332169837A838B839C83A1E0AD8385
:100DB000B6CF80E090E0AFE7B3E489839A83AB835A
:100DC000BC831D82ACCF9230D9F461857285838556
:100DD00094850F9433216E837F8388879987A1E060
:100DE000AD83B2CF80E090E0AFE7B3E489839A832C
:100DF000AB83BC831E821F82188619861D82A4CFF6
:100E00001E821F82188619869FCF40EC842E47E2EF
:100E1000942E49E0A42EB12C823009F0A7CF818412
:100E20009284A384B484A2CF50EC852E57E2952EF1
:100E300059E0A52EB12C80E090E0AFE7B3E48983C0
:100E40009A83AB83BC831E821F82188619861D82FB
:100E50008DCF823009F07BC0618572858385948552
:100E60000F9433216E877F87888B998B62E08A8904
:100E70009B890E949FC1FC0180858F70833009F09F
:100E80006BC0418452846384748461E08A899B8945
:100E90000E949FC1FC0180858F70833009F087C05C
:100EA00081859285A385B4858A879B87AC87BD871A
:100EB00060E08A899B890E949FC1FC0190859F7098
:100EC000933009F0AAC0C184D284E384F48420E082
:100ED00030E0A901C701B6010F942C2187FFD6C0CD
:100EE000F7FAF094F7F8F094A1E0B0E0BB8BAA8B8E
:100EF000AC89BD891496ED91FC9180858F7082300C
:100F000009F4C7C0833009F40AC280E090E0A0EA87
:100F1000B1E409C230EC832E37E2932E39E0A32EE0
:100F2000B12C80E090E0A0EAB0E48E879F87A88B88
:100F3000B98B80E090E0AFE7B3E489839A83AB8319
:100F4000BC831E821F82188619861D828FCF80E087
:100F500090E0A0EAB0E419CF823029F5618572856E
:100F6000838594850F9433212B013C018ECF20EC97
:100F7000822E27E2922E29E0A22EB12C80E090E072
:100F8000A0EAB0E48E879F87A88BB98B80E090E0C1
:100F9000AFE7B3E489839A83AB83BC831E821F824D
:100FA000188619861D82412C512C32016ECF823059
:100FB00079F561857285838594850F9433216A87DD
:100FC0007B878C879D8774CF90EC892E97E2992E32
:100FD00099E0A92EB12C80E090E0A0EAB0E48E87E1
:100FE0009F87A88BB98B80E090E0AFE7B3E489835B
:100FF0009A83AB83BC831E821F82188619861D824A
:10100000412C512C32014A865B866C867D8650CFFE
:101010001A861B861C861D864BCF923089F561850A
:101020007285838594850F9433216B017C014FCFAA
:1010300080EC882E87E2982E89E0A82EB12C80E0E3
:1010400090E0A0EAB0E48E879F87A88BB98B80E000
:1010500090E0AFE7B3E489839A83AB83BC831E82BD
:101060001F82188619861D821B8A1A8A412C512CD0
:1010700032014A865B866C867D867301620138CFB9
:101080001B8A1A8AC12CD12C760132CF1B8A1A8A6C
:101090002FCF61857285838594850F943321F80164
:1010A0006287738784879587D80116961D921D9253
:1010B0001D921C921997F8011282138214821582D4
:1010C0000E949DD1D80152966D937D938D939C93F0
:1010D0005597D1011496ED91FC91B1E0B68B908EAD
:1010E000878A61E0C1010E94ED7EF10104811581D2
:1010F000D8018D919C9167EF74E2892B09F0DDCDC9
:101100008CE390E00F94FE189D8B8C8BC8010296A7
:10111000EC89FD89978F868F0496958F848F065F63
:101120001F4F11A300A312AE12AA13AA14AA15AA44
:1011300080E090E0AFE7B3E486AB97ABA0AFB1AF90
:1011400084E690E0A0E0B0E086A797A7A0ABB1ABA3
:101150008A899B89918F808F20E030E0A901C701A7
:10116000B6010F942C2187FD8AC020E030E0A90150
:101170006A857B858C859D850F942C2187FD7FC09A
:1011800020E030E0A901C301B2010F942C2187FDBA
:1011900076C081E090E0AC89BD895B969C938E938C
:1011A0005A97E1E0DB96EC93DB97CD92DD92ED92DE
:1011B000FC9213978A859B85AC85BD85EC89FD895A
:1011C00084839583A683B78340865186628673861F
:1011D000C486D586E686F7862DEC3CEC4CEC5DE3C8
:1011E0006A857B858C859D850F9492214B015C01DE
:1011F000AC89BD8950968D929D92AD92BC925397C9
:101200002DEC3CEC4CEC5DE3C301B2010F948C235C
:101210002B013C01EC89FD89448A558A668A778ACC
:101220008A899B89019759F5A701960160E070E0D2
:10123000CB010F941F23AC89BD891C966D937D93C0
:101240008D939C931F97A501940160E070E0CB0102
:101250000F941F23EC89FD89608B718B828B938B9C
:10126000A301920160E070E0CB010F941F23AC89D1
:10127000BD8954966D937D938D939C9357970E944F
:101280009DD1EC89FD8986A497A4A0A8B1A868196E
:1012900079098A099B0962A373A384A395A3D10149
:1012A0001496ED91FC918C899D89918380830097A0
:1012B00009F4DFCCDC01DA968C91DA97811147C012
:1012C0005E96ED91FC915F97C080D180E280F380C3
:1012D000FD01C6A2D7A2E0A6F1A65C96ED91FC9115
:1012E00080819181A281B381EC89FD8982A793A736
:1012F000A4A7B5A746A857A860AC71ACA3019201FA
:10130000C701B6010F94342418169CF4AC89BD892A
:1013100096964D925D926D927C92999718C08185B8
:101320009285A385B485F80182879387A487B587C2
:10133000BBCEEC89FD8942A853A864A875A8A30177
:101340009201C701B6010F942C2187FDDFCF81E008
:10135000EC89FD8982AFFD81FF2309F474C02981E6
:101360003A814B815C816E817F81888599850F945C
:10137000342487FF68C08E819F81A885B985EC8958
:10138000FD8982AB93ABA4ABB5AB89819A81AB816C
:10139000BC8186AB97ABA0AFB1AF068D178DD801DE
:1013A000CD90DD90ED90FC90A701960169817A8146
:1013B0008B819C810F942C2187FF26C089819A8183
:1013C000AB81BC81F80180839183A283B383AC8914
:1013D000BD8996964D905D906D907C909997D6962C
:1013E000CD90DD90ED90FC90D997A7019601C301B7
:1013F000B2010F9434241816B4F4EC89FD89C6A206
:10140000D7A2E0A6F1A61FC0A70196016E817F8139
:10141000888599850F9434241816CCF68E819F8187
:10142000A885B985CFCFAC89BD89D296CD90DD9006
:10143000ED90FC90D597A7019601C301B2010F94DE
:101440002C2187FDDACF20E030E04AE754E46E85B6
:101450007F85888999890F9492210F94FE2316160F
:101460001706ECF56B01770FEE08FF08C701B60110
:101470000F9433212B013C01C501B4010F9431219C
:101480009B01AC01C301B2010F948C234B015C01A1
:10149000AC019B01AC89BD8950966D917D918D9178
:1014A0009C9153970F949221EC89FD89608B718BED
:1014B000828B938BA50194016489758986899789AC
:1014C0000F948C23AC89BD8954966D937D938D9335
:1014D0009C935797FD01C6A6D7A6E0AAF1AA68E596
:1014E00075E281EA9CE00E9431F3D1011296ED9100
:1014F000FC910190F081E02D6081718181EA9CE096
:101500000E94CBF281EA9CE00E947BF1D10114960B
:10151000ED91FC9180E090E0A0E0B0EC86879787A9
:10152000A08BB18BD101ED91FC910484F585E02D68
:1015300062E0C101199581E090E065960FB6F894DC
:10154000DEBF0FBECDBFDF91CF911F910F91FF90F6
:10155000EF90DF90CF90BF90AF909F908F907F9053
:101560006F905F904F903F902F9008952F923F92F1
:101570004F925F926F927F928F929F92AF92BF92A3
:10158000CF92DF92EF92FF920F931F93CF93DF934F
:10159000CDB7DEB7C057D1090FB6F894DEBF0FBE86
:1015A000CDBFFC0162960FAF629763961FAF639742
:1015B00064962FAF649765963FAF659766964FAF79
:1015C000669767965FAF679768966FAF68976996FB
:1015D0007FAF699786EF800F823008F4A4C4E1964C
:1015E000FFAEEEAEE197A396FFAFEEAFA397812FCC
:1015F0008F70282F30E0AB963FAF2EAFAB97002314
:1016000061F1232B09F4C0C1873039F5013109F4A8
:1016100093C1023109F4B0C10031F9F46FEF70E009
:10162000CE018F5A9F4F0E94851D2A962FAF2A9771
:101630002B963FAF2B972C964FAF2C972D965FAFE5
:101640002D972E966FAF2E972F967FAF2F97609680
:101650008FAF609761969FAF6197A396AEADBFAD18
:10166000A3971496ED91FC91309709F47DC2868082
:101670009780AD961FAE1EAEAD97A5961FAE1EAE5F
:10168000A5976F961FAE1EAE6F97712C612C512CD3
:10169000412C8114910409F473C264EB75E0C40118
:1016A0000E9427C11C0162EB78E0C4010E9427C19F
:1016B0006B969FAF8EAF6B9760E776E0C4010E9498
:1016C00027C1AF969FAF8EAFAF972114310409F4B5
:1016D0002EC16B96EEADFFAD6B97309709F427C125
:1016E000D10118968C918F70823009F020C18085CD
:1016F0008F70823009F01BC165EA76E0C4010E9458
:1017000027C1DC0119962D913D914D915C911C975B
:10171000A9962CAF3DAF4EAF5FAFA997E196EEAD66
:10172000FFADE197309709F4BBC0D401CD90DC90B8
:10173000BF01C6010F945A27892B09F0B1C06296E8
:101740008FAD6297811127C163968FAD6397807FBC
:10175000AB96EEADFFADAB97379709F0B2C18823DA
:1017600009F478C0CE018F5A9F4F0E94461F6B9696
:10177000EEADFFAD6B970185128523853485672B10
:10178000682B692B09F4BAC1023011052105310516
:1017900029F00F3F1F4F2F4F3F4F31F564E776E0A1
:1017A00082E59DE00E94CBF282E59DE00E947BF104
:1017B00021E030E040E050E06B96AEADBFAD6B97FE
:1017C00019962D933D934D935C931C9761E0CE0148
:1017D0008F5A9F4F0E941F1B29A33AA34BA35CA3C0
:1017E0006DA37EA38FA398A7CE018F5A9F4F0E940F
:1017F000461FF10161877287838794878091810EEC
:101800009091820E059731F1D401CD90DC90E12CBE
:1018100093E0F92E62960FAD629763961FAD6397C2
:1018200064962FAD649765963FAD659766964FAD0C
:10183000669767965FAD679768966FAD689769968C
:101840007FAD6997A396EEADFFADA397828193819B
:101850000E94B630AF96EEADFFADAF97309701F175
:10186000B12CA12CD12CC12C6296EFAC629763965F
:10187000FFAC639764960FAD649765961FAD65974F
:1018800066962FAD669767963FAD679768964FADA2
:10189000689769965FAD69976FEFCF010F9412114A
:1018A0006B96EEADFFAD6B9781859285A385B48570
:1018B00082309105A105B105A1F18F3F9F4FAF4F38
:1018C000BF4F79F1F10181859285A385B485A796F3
:1018D0004EAD5FADA797849F9001859F300D949F7B
:1018E000300D1124420E531EAD96EEADFFADAD97F7
:1018F000AF01FF0F660B770B481759076A077B0785
:1019000084F4AD969FAF8EAFAD97A5963FAF2EAF47
:10191000A597A7962EAD3FADA7976F963FAF2EAF79
:101920006F97A7964EAD5FADA797640E751ED40155
:1019300012968D909C90ADCE60E870E0CE018F5AEB
:101940009F4F0E94851D22962FAF229723963FAF6F
:10195000239724964FAF249725965FAF2597269619
:101960006FAF269727967FAF279728968FAF289738
:1019700029969FAF299771CE6AE070E0CE018F5A09
:101980009F4F0E94AB1E69CE41E050E0AB965FAF27
:101990004EAFAB9762CE482F50E070E060E06B96A0
:1019A000AEADBFAD6B9719964D935D936D937C93E0
:1019B0001C97813009F462C0823009F472C08091B2
:1019C000810E9091820E059761F16B96EEADFFADA1
:1019D0006B9781859285A385B4850197A105B10593
:1019E00001F5F10181859285A385B4854497A10510
:1019F000B105BCF42EE130E040E050E021873287B1
:101A0000438754876EE170E0CE018F5A9F4F0E944A
:101A1000851D29A73AA74BA75CA76DA77EA78FA70F
:101A200098AB8091810E9091820E059709F412CFA8
:101A3000F401C080D180E12C23E0F22E62960FAD3C
:101A4000629763961FAD639764962FAD6497659612
:101A50003FAD659766964FAD669767965FAD6797A2
:101A600068966FAD689769967FAD6997A396AEAD9E
:101A7000BFADA39712968D919C91EACEF10161853D
:101A80007285CE018F5A9F4F0E94851D29AF3AAFB4
:101A90004BAF5CAF6DAF7EAF8FAF21969FAF2197FD
:101AA0008ECF70E060E0CE018F5A9F4F0E94851D5F
:101AB00029AB3AAB4BAB5CAB6DAB7EAB8FAB98AFAE
:101AC0007ECF882309F4C6CE60E0CE018F5A9F4FA7
:101AD0000E94DE1D092E000CAA0BBB0BF1018187B1
:101AE0009287A387B4878091810E9091820E05978B
:101AF00009F4B0CEE12C82E0F82EA0CF023011051F
:101B00002105310559F10F3F1F4F2F4F3F4F31F145
:101B10006FE776E082E59DE00E94CBF282E59DE0F2
:101B20000E947BF122E030E040E050E06B96AEADE9
:101B3000BFAD6B9719962D933D934D935C931C9776
:101B400062E0CE018F5A9F4F0E941F1B298F3A8F50
:101B50004B8F5C8F6D8F7E8F8F8F98A3F1011186D5
:101B60001286138614864ACEA5961FAE1EAEA59782
:101B70006F961FAE1EAE6F97712C612C512C412CAD
:101B80006114710409F4CFC1C201B3010F94D922C9
:101B90004B016EEE74E282E59DE00E9431F34AE073
:101BA00050E0B30182E59DE00E9482F263EE74E2B0
:101BB00082E59DE00E9431F30FEF10E0C201B80111
:101BC0000F94D9224AE050E082E59DE00E9482F223
:101BD0006CED74E282E59DE00E9431F34AE050E052
:101BE000B40182E59DE00E9482F26EEC74E282E52F
:101BF0009DE00E9431F3A5968EAD9FADA597B801EB
:101C00000F94D9224AE050E082E59DE00E9482F2E2
